:020000040800F2
:1000000000000220697A0C08ED7A0C08E5F6060873
:10001000ED7A0C08ED7A0C08ED7A0C08000000006F
:10002000000000000000000000000000ED7A0C0855
:10003000ED7A0C0800000000ED7A0C082536050862
:10004000ED7A0C08ED7A0C08ED7A0C08ED7A0C08C4
:10005000ED7A0C08ED7A0C0899F404089DF4040874
:10006000A1F40408A5F40408A9F40408DD41040877
:10007000F141040805420408194204082D4204080D
:100080004142040855420408ED7A0C08ED7A0C0848
:10009000ED7A0C08ED7A0C08ED7A0C08ADF4040842
:1000A000ED7A0C08ED7A0C08ED7A0C08F15604088C
:1000B00005570408195704082D5704080535040886
:1000C000F9340408393504082D350408ED7A0C0894
:1000D000ED7A0C089D600408A9600408B560040866
:1000E000B1F40408ED7A0C08000000006957040818
:1000F000B9570408E1570408555704086942040831
:10010000ED7A0C08ED7A0C0841570408ED7A0C08DA
:10011000C1600408CD600408ED7A0C08AD760408CF
:100120007D42040891420408A5420408B94204082B
:10013000CD420408ED7A0C08ED7A0C08ED7A0C0833
:1001400000000000000000000000000000000000AF
:10015000E1420408F542040809430408ED7A0C085A
:100160006D35040861350408ED7A0C08ED7A0C0849
:10017000ED7A0C08ED7A0C08ED7A0C08000000000E
:10018000ED7A0C08ED7A0C08D9600408E5600408E3
:10019000ED7A0C08ED7A0C08ED7A0C08ED7A0C0873
:1001A000ED7A0C08ED7A0C08ED7A0C08ED7A0C0863
:1001B000ED7A0C08ED7A0C08ED7A0C08ED7A0C0853
:1001C000ED7A0C08ED7A0C08ED7A0C08ED7A0C0843
:1001D000ED7A0C08BD620408ED7A0C08ED7A0C0883
:1001E000ED7A0C08ED7A0C08ED7A0C08ED7A0C0823
:1001F000ED7A0C08ED7A0C08ED7A0C08ED7A0C0813
:10020000ED7A0C08ED7A0C08ED7A0C08ED7A0C0802
:100210007D57040891570408A5570408ED7A0C0887
:10022000ED7A0C08ED7A0C08ED7A0C08000000005D
:10023000ED7A0C08ED7A0C0800000000ED7A0C084D
:10024000ED7A0C08ED7A0C08ED7A0C08ED7A0C08C2
:10025000ED7A0C08ED7A0C08ED7A0C08ED7A0C08B2
:10026000ED7A0C08ED7A0C08ED7A0C08ED7A0C08A2
:10027000ED7A0C08ED7A0C08ED7A0C08000000000D
:10028000ED7A0C0800000000ED7A0C080000000078
:0802900000000000ED7A0C08EB
:08029800482B0C0001000000DE
:1002A00060A70124020800000500140080A70124B3
:1002B0000208000106035B00A0A701240110000052
:1002C00000017600C0A701240112000000017600A1
:1002D000E0A701240114000000001E0000A8012472
:1002E000011A000000000D0020A80124011B0000DD
:1002F00000002C0040A801240115000000000C00A3
:1003000060A801240116000000000C0080A8012450
:10031000011C000000000E00A0A80124011D000027
:1003200000001E00C0A801240117000000000C00FE
:10033000E0A801240118000000000E0000A901241B
:100340000119000000000C0020A90124011F000079
:1003500000000C0040A901240120000000000C0056
:1003600060A90124012901000001180080A90124CD
:100370000121000000014800A0A901240122000081
:1003800000014900C0A901240123000000014A0026
:10039000E0A901240124000000014B0000AA01246F
:1003A0000125000000014C0020AA012401260000C4
:1003B00000014D0040AA01240127000000014E0069
:1003C00060AA01240128000000014F0080AA012436
:1003D000012C000000002900A0AA0124012D010029
:1003E00000002900C0AA0124012E010000007000B5
:1003F000E0AA0124013000000000310000AB01241C
:10040000012F01000000520020AB01240131010046
:100410000001280040AB0124013201000001280046
:1004200060AB0124022A050000012C0080AB0124EE
:100430000236040000024700A0AB01240135000091
:1004400000003C00C0AB0124013800000000200087
:020000040804EE
:10000000836B5A6D12F0500F5A6D1AD1196842F471
:1000100000725A650A6812F0080FCA6816D012F406
:10002000406F15D1CA68920412D45A6D22F48072BE
:100030005A655A6DD1040BD45A6D42F001025A65CB
:100040007047D20604D4DB6CDB6C18479007ECD009
:10005000704700BF704700BF836B5A6D42F040028B
:100060005A659A6D42F004029A65704702685549D4
:1000700038B5554B554D564CAA4218BF9A420CBF45
:10008000012300238A4208BF43F001033031A2421A
:1000900008BF43F0010330348A4208BF43F0010334
:1000A0003031A24208BF43F0010330348A4208BF16
:1000B00043F0010301F55C71A24208BF43F0010364
:1000C00004F55C748A4208BF43F001033031A24258
:1000D00008BF43F0010330348A4208BF43F00103F4
:1000E0003031A24208BF43F0010330348A4208BFD6
:1000F00043F001033031A24208BF43F001038A42BA
:1001000008BF43F0010313B9324B9A4208D10423CC
:1001100080F83530136823F001031360002038BDE8
:100120002D4B2E4D1168AA4218BF9A422C4C21F03B
:100130000E0105F13C050CBF012300231160A24212
:1001400008BF43F0010311682834AA4208BF43F0F6
:10015000010321F00101A24208BF43F0010314345E
:100160001160A24208BF43F001031E498A4208BF42
:1001700043F0010313B91C4B9A4217D10123856D3B
:10018000D0E91714226801F01F0122F480728B401D
:1001900022606B60C36ED0E91921516033B11A68D7
:1001A000D0E91C1422F480721A604C6001210022F4
:1001B000036D80F8351080F83420002BAED09847BE
:1001C000ACE700BF4000024010000240280002409F
:1001D00058000240B80402401C5402580854025807
:1001E0003054025880540258945402580168002236
:1001F0000B6880F842205A0410B40ED50B6823F423
:1002000080430B6090F84130292B10D090F841309A
:100210002A2B24D05DF8044B70471B04F2D50B68E1
:1002200023F400430B6090F84130292BEED12822B3
:10023000212380F841200022036390F841300C68AC
:1002400003F02803282B14BF6FF0F2036FF0420372
:1002500023405DF8044B0B6080F840207047282253
:10026000222380F841200022036390F841300C687B
:1002700003F02803282B14BF6FF0F4036FF044033E
:1002800023405DF8044B0B6080F84020704700BFAE
:100290000023202210B4174C4363C462036380F828
:1002A000412080F842304B07026811D5526A436AF8
:1002B0001A70436A028D013343624AB1438D013A99
:1002C000013B02859BB24385436C43F004034364C6
:1002D0000368102490F84120002190F841201A680A
:1002E00022F0FE021A60DC615DF8044B80F84010D9
:1002F000704700BF0000FFFF70B5574B002590F816
:100300004120044680F84250283AC3624585436C38
:10031000022A41EA0301036841642FD890F8411092
:1003200090F84120282001F0280102F02802282915
:1003300014BFF6214621282A1A680CBFC9436FF062
:10034000F6010A4045491A6084F84100A06B226B0F
:10035000616318B1112A42D0212A40D0E06B18B154
:10036000122A51D0222A4FD094F84130602B4FF0FE
:1003700000032DD0236384F8403070BD90F84120F5
:1003800090F841201A6822F0FE021A609A699207DA
:1003900000D59D629A69D60703D49A6942F001029A
:1003A0009A6194F84120602A10D0202284F84120DC
:1003B0009A6995060AD59A69D00605D51022DA61A0
:1003C000626C42F0040262642022DA610021BDE71F
:1003D000202284F8403084F84120236370BD1A68DD
:1003E00051042CD490F83530012BBDD000221C4B89
:1003F000036584F8402090F83520022A24D080221A
:100400004265BDE8704018471A68120403D51A689F
:1004100022F400421A6090F83530012BA4D000225B
:100420000F4B036584F8402090F83520022AE6D16E
:10043000FFF71CFE0028A0D0E06B036DE1E71A680F
:1004400022F480421A60CDE7FFF710FE002894D016
:10045000A06B036DD5E700BF0000FFFFDD040408BB
:100460002D08040803689A69196810B4D40528D5C2
:100470000C0606D4416C11F00B0F1FD15DF8044B34
:100480007047416C4FF4807441F0010141645105A3
:10049000DC6120D5416C4FF48064920541F0080185
:1004A0004164DC61E6D5426C4FF4007142F0020217
:1004B0004264D961416C11F00B0FDFD05DF8044B41
:1004C0001AE7540502D50906E4D4D3E79405D1D53B
:1004D0000906E8D4CEE79205E5D4CBE7F8B590F865
:1004E00040300D46C16A012B00F008810123AE06A1
:1004F000044680F8403001D5900656D4EB0619D555
:10050000D70617D5638D9BB2002B40F0F98094F885
:100510004130B1F1007FDBB240F0D580282B40F0B4
:10052000D28029462046FFF7B3FE0023184684F800
:100530004030F8BD68071AD42F0701D516074AD4F2
:10054000A807F2D59307F0D5638D9BB2002B00F07E
:10055000FA80616A236811F8010B228D9862638D1D
:10056000013A6162013B22859BB26385DDE7530757
:10057000E2D5638D9BB26BB12268636A526A1A70CE
:10058000638D606A228D013B0130013A9BB260624B
:1005900022856385638D9BB2002BC6D111F5803F08
:1005A000C3D02046FFF722FEBFE72368202118684A
:1005B000E66A94F84120D961213A092A1ED8DFE879
:1005C00012F0C70015001D001D001D001D001D00BC
:1005D000F000C700150094F84130226803F02803AA
:1005E000282B00F0C5800823D3619EE794F84120B2
:1005F0001A6822F0FC021A60222222635A68894992
:1006000042F400425A605A680A405A609A69910757
:1006100001D500229A629A69D20703D49A6942F0FE
:1006200001029A6147047BD51A6822F480421A605D
:10063000A26B1AB111684A6892B262856A070BD53B
:100640005A6A25F00405636A1A70636A01336362AB
:10065000238D002B40F08580638D9BB21BB1636CB2
:1006600043F004036364EB061AD5C70618D5638DFF
:100670009BB2002B40F0AA8094F84130282B03D184
:10068000B6F1007F00F0C98094F8413016F5803F44
:100690002268DBB202D0292B00F0AD801023D36199
:1006A000002384F84230666C6363002E40F084803F
:1006B000E36A5D4DAB423DD194F84130202384F88C
:1006C0004130266331E794F841202368292A4FF00E
:1006D0001002DA617FF429AF11F5803F3FF425AFB6
:1006E0009A69960701D500229A629A69D5073FF563
:1006F00058AF9A6942F001029A6152E70220F8BDB0
:1007000023681022DA61636C43F00403636431F000
:1007100080737FF40AAF616C2046FFF7EDFD04E7BC
:1007200001048BD51A6822F400421A60E26B002A99
:1007300080D183E72046FFF759FD2023E56284F846
:1007400041302663F1E631F080737FF4EEAE28E7A6
:1007500094F841201A6822F0FA021A6021222263DA
:100760004CE7013B2385638D013B9BB2638573E7B7
:10077000E1689369022990699368D56836D1C3F31B
:10078000C21383EA104313F006032FD1A16C013189
:10079000A164A16C02297FF4C8AE0821A364D161D1
:1007A000C3E694F8412094F841201A6822F0FE0232
:1007B0001A600022226321E7616C2046FFF79CFD4E
:1007C00094F84130282B7FF4B0AEAAE623681022BB
:1007D000DA61636C43F00403636436F080737FF482
:1007E0005FAF616C2046FFF787FD59E7136823F080
:1007F000B803136099E61023D3619369980701D574
:10080000002393629369D90703D4936943F00103EA
:1008100093612046FFF7EAFC42E729462046FFF7AE
:1008200037FD3DE700E800FE0000FFFF836B9A6B99
:100830000AB100211165DA6B0AB10021116593F844
:100840004120602A05D000221A63002283F840204C
:1008500070470022202183F841101A63002283F898
:1008600040207047016870B4CC072DD5914A1369B8
:10087000926A03F03803102B00F0E180182B00F08F
:10088000D9804368B3F5803F00F00581002B00F06C
:100890005A81B3F5A02F874B1A6800F0678222F4C3
:1008A00080321A601A6822F480221A60824B41F268
:1008B000883C804C1D6804E01A68521B624500F2B7
:1008C0003F8122689603F7D58A0768D4CD0631D5D3
:1008D000784A1369926A03F03803082B00F0C0804D
:1008E000182B00F0B880C369724C002B00F05F81B8
:1008F0002268714B42F0800222601D6804E01A6891
:10090000521B022A00F21C812268D205F7D56B4BDC
:10091000026A1D6841F20303B3EB154FC0F0448235
:100920006368202A23F0F8430CBF43F0804343EA76
:10093000826363600D0713D543695E4C002B00F0A2
:100940001881626F5C4B42F0010262671D6804E02F
:100950001A68521B022A00F2F380626F9207F7D5E1
:100960008C0613D58369534C002B00F0118122684B
:10097000514B42F4805222601D6804E01A68521BF9
:10098000022A00F2DD8022689204F7D5490700F1BF
:100990008880436A002B40F0BC80002059E0454A23
:1009A0001369926A13F038032BD1424AC368126864
:1009B000520701D5002B4BD03E4C226822F0190281
:1009C0001A433D4B22601D6804E01A68521B022A3C
:1009D00000F2B68022685607F7D5384B02691D68C9
:1009E00041F20303B3EB154F6368C0F0028123F4B7
:1009F0007C33402A0CBF43F4003343EA0233636084
:100A000064E7182B00F0F180C3682A4C002B00F03B
:100A1000DD80226822F019021A43274B22601D68EC
:100A200004E01A68521B022A00F28A8022685207E8
:100A3000F7D5D2E702F00302022A7FF422AF1D4B62
:100A40001B689B037FF540AF4368002B7FF43CAFEE
:100A5000012070BC704702F00302012A7FF443AF0B
:100A6000144B1B68DC0502D5C369802BF0D1134CF5
:100A700041F20303026A2468B3EB144FC0F0BF8055
:100A8000202A00F09E810B4C636823F0F84343EA70
:100A9000826363604EE7074A136843F48033136050
:100AA00004E70749044B0A6842F480720A601C6834
:100AB0000CE000BF00440258802D00240010005CB0
:100AC000004802581A68121B642A39D80A68D505EA
:100AD000F8D58268012A00F06E81002A00F04E816C
:100AE000052A9F4A116F00F0748121F001011167FE
:100AF000116F21F0040111671D6841F28834984993
:100B000003E01A68521BA2421AD80A6F9207F8D55E
:100B10003FE793490A6902F03802182A00F0D580AD
:100B20000A68022B8F4B22F080720A606FD018681F
:100B30000A6892017FF531AF1A68121A022AF7D9B2
:100B4000032070BC7047864C41F28835854B226883
:100B500022F480322260226822F4802222601E6801
:100B600003E01A68921BAA42EAD822689203F8D4DA
:100B7000AAE6626F7B4B22F0010262671D6803E008
:100B80001A68521B022ADBD8626F9607F8D4E7E690
:100B90002268744B22F4805222601D6803E01A68B8
:100BA000521B022ACCD822689604F8D4EEE62268BA
:100BB0006C4B22F0800222601D6803E01A68521B11
:100BC000022ABDD82268D605F8D4B3E62268654B60
:100BD00022F0010222601D6803E01A68521B022AFB
:100BE000AED822685607F8D470E694077FF40CAFAD
:100BF000DBE623F0FE4343EA0263636066E6584C9B
:100C0000E36823F07C5343EA0263E36092E61C68E6
:100C100003E01A68121B022A92D80A689501F8D4D8
:100C20008C6A514A2240846A2243C46A42EA04120E
:100C30008A62D0E90D24013A013C5202240492B2A6
:100C400004F4FE042243046B013CC4F30804224371
:100C5000C46B013C240604F0FE4422430A63CA6AC2
:100C600022F00102CA624A6B846C6FF3CF0242EA3F
:100C7000C4024A63CA6A046C22F00C022243384C54
:100C8000CA62CA6A406C22F002020243CA62CA6A9D
:100C900042F48032CA62CA6A42F40032CA62CA6A44
:100CA00042F48022CA62CA6A42F00102CA620A6839
:100CB00042F080720A601968226890013FF56DAEBB
:100CC0001A68521A022AF7D93AE7012B8A6A0D6B81
:100CD0003FF4BEAE02F00303846AA3427FF4B8AED1
:100CE000C2F30512C36A9A427FF4B2AE036BC5F336
:100CF0000802013B9A427FF4ABAE436BC5F3462238
:100D0000013B9A427FF4A4AE836BC5F30642013BDC
:100D10009A427FF49DAEC36BC5F30665013B9D42CD
:100D20007FF496AE4B6B816CC3F3CC0399423FF4D6
:100D300034AE0B480B4BC26A22F00102C2621A6841
:100D400018688242FCD0064A536B6FF3CF0343EA24
:100D5000C1035363D36A43F00103D3621DE600BFAE
:100D600000440258802D00240CFCFFFF42F4802236
:100D70001A601A6842F480321A6097E5194941F204
:100D800088350A6F22F001020A670A6F22F0040216
:100D90000A671C6804E01A68121BAA423FF6D0AE2C
:100DA0000A6F9607F7D4F4E5E36823F07C5343EA2F
:100DB0000263E360BEE50B490A6F42F001020A6775
:100DC0009AE6084A536823F0F84343F0804353609F
:100DD000B0E541F004011167116F41F001011167A5
:100DE0008AE600BF00440258334B30B4996A9C6ACB
:100DF000DD6A14F47C7F5A6BC4F3051036D0C2F35D
:100E0000CC0205F0010501F0030107EE900A05FB95
:100E100002F20129B8EEE77A06EE902AFAEEE96AC4
:100E200002D0022942D019B3DFED247A87EE876A17
:100E30001B6BC3F3080307EE903AF7EE005AF8EE87
:100E4000E77A77EEA67A77EEA57A67EE867A1A4B7E
:100E50001B6BC3F34623013307EE103AF8EEC76A63
:100E600087EEA67AFCEEC77A17EE900A30BC704780
:100E70001A6892061DD51968F7EE005A104A1B6BC6
:100E8000C1F3C101C3F30803CA4007EE903A06EE6E
:100E9000102AF8EEE77AB8EEC66A77EEA66AC6EED2
:100EA000077A36EEA57A67EE877AD0E7DFED057A26
:100EB000BCE7DFED057AB9E7004402580024744A24
:100EC0000090D0030024F44A0024744CF0B5354A55
:100ED000B0F1804F344DA0EB02020368A0EB050E89
:100EE0004C69B2FA82F28F68BEFA8EFE0E684FEA43
:100EF00052124FEA5E1E1FD0F2B9DFF8B8C060454B
:100F000037D00CF5806C604533D00CF5806C6045B3
:100F100012D0BEF1000F0FD1244D254A904218BFC8
:100F2000A8422AD002F58062904226D023F08003A6
:100F3000C76286621C4314E04D6823F07003D1F849
:100F40000CC02B43C762866223F4407343EA0C0350
:100F500023F080031C4312B9BEF1000F16D00B69B9
:100F600003630368012243F00403036042610460E9
:100F7000F0BD23F070034A681343CA6823F440733A
:100F8000C7621343866223F080031C43074A084B61
:100F9000984218BF9042E2D003F580639842DED0B9
:100FA000DFE700BF000001400004014000400140B5
:100FB0000044014000040040836A1A0710B406D5BB
:100FC0000168846B4A6822F4004222434A60DC07CD
:100FD00006D50168C46A4A6822F4003222434A6096
:100FE000990706D50168046B4A6822F480322243CF
:100FF0004A605A0706D50168446B4A6822F4802289
:1010000022434A60DC0606D50168C46B8A6822F474
:10101000805222438A60990606D50168046C8A686A
:1010200022F4005222438A605A060AD50168446CB1
:101030004A68B4F5801F22F4801242EA04024A6032
:101040000BD01B0606D50268C16C536823F400233D
:101050000B4353605DF8044B70474A68846C22F47C
:10106000C00222434A60ECE70022836BA3F85E20B3
:10107000704700BF036942681F2B70B430D9A3F1D9
:10108000200520215468A940214227D08169087C8D
:10109000022835D048681F2BC9681B4D4E6801696E
:1010A000C1F30324194951F8244015F804C0056818
:1010B00056F80C4024F0010446F80C40407901EB4E
:1010C0004001088CE96800F4F05021EA0001E96071
:1010D00010D9A3F1200120238B40D36070BC70474E
:1010E0002021146899402142F8D08169087C0228A7
:1010F000D0D105E0202101FA03F370BC9360704762
:1011000000200874C6E700BF4CA20C0818A10C0808
:10111000D0E907239A423CBFC1685218D01A7047E1
:10112000D0E9092300699A4238BF12180138D31A4E
:10113000C01A7047D0E90902101AB0FA80F04009CD
:10114000704700BF016A034640694A1C405CD96889
:101150008A4228BF00221A62704700BF436A826930
:1011600010B4D154436A416B046901330A68A34245
:1011700028BF00235DF8044B42F0800243620A60FE
:10118000704700BF436BD86910F0100002D01022E6
:1011900001201A62704700BF704700BF704700BF50
:1011A000704700BF01207047014B5868704700BF6F
:1011B000802D0024074B93F8A422012A01D100209E
:1011C000704793F8A402A0F10300B0FA80F0400940
:1011D000704700BF802D0024012380F849307047FC
:1011E000EFF31182702383F312880849D2B2D1E958
:1011F000B93182F31188581E8B42A0EB01008CBFDD
:101200000023012300EB0330704700BF802D002432
:1012100070B5D0F8D442D0F8C86200EB840EDEF886
:10122000C05245B301F00F040A4604EB840C00EBF6
:101230008C0CDCF818306BB9DEF8C43200211B6965
:10124000C5F8141223B105F50471D5F808029847C2
:10125000002070BD04EBC40406EB8406F469B3FB04
:10126000F4F604FB1633002BE6D11A46CCF81830FE
:101270007BF05CF9ECE7032070BD00BFD0F8D4220E
:1012800000EB820210B5D2F8C042ACB101F00F03FE
:10129000D0F8C802D2F8C42204F5037103EBC303EB
:1012A000D26800EB8303D4F80402D3F86832C4F8A0
:1012B0000C329047002010BD032010BDD0F8D4326E
:1012C00000EB830010B5D0F8C04284B1D0F8C4322E
:1012D0005BB194F80002FF2807D09B68214694F880
:1012E00001229847FF2384F80032002010BD03201C
:1012F00010BD00BF30B52A4C8646237865889D42D4
:1013000041D9184619461A4602E0954246D9217835
:101310000C440A44617892B20529F6D1A178822959
:10132000F3D19C461A461E4903E0AA4234D291F8F2
:1013300000C06144624491F801C092B2BCF1050F53
:10134000F3D191F802C0BCF1010FEED1144A02E0D2
:10135000A8421DD213781A44034492F801C098B2EF
:10136000BCF1050FF4D19378812BF1D10CB110238E
:10137000A37119B10020022308714B711AB1002129
:1013800002231171537143230548AEF8003030BD7C
:101390000022002CEBD1ECE70021D7E70024C0E7C6
:1013A0000000002430B52A4C8646237865889D428B
:1013B00041D9184619461A4602E0954246D9217885
:1013C0000C440A44617892B20529F6D1A1788229A9
:1013D000F3D19C461A461E4903E0AA4234D291F842
:1013E00000C06144624491F801C092B2BCF1050FA3
:1013F000F3D191F802C0BCF1010FEED1144A02E022
:10140000A8421DD213781A44034492F801C098B23E
:10141000BCF1050FF4D19378812BF1D10CB11023DD
:10142000A37119B10020402348710B711AB100213A
:1014300040235171137143230548AEF8003030BD8D
:101440000022002CEBD1ECE70021D7E70024C0E715
:1014500000000024A6E700BF03460A2201481A80C4
:10146000704700BF44000024064B4FF0120C064AA0
:10147000A3F11400526DA1F800C0022A18BF18464B
:10148000704700BF64000024004000580423014856
:101490000B807047780000241D48D0F80038D0F841
:1014A000082830B59B184FF01A040C8001D1194858
:1014B00030BD184A0024D0F8040802F11005114686
:1014C0004FEA137EB3F1204FCC7001F102010EF10F
:1014D000370C38BF0EF1300C8D424FEA031381F800
:1014E00000C0EDD102F108050024010FB0F1204F3A
:1014F000D47402F1020201F1370338BF01F1300365
:1015000095424FEA00101374EFD1024830BD00BF7E
:1015100000E0F11F7C000024122301480B8070477B
:101520005000002400207047212808B527D0222829
:1015300018D0202814D199B1072A11D1184A194B73
:101540000868B1F804C0D2F8EC228979C3F8980091
:10155000A3F89CC083F89E1012B10146002090476A
:10156000002008BD0029FBD0022AF9D10C4BD3F88A
:10157000F032002BF4D0098800209847F0E70029CA
:10158000EED0072AECD1074BD3F89800B3F89C2093
:1015900093F89E30086000208A808B7108BD00BFE0
:1015A000802D002400000024002070471149D1F84C
:1015B00048231379022B00D0704793689B07FBD513
:1015C000D1F84C130C4B0D4810B44FF4FA7404FBD3
:1015D00001F14468A3FB0131890943681B1B99424F
:1015E000FBD2536913B11A689B8893615DF8044B71
:1015F000704700BF802D0024D34D6210001000E022
:10160000034B93F81803003818BF0120704700BF40
:10161000802D00240E4BD3F8442342B110689188EA
:101620000269114203D1002283F81823704793F80E
:101630000C230132D2B2072A83F80C23F3D8D3F853
:1016400050130122C3F8081383F81823704700BF12
:10165000802D0024034B93F81803032894BF002027
:1016600001207047802D0024004870479C300024E2
:10167000564B0021564AD3F8A0305648A2FB03230C
:1016800030B5DB0C544C83B0013BC4F86413C4F890
:101690005C1342F20F7194F89123C4F85403C4F818
:1016A0006013C4F85833002A00F08A8002254B49A1
:1016B000484884F89153FFF709FC0123484A062162
:1016C000372084F89C3384F8923384F8933384F879
:1016D000943384F8953384F8963384F8973384F8F8
:1016E000983384F8993384F89A3384F89B3384F8D8
:1016F0009133D2F8E83043F02003C2F8E830D2F852
:10170000E83003F020030193019B72F0FFFB354B9F
:101710004FF400025A6094F89133012B3BD1D4F876
:101720005423314B3148B2F1804F18BF9A4284F8AC
:101730009153D1680CBF0123002341F00101824283
:1017400008BF43F0010300F58060D160824208BF0A
:1017500043F0010300F580602549824208BF43F051
:10176000010300F57840824208BF43F001038A423A
:1017700008BF43F0010313B91E4B9A4207D1916889
:101780001D4B0B40062B06D0B3F5803F03D01368EA
:1017900043F001031360D4F8DC3204EB8303D3F885
:1017A000C83243B115480021154AC3F80802C3F8EE
:1017B0001012C3F804220020C4E9BB0003B030BDFE
:1017C00002F0FF0084F8900370E700BF00000024DF
:1017D00083DE1B4300140040802D0024D8300024F9
:1017E0000044025800E100E0000001400004004015
:1017F000001800400040014007000100944C002404
:10180000943C00242DE9F84F234E80468946D6F8B3
:10181000C432D3F81422002AFBD1B9F1000F37D01B
:1018200008EB090ADFF874B008F1FF3870270AF1F5
:10183000FF3AD6F8E82218F8011F531C0BF80210E3
:10184000C3F30B03C6F8E832EFF3118287F3128873
:10185000D6E9B931D2B282F311888B42A3EB0103EE
:101860008CBF0022012203EB0233012B0ED111F0B9
:1018700027FF04460D4611F023FF001B61EB050115
:10188000B0F57A7F71F10001F5D3DDE7D045D0D115
:101890004846BDE8F88F00BF802D0024944C0024FA
:1018A000F8B50E4E96F8A432012B00D1F8BD96F88B
:1018B000A432032BFAD10D461446D6F8507308E033
:1018C000FFF7A0FFD6F85033241A0544DB1B322B58
:1018D000ECD8002C21462846F2DCF8BD802D0024EF
:1018E000F8B590F848305D1C0344EDB280F84850DC
:1018F00083F8341090F8493053B1132D07D90023E1
:1019000080F84830104F97F8A432012B05D1F8BD6C
:1019100080F84830002DF5D1F8BD97F8A432032B9C
:10192000F5D1D7F8506300F1340429462046FFF77B
:1019300069FFD7F850332D1A04449B1B322BE6D88D
:10194000002DF2D1F8BD00BF802D0024F8B5002392
:1019500090F84850A0F8483005B9F8BD0D4F97F8F9
:10196000A432012BF9D097F8A432032BF5D1D7F884
:10197000506300F1340429462046FFF743FFD7F8AF
:1019800050332D1A04449B1B322BE6D8002DF2D184
:10199000F8BD00BF802D00242DE9F047046982B016
:1019A000C3681C4046D0814688464FF0004501F18F
:1019B000500701F13806B4FA84F325FA03F21B3B11
:1019C000D2431440C9F81020B8F1000F5FD0042BA7
:1019D0002ED8DFE803F052483D320300D8F810302B
:1019E000D9F82CA033B19B6823B11FFA8AF108F112
:1019F00008009847D8F8283033B19B6823B11FFA04
:101A00008AF108F120009847D8F8403033B19B683C
:101A100023B11FFA8AF108F138009847D8F85830F6
:101A200033B19B6823B11FFA8AF108F1500098473F
:101A3000002CC0D102B0BDE8F087D8F8103008F112
:101A40000800D9F834105B689847002CB3D1F1E74F
:101A5000D8F8283008F12000D9F838105B6898478A
:101A6000002CA8D1E6E7D8F840303046D9F83C1031
:101A70005B689847002C9ED1DCE7D8F85830384690
:101A8000D9F840105B689847002C94D1D2E7042B1A
:101A900007D8DFE803F01903140F0A00D9F83C3027
:101AA0000193019B002C86D1C4E7D9F82C30019317
:101AB000019BF7E7D9F834300193019BF2E7D9F89D
:101AC00038300193019BEDE7D9F840300193019B39
:101AD000E8E700BF0A49D1F8A0334A685BB1002AA1
:101AE000FCD0013A10B513F8014B4A60C1F8A0339D
:101AF00012B1204610BDFEE772F0CEFD204610BDAB
:101B0000802D002408B5064A0B68C2F8A003536074
:101B10000BB1002008BD72F0BFFD002008BD00BF62
:101B2000802D00242DE9F041012104464FF4077077
:101B300084F044FE054600286CD0D4F8D46204EB4F
:101B40008606C6F8C002237CC4F8BC02002B40D035
:101B500040230222812120467AF05AFA01214023B3
:101B60000222204621877AF053FA4FF00108082319
:101B7000032282212046A4F878817AF049FA294B81
:101B80000027E364D6F8C432C5F804721B6898478E
:101B9000D5F80402C5F81472C5F8187200283ED0B2
:101BA000227CD4F8C83222BBC3F88C224FF40074D4
:101BB0009A7903F51E71C3F88402012AA3F878828A
:101BC000C3F8884223D018687AF0A0FB0020BDE853
:101BD000F08120464FF40073022281217AF018FA36
:101BE00001214FF400730222204621877AF010FA77
:101BF000BBE79A79402403F51E71C3F88C72012A61
:101C0000C3F88402A3F87882C3F88842DBD1C3F812
:101C10009402D8E7D4F8D432B03344F82300022039
:101C2000BDE8F08101001000F8B5D0F8C85240F2CC
:101C30000112044695F894342A87012B3ED00126E0
:101C4000002728683246314685F894647AF0EEFC25
:101C500027873A4631462868A5F8786285F8946463
:101C60007AF0E4FC4FF48173A4F8787132460221D3
:101C7000286885F89464A5F85C307AF0D7FC85F87C
:101C80009474D4F8D432002504EB8303E564D3F8CC
:101C9000C0228AB1D3F8C4325B689847D4F8D432F2
:101CA000B03354F8230082F025FED4F8D432B03398
:101CB00044F82350C4F8BC520020F8BD00224FF471
:101CC00081710287A5F87832A0F87821A5F85C1018
:101CD000D7E700BFD0F8D43200EB8303F0B500267D
:101CE00083B0D3F8C0728DF80560ADF806605FB1BF
:101CF00091F800C004460D461CF060022FD0202A47
:101D000005D020467AF0C8FA032003B0F0BDCA8897
:101D10004878002A42D01CF0800F00F08380D3F86E
:101D2000C43239469B689847EA8802234FF4807191
:101D3000072AC4F8943228BF0722D4F8C832C4E96D
:101D400006225A629A79998203F11401012A1F62CC
:101D50009E6200D11F6318687AF0D8FA22E04B78AF
:101D60000B2BCED801A252F823F000BFA91D040806
:101D7000A51D0408031D0408031D0408031D040811
:101D8000031D0408031D0408031D0408031D0408A3
:101D9000031D0408E91D0408DF1D0408D3F8C4323C
:101DA0009B6898470020B0E790F89C32032BA8D19D
:101DB0000222D0F8C8320020C4F8942203F11401A2
:101DC000C4E906220DF106049862C3E908424FF403
:101DD00080729A829A79012ABDD11C63BBE790F880
:101DE0009C32032BDED08CE790F89C32032B88D1F9
:101DF00001220221D0F8C832C0F8941203F1140174
:101E0000C0E906220DF10500C3E908024FF4807213
:101E100000209A829A799862012A9CD10DF10500DE
:101E2000186398E7402A4FF0030387F8000228BFA1
:101E3000402287F80122C4F89432D4F8C832C4F89A
:101E40005821C4F85C2103F51571C3F864229A790E
:101E5000C3F86072012AC3F86862A3F8546208BF2D
:101E6000C3F8707277E700BF08B520B9044871F075
:101E70001BFE044808BD044871F016FE014808BD69
:101E8000DC540D082431002400550D08024808B523
:101E900071F00AFE014808BD24550D0824310024C4
:101EA000024808B571F000FE014808BD2C550D0828
:101EB00024310024024808B571F0F6FD014808BD40
:101EC00038550D082431002408B520B9044871F0B4
:101ED000EBFD044808BD044871F0E6FD014808BD6B
:101EE00048550D082431002468550D08024808B5EE
:101EF00071F0DAFD014808BD88550D082431002431
:101F0000024808B571F0D0FD014808BD94550D0890
:101F10002431002470B5134D134AD5F8A030A2FB2C
:101F200003239B09013BB3F1807F01D3012070BDE6
:101F30004FF0E0220D4900240F2853614FF0F003C9
:101F4000064681F823304FF0070394611361EDD802
:101F500001464FF0FF3071F0D9FF2046C5F8A4606C
:101F600070BD00BF00000024D34D621000ED00E002
:101F70003749024603688B4233D01831591AB1FAF7
:101F800081F1490969BB3348834240D0183083420C
:101F900040D01830834236D0183083423DD01830BC
:101FA000834240D0183083422CD000F556708342D3
:101FB00037D029498B4233D018318B4236D0183173
:101FC0008B4236D018318B4236D018318B4236D006
:101FD00018318B4236D018318B4236D023F0FF00B7
:101FE00013E0DBB21D491E48103B10B41D4CA4FB8E
:101FF00003435DF8044B01EB131393F82810C2E977
:102000001601704716211848D16590657047102158
:102010001348F9E716211248F6E706211248F3E7BC
:1020200006211248F0E710210F48EDE710210F4874
:10203000EAE716210D48E7E700210D48E4E706210D
:102040000B48E1E710210A48DEE716210848DBE7E4
:1020500010000240400002402804024018A10C0871
:1020600000000240ABAAAAAA0400024000040240F9
:1020700004040240F0B50C46114602688646936996
:1020800013F0100C72D04FF0000C10233848654646
:10209000D36193699E065FD445B903685B1AA34276
:1020A0003DD893699F06F8D52023D3614CF0040CEA
:1020B00001209369D90552D54FF480715F054CF02A
:1020C000010CD16104D54FF480614CF0080CD16152
:1020D0009D0504D54FF400734CF0020CD361936955
:1020E000990701D5002393629369DB0703D49369B1
:1020F00043F001039361536820241E4901200B40E3
:1021000000215360DEF844308EF8401043EA0C039F
:10211000CEF844308EF841408EF84210F0BD57683A
:102120009EF842309669DBB2360408D57E0406D4A8
:10213000202B04D0536843F48043536001689369B3
:102140009F06A6D403685B1A192BF8D993694FF040
:10215000200C01259E069FD5002DA5D0A6E75E0583
:10216000B1D49C05B6D40028B9D1F0BD6046A0E733
:10217000802D002400E800FE2DE9F04707689A460C
:10218000089EBB6931EA03030CBF0123002393427D
:1021900020D180460C461546DFF85C903246514609
:1021A0004046FFF767FF20BBD9F80030A3EB060CD1
:1021B000D44507D9BB6934EA03030CBF01230023CC
:1021C000AB420AD0BB6934EA03030CBF01230023EE
:1021D000AB42E3D00020BDE8F087D8F8443020229D
:1021E00088F840001343C8F8443088F8412088F844
:1021F00042000120BDE8F087802D00240C4A1369BD
:1022000003F03803102B0DD0182B09D063B91368D5
:102210009B060BD513680748C3F3C103D84070472A
:10222000FEF7E2BD04487047044870470148704714
:10223000004402580090D00300127A0000093D00CB
:10224000194A136903F03803102B10B525D0182B49
:1022500009D023BB13689B0623D513681348C3F327
:10226000C103D84001E0FEF7BFFD0F49104A8B695A
:102270008969C3F303230F4C01F00F0113440A448F
:1022800093F8301092F8303001F01F0203F01F0372
:10229000D040C4F8A000D84010BD0748E5E7074883
:1022A000E3E70248E1E700BF004402580090D00392
:1022B00018A10C080000002400127A0000093D005B
:1022C000474A70B4946A956AD66A15F47C3FC5F3A0
:1022D0000533D16B5BD0C1F3CC01C6F3001604F01B
:1022E000030407EE903A06FB01F1012CB8EEE77A01
:1022F00006EE901AFAEEE96A03D0022C6AD0002C9E
:102300004AD0DFED387A87EE876A936BC3F3080310
:1023100007EE903AF7EE005AF8EEE77A77EEA67AF3
:1023200077EEA57A67EE867A2D4AB7EE006A936B50
:10233000C3F3462307EE103AB8EEC77A70BC37EE07
:10234000067AC7EE876AFCEEE66AC0ED006A936B18
:10235000C3F3064307EE103AB8EEC77A37EE067AB3
:10236000C7EE876AFCEEE66AC0ED016A936BC3F3C1
:10237000066306EE903AF8EEE66A76EE866A87EE37
:10238000A67AFCEEC77A17EE903A8360704770BC6D
:10239000C0E900338360704713689B061DD514683D
:1023A000F7EE005A936B1049C4F3C102C3F308035C
:1023B000D14007EE903A06EE101AF8EEE77AB8EE42
:1023C000C66A77EEA66AC6EE077A36EEA57A67EE9B
:1023D000877AA9E7DFED057A95E7DFED057A92E7E1
:1023E000004402580024744A0090D0030024F44AA8
:1023F0000024744C474A70B4946A956AD66A15F002
:102400007C7FC5F30553516C5BD0C1F3CC01C6F39F
:10241000002604F0030407EE903A06FB01F1012CBC
:10242000B8EEE77A06EE901AFAEEE96A03D0022CCB
:102430006AD0002C4AD0DFED387A87EE876A136CB9
:10244000C3F3080307EE903AF7EE005AF8EEE77A86
:1024500077EEA67A77EEA57A67EE867A2D4AB7EE02
:10246000006A136CC3F3462307EE103AB8EEC77A3E
:1024700070BC37EE067AC7EE876AFCEEE66AC0EDFE
:10248000006A136CC3F3064307EE103AB8EEC77A3E
:1024900037EE067AC7EE876AFCEEE66AC0ED016A9F
:1024A000136CC3F3066306EE903AF8EEE66A76EE36
:1024B000866A87EEA67AFCEEC77A17EE903A8360BA
:1024C000704770BCC0E900338360704713689B0697
:1024D0001DD51468F7EE005A136C1049C4F3C102FD
:1024E000C3F30803D14007EE903A06EE101AF8EE57
:1024F000E77AB8EEC66A77EEA66AC6EE077A36EED7
:10250000A57A67EE877AA9E7DFED057A95E7DFED33
:10251000057A92E7004402580024744A0090D003E0
:102520000024F44A0024744C0269836870B50446A0
:1025300005681343C069626986B029681343AC4AD1
:1025400003430A40616A1343E2682B606B6823F41B
:1025500040531343A2696B60A64B9D4200F0668115
:10256000236AAE681A43A44B33401A43AA60EB6A4D
:1025700023F00F030B43EB62A04B9D4228D0A04BEE
:102580009D421AD09F4B9D4217D09F4B9D4214D025
:102590009E4B9D4211D09E4B9D4219D09D4B9D421A
:1025A0000BD09D4B9D4208D0012000234FF001121B
:1025B0006367A266A36706B070BD984B5B6D03F0BE
:1025C0000703052BF0D8DFE803F09F7F8A925F793D
:1025D000924B5B6D03F03803282BE5D801A252F82B
:1025E00023F000BF91270408A9250408A9250408A1
:1025F000A9250408A9250408A9250408A925040873
:10260000A9250408C9260408A9250408A925040841
:10261000A9250408A9250408A9250408A925040852
:10262000A9250408DF260408A9250408A92504080B
:10263000A9250408A9250408A9250408A925040832
:10264000A9250408EF260408A9250408A9250408DB
:10265000A9250408A9250408A9250408A925040812
:10266000A925040889260408A9250408A925040821
:10267000A9250408A9250408A9250408A9250408F2
:10268000A9250408BD260408B0F5004F644853D0BE
:10269000644B626803EB4103B3F84030B0FBF3F0E6
:1026A00000EB52004FF6EF73B0FBF2F0A0F1100216
:1026B0009A423FF679AFE860002076E7B0F5004F28
:1026C0003AD04FF40040E3E7B0F5004F2DD003A817
:1026D000FFF7F6FD04980028EED0616AD8E7B0F560
:1026E000004F71D06846FFF785FE0198F3E7B0F51B
:1026F000004F5ED0494B1A68920639D51B684A488C
:10270000C3F3C103D840C3E7B0F5004F32D0FFF7A1
:1027100097FD424A434BD269C2F30212134493F825
:10272000303003F01F03D840D5E703A8FFF7C8FDFA
:1027300004980028C0D0616A3A4B626803EB4103F9
:102740004FF6EF71B3F84030B0FBF3F0530803EBF2
:102750004003B3FBF2F3A3F110028A423FF624AF29
:1027600023F00F02C3F3420392B21343EB60A3E7DB
:102770002D488DE7FFF764FD284A2A4BD269C2F342
:102780000212134493F8303003F01F03D840D0E70F
:10279000B0F5004F1DD0FFF753FD204A214BD26901
:1027A000C2F30222134493F8303003F01F03D840E1
:1027B00091E71A4B1A68900640F1A5801B681A48E9
:1027C000C3F3C103D840B7E76846FFF713FE01988B
:1027D000AFE7FFF735FD114A124BD269C2F302226F
:1027E000134493F8303003F01F03D840A1E700BF33
:1027F000F369FFCF000C0058FFF4FF1100100140F7
:102800000044004000480040004C004000500040A0
:102810000014014000780040007C00400044025851
:1028200000093D0018A10C080090D003A868374BA0
:1028300003401343364AAB60EB6A23F00F030B43AC
:10284000EB62936D03F00703052B3FF6ADAEDFE8B7
:1028500003F0413C3303524F2D4B1A6895064CD47C
:102860002C482D4B656803EB410305EB4501B3F89C
:102870004020B0FBF2F399423FF696AEB3EB053F32
:102880003FF692AE0023194684F062FF2A46090201
:10289000030241EA1061680818184FF0000341F183
:1028A000000184F055FF1D4BA0F540729A423FF69F
:1028B0007BAE1B4BD860FFE66846FFF79BFD019897
:1028C00000283FF4F9AE616ACBE703A8FFF7F8FCF4
:1028D0000498F5E7FFF7B4FC0D4A0F4B126AC2F3F8
:1028E0000212134493F8303003F01F03D840E7E797
:1028F0004FF40040B5E70B48B3E71B680548C3F346
:10290000C103D840ADE7034816E700BFFFF4FF114D
:10291000004402580090D00318A10C08FFFC0F00DF
:10292000000C005800093D00344A136830B423F00D
:102930008063334C1360256803E023685B1B022B24
:1029400054D813681B01F8D4936A056823F47C33C8
:1029500043EA053393628368C568013B013D5B022E
:102960002D049BB205F4FE052B434568013DC5F3DC
:1029700008052B430569013D2D0605F0FE452B4357
:102980009363D36A456923F0C0032B43D362D36AB0
:10299000856923F020032B43D362D36A23F010030D
:1029A000D362D36BC0696FF3CF0343EAC003D36331
:1029B000D36A43F01003D362D36AD1B101290CBFAB
:1029C00043F4801343F40013D3620C4A136843F0BA
:1029D00080631360216803E023685B1A022B05D82B
:1029E00013681B01F8D5002030BC7047032030BCB1
:1029F000704743F40023D362E7E700BF0044025866
:102A0000802D0024344A136830B423F08053334CB3
:102A10001360256803E023685B1B022B54D81368FE
:102A20009B00F8D4936A056823F07C7343EA05534E
:102A300093628368C568013B013D5B022D049BB234
:102A400005F4FE052B434568013DC5F308052B43FE
:102A50000569013D2D0605F0FE452B431364D36A3D
:102A6000456923F440632B43D362D36A856923F419
:102A700000732B43D362D36A23F48073D362536C05
:102A8000C0696FF3CF0343EAC0035364D36A43F4CE
:102A90008073D362D36AD1B101290CBF43F4000320
:102AA00043F08073D3620C4A136843F08053136081
:102AB000216803E023685B1A022B05D813689B008A
:102AC000F8D5002030BC7047032030BC704743F479
:102AD0008003D362E7E700BF00440258802D002442
:102AE000026810B452E8003F23F4907342E80031CA
:102AF0000029F7D1144C02F1080353E8003F2340AA
:102B000002F1080C4CE800310029F4D1C36E012B0E
:102B100008D0002320225DF8044BC0F88C204367C6
:102B2000C366704752E8003F23F0100342E80031CB
:102B30000029EED052E8003F23F0100342E80031B4
:102B40000029EFD1E5E700BFFEFFFFEF436BDA6935
:102B5000F0B5970683B0044642D5586AE36AC0B21E
:102B6000002B00F09580216B9847636B1A681D4617
:102B700022F480721A609A6822F001029A609A69BF
:102B800042F008029A61DA69D6072DD4DA69900713
:102B900001D502221A62DA69510701D504221A62AC
:102BA000DA69120701D508221A62DA69170612D506
:102BB000D4F8BC20212A0ED0D4E909128A4273D05D
:102BC000A169895C0132C9B299622169B2FBF1F055
:102BD00001FB1022A262DA69560608D403B0F0BDE8
:102BE000DA691D46D607D1D501221A62CEE7DA6925
:102BF00040F60F0C1E6804F1340012EA0C0F9968BD
:102C000036D0B24F0F4040F0BB80DFF8CCC216EA9E
:102C10000C0F40F06381D4F8A050012D4CD0D502A8
:102C200002D54F0200F16781150606D501F40001B7
:102C300006F080050D4340F043815106CED5720663
:102C4000CCD553E8002F22F0400243E8002141B1E7
:102C5000626B52E8003F23F0400342E80031002954
:102C6000F7D120220023C4F8BC20C4F8AC30B5E76B
:102C70009506D0D506F0200501F080573D43CAD017
:102C8000D4F8A830002BA9D003B0BDE8F040184715
:102C9000E3696269D054E369E2680133B3FBF2F19E
:102CA00002FB1133E36160E70022A4F88A201A686E
:102CB00022F080021A608EE7D706B0D5F506AED5B1
:102CC0001022B4F890501A629A68570640F11D819C
:102CD000D4F8B40001684A6892B2002A00F050812A
:102CE000AA4280F04D81C169A4F89220B1F5807F9D
:102CF00040D053E8002F22F4807243E8002141B114
:102D0000626B52E8001F21F4807142E80015002D2B
:102D1000F7D103F1080252E8002F22F0010203F17B
:102D2000080545E800210029F3D103F1080252E823
:102D3000002F22F0400203F1080545E80021002998
:102D4000F3D12022C4F8C020C4F8A01053E8002F0B
:102D500022F0100243E80026002EF7D15C490D68EE
:102D600040B190F83530022B00F01381802380F8B9
:102D7000346043650223C4F8A430B4F892302DE7E0
:102D800012F0010F0CD016F4807F09D04FF0010C27
:102D9000C3F820C0D4F8C4C04CF0010CC4F8C4C0BF
:102DA00012F0020F7BD112F0040F0CD011F0010FC2
:102DB00009D04FF0040CC3F820C0D4F8C4C04CF0C4
:102DC000020CC4F8C4C012F0080F0CD006F0200C9E
:102DD0005CEA070C07D008271F62D4F8C47047F0DC
:102DE0000807C4F8C47017050AD5770108D54FF451
:102DF00000671F62D4F8C43043F02003C4F8C43025
:102E0000D4F8C430002B3FF4E9AE92060CD506F09E
:102E1000200601F080510E4306D0D4F8A8301BB133
:102E200001909847656B0198D4F8C420AB6802F014
:102E3000280203F04003134361D0FFF751FEAB6853
:102E40005B067FF5CBAE05F1080353E8003F23F0A6
:102E5000400305F1080141E8003262B1626B02F102
:102E6000080353E8003F23F0400302F1080040E864
:102E700000310029F3D1D4F8B40000283FF4AEAEFD
:102E800090F83520134B022A03653BD1FDF7EEF88D
:102E900000283FF4A3AED4F8B400036DF4E611F0BB
:102EA000010F90D04FF0020C12F0040FC3F820C0B5
:102EB000D4F8C4C04CF0040CC4F8C4C083D078E784
:102EC000D4F8AC30002B7FF4DFAE87E601000010B1
:102ED000802D0024691004082001000412F0010F65
:102EE0003FF471AF16F4807F7FF450AF12F0020F01
:102EF0007FF469AF57E74FF480121A626EE6C4F8A8
:102F0000C4306BE680224265BEE6B4F89220B4F885
:102F1000921092B289B2AA423FF460AE00293FF407
:102F20005DAE53E8002F22F4907243E8002141B1D6
:102F3000626B52E8001F21F4907142E800100028F3
:102F4000F7D1954803F1080252E8002F024003F13F
:102F5000080545E800210029F4D12022C4F8A81072
:102F6000C4F8C020C4F8A01053E8002F22F01002CB
:102F700043E800210029F7D10223C4F8A4302DE64C
:102F8000AA427FF42BAEC369B3F5807F7FF426AEEF
:102F9000F2E70368814A824E824FB34218BF9342E0
:102FA00006F118060CBF01220022B34208BF42F00E
:102FB00001021836B34208BF42F001021836B3428C
:102FC00008BF42F001021836B34208BF42F00102C6
:102FD00006F55676B34208BF42F001021836B342F6
:102FE00008BF42F001021836B34208BF42F00102A6
:102FF0001836B34208BF42F001021836B34208BF88
:1030000042F001021836B34208BF42F001021836FE
:10301000B34208BF42F00102A6F59266BB4218BF58
:10302000B34207F592670CBF01260026BB4208BFDA
:1030300042F0010256EA020779D0D3F800C02CF022
:103040001E0CC3F800C0D3F814C02CF0800CC3F8D9
:1030500014C0D0F860C076BBD0F860C0DCF8006067
:1030600026F48076CCF800601A6822F001021A601B
:1030700003E00A68521B052A24D81A68D607F8D438
:10308000D0E9165101F01F012FB33F238B40AB60F5
:10309000C36ED0E91921516033B11A68016F22F46F
:1030A00080721A60436F4B600122002380F8352044
:1030B00080F834305EE6DCF8002022F48072CCF830
:1030C0000020D1E7202103220023416580F834301D
:1030D00080F835204EE6344A344EB34218BF93424E
:1030E00006F114060CBF01220022B34208BF42F0D1
:1030F00001021436B34208BF42F001021436B34253
:1031000008BF42F001021436B34208BF42F0010288
:10311000012606FA01F1696025498B4208BF42F099
:103120000102002AB4D1234A9342B1D0BCE71E4E1B
:10313000DFF878C0634518BFB3420CF1140C0CBF24
:1031400001260026634508BF46F001060CF1140C69
:10315000634508BF46F001060CF1140C634508BF37
:1031600046F001060CF1140C634508BF46F0010659
:10317000D3F800C02CF00E0CC3F800C0DFF830C04C
:10318000634508BF46F00106002E7FF465AF094E87
:10319000B3423FF461AF67E7FEFFFFEF400002403C
:1031A0005800024028000240085402581C5402589B
:1031B000805402589454025882B00023019302E0D4
:1031C0000369002B09DB019B01330193019BB3F1E0
:1031D000706FF5D9032002B070478901002341F0D8
:1031E00020010193016103E0036913F0200307D07C
:1031F000019B01330193019BB3F1706FF4D9E9E7AF
:10320000184602B0704700BF82B00023019302E06D
:103210000369002B09DB019B01330193019BB3F18F
:10322000706FF5D9032002B070470022102301927D
:10323000036103E0036913F0100307D0019B01331E
:103240000193019BB3F1706FF4D9EBE7184602B01C
:10325000704700BF82B00023019302E00369002B96
:1032600009DB019B01330193019BB3F1706FF5D929
:10327000032002B0704700230193036943F0010368
:10328000036103E0036913F0010307D0019B0133DD
:103290000193019BB3F1706FF4D9E9E71846E8E7B1
:1032A0002DE9F843056807460C46C5F31009B9F146
:1032B000000F39D18A4B4FF6FF72B3F8803093423A
:1032C00056D0002B54D0874A02EA432808F1006800
:1032D000454534BF4FF001084FF00208824B9D4234
:1032E00006D903F500339D4200F2CF804FF001096B
:1032F0007E4E96F8B834012B12D00123B8F1010F9D
:1033000086F8B8344FF00003C6F8BC3436D002203B
:1033100070F0A8FD002800F09980002386F8B834EA
:103320004FF0FF30BDE8F883704E96F8B834012BAB
:103330004CD0012386F8B83405F17843B3F5801FEB
:1033400048D3A5F10163B3F5801F3FD200230220CB
:10335000C6F8BC3470F086FD002870D1644A4FF086
:103360000208D2F80C3143EA0803C2F80C313FE0FE
:10337000B5F1016F67D3052010F0FEF9404670F0FB
:1033800071FD0028C9D14046DFF86481D8F80C30BF
:1033900023F4E663C8F80C30D8F80C3043EA09236C
:1033A00043F0A403C8F80C3070F05CFDD8F80C2092
:1033B000504B1340C8F80C300028AED105F17843CB
:1033C0000122B3F5801F86F8B82403D36FF0010003
:1033D000BDE8F88300230120C6F8BC3470F042FD3C
:1033E00068BB434A4FF00108D36843F00203D3603F
:1033F000BFF36F8FBFF34F8F04F1200254F8043BEB
:10340000944245F8043BF9D1BFF36F8FBFF34F8F60
:10341000404670F027FDB8F1010F354A30D0D2F8A0
:103420000C3123F00203C2F80C31002386F8B834C3
:103430000028CBD13B6820333B60BDE8F8830023F4
:1034400086F8B834C2E74FF0010847E7DFF8A080FC
:103450000220D8F80C3123F4E663C8F80C31D8F810
:103460000C3143EA092343F0A403C8F80C3170F08F
:10347000F9FCD8F80C211F4B1340C8F80C319BE71E
:10348000D36823F00203D360CFE703F500339D42F6
:1034900011D903F500339D4210D903F500339D4245
:1034A00006D903F500339D420BD84FF005091FE7FD
:1034B0004FF004091CE74FF0020919E74FF0030928
:1034C00016E703F500339D4206D9B5F1016FBFF44D
:1034D00052AF4FF007090BE74FF0060908E700BFAE
:1034E00000E8F11F00FE1F00FFFF0108802D0024EF
:1034F00000200052FBF8FFFF0148FCF7B3BF00BFFC
:1035000044320024084810B4D0F8C434D0F8F84449
:1035100099691A682CB1234600F2C4405DF8044B47
:1035200018475DF8044B7047802D00240148FCF7D4
:1035300099BF00BF9C320024084810B4D0F81C3555
:10354000D0F8504599691A682CB1234600F21C50F6
:103550005DF8044B18475DF8044B7047802D00243C
:103560000148FCF77FBF00BFF4320024084810B4C4
:10357000D0F87435D0F8A84599691A682CB123465B
:1035800000F274505DF8044B18475DF8044B704727
:10359000802D00242DE9F04FDFF8649300EB400507
:1035A00083B0430009EB85050093D5F8A83001935B
:1035B000002B00F062818046B5F8AE0070F0A2FAF0
:1035C00095F8AC000CF024F8044695F8AD000CF02A
:1035D0001FF808F101030746DBB2002C00F07281EE
:1035E00040F60C12A1882372E2802268002800F0C5
:1035F0005D81037240F60C23C38091613B68BA88F9
:103600009A611121204609260BF0BEFF1121384690
:103610000BF0BAFF6525002C00F032812268A388E8
:1036200011690B4200F02C811B04936110F048F8E3
:1036300005468B4610F044F8401B61EB0B01052852
:1036400071F10001F6D314B12368A2889A6110F0D9
:1036500037F805468B4610F033F8401B61EB0B0141
:10366000052871F10001F6D3013ED3D11CB1A38826
:1036700022681B04936110F023F805460E4610F0F3
:103680001FF8401B61EB0601052871F10001F6D31C
:103690001FB1BB883A681B04936110F011F805460E
:1036A0000E4610F00DF8401B61EB0601052871F184
:1036B0000001F6D314B12368A2889A6110F000F8D3
:1036C00005460E460FF0FCFF401B61EB0601052886
:1036D00071F10001F6D317B13B68BA889A61009B7B
:1036E00020463E21434409EB830393F8B34022462E
:1036F0000BF06CFF224638463E210BF067FF7A4CF8
:103700005823019A03FB0843C3F8C424774B9A4219
:1037100000F0C780FEF794FD754BDA69C2F3021220
:10372000744B134493F8303003F01F03D840009BD0
:10373000434409EB830393F8B030022B00F0BD80C3
:10374000032B00F0B580012B14BF4FF4C8714FF468
:10375000487170F065FA03465822002102FB0842C6
:10376000C2F8CC14C2F8D414C2F8D814C2F8E014C9
:10377000C2F8E4140121C2F8C834C2F8D01492F897
:10378000051501F0FF00002900F0A480582123F066
:10379000706224264FF4004701FB08415648D1F8D7
:1037A000C43481F805651D6825F001051D601A61A6
:1037B0009A6822F400429A609F605A6822F400627C
:1037C0005A605A681043D1F8DC2458601202D86855
:1037D00020F40040D860DA6000221A60186840F0D7
:1037E000010018602020C1F8082581F80505C1F8FE
:1037F000F42481F8062591F805052028C5B217D1D3
:1038000091F80405012813D081F80565186820F0A7
:1038100001001860186820F480501860186818605B
:10382000186840F00100186081F8055581F80425FA
:10383000009B02210126314F434409EB830999F88B
:10384000B250284670F062FB05F01F036A0999F830
:10385000B15006FA03F30221284647F8223070F0EF
:1038600055FB582303FB084405F01F036D0906FAB6
:1038700003F347F8253084F8C06403B0BDE8F08F47
:10388000013D2AD00FF01CFF83468A460FF018FF37
:10389000B0EB0B0061EB0A01052871F10001F5D3D3
:1038A000B9E6FEF7CDFC124B1A6A37E79161A8E63C
:1038B000C82170F0B5F903464EE7642170F0B0F905
:1038C000034649E700283FF49CAE037240F60C2300
:1038D000C38093E682F8040558E7002C3FF4A6AEB7
:1038E000A3882268A0E600BF802D0024001C005899
:1038F0000044025818A10C080080000200E100E01A
:10390000000000242DE9F04F441C85B017469DF8B7
:103910003C202DD05824DFF8A8831E46054600FB26
:1039200004F408EB040393F8C094B9F1000F1FD01E
:1039300044444900FF2F04F2C444039100D0EEB97F
:10394000002A40F0C680582303FB058393F8052521
:10395000202A04D1B6B94FF40072C3F80825B8F88C
:10396000C835284601339BB2A8F8C835FFF712FEC8
:103970004FF00009484605B0BDE8F08F93F80535D3
:10398000202BECD14FF0580A0AFB058A9AF804352F
:10399000012BE4D00122D8F800B019234FF40041E4
:1039A0008AF804252046CDF800B0FEF7E5FB002894
:1039B000D5D10E9BDAF8C414CAF8E8342123BA4AE8
:1039C0008AF805354023CAF8F8048AF80635CAF89B
:1039D00008052046AAF8EE644B681340039A134387
:1039E000B24A1A434A60594670F00EFA024600285D
:1039F00040F0FB80DAF8C434802120469F620A231D
:103A0000CDF800B0FEF7B8FB002840F0EE80BAF821
:103A1000EE349BB2FF2B40F21681DAF8C414FF2378
:103A2000A348AAF8EC344B68A24A03400398034326
:103A30001A434A605826DDF80CA05F46039506FB42
:103A4000058605E0B6F8EE349BB2002B00F010813D
:103A50003946204670F0D8F9002840F0F280D6F8B8
:103A6000E814D6F8C45411F8012BB6F8EC34AA6265
:103A7000C6F8E814013BB6F8EE149BB20139A6F87B
:103A8000EC3489B2A6F8EE14B6F8EE1489B2002B25
:103A9000D8D10029D6D002460A238021204600979B
:103AA000FEF76AFBFF22002840F0CB80B6F8EE3428
:103AB0009BB2934240F2A080D6F8C414A6F8EC243E
:103AC0004B687B4A13407B4A43EA0A031A434A6025
:103AD000B8E74FF0580A0AFB058A9AF80535202BFB
:103AE0007FF43DAF9AF80435012B3FF438AF012243
:103AF000D8F8007019234FF400418AF804252046B5
:103B00000097FEF739FB00287FF429AF0E9BCAF817
:103B1000F804CAF8E83421238AF8053510238AF816
:103B20000635CAF80805AAF8EE64BAF8EE349BB276
:103B3000FF2B00F2C780BAF8EE349BB2AAF8EC343F
:103B4000002B40F0F180DAF8C41457484B685A4A09
:103B50000340039803431A434A605826AA4606FBCB
:103B60000586B6F8EE3439469BB2002B00F0D480BF
:103B7000204670F049F9002878D1D6F8E814D6F834
:103B8000C45411F8012BB6F8EC34AA62C6F8E81454
:103B9000013BB6F8EE149BB20139A6F8EC3489B2B9
:103BA000A6F8EE14B6F8EE1489B2002BD9D100298C
:103BB000D7D002460A23802120460097FEF7DCFA80
:103BC000FF22002852D1B6F8EE349BB2934225D999
:103BD000D6F8C414A6F8EC244B68354A1340039A6F
:103BE0001343344A1A434A60BBE75823002203FBBD
:103BF000058383F80425B2E6B6F8EE34D6F8C4247B
:103C00009BB22B485168A6F8EC34DBB201404AEA7B
:103C100003430B4343F00073536013E7B6F8EE34ED
:103C2000D6F8C4149BB2039A2148A6F8EC34DBB250
:103C300042EA03434A680240134343F000734B6077
:103C40008FE7039D8BE6BAF8EE34DAF8C4149BB222
:103C5000039A1748AAF8EC34DBB242EA03434A68F5
:103C60000240134343F000734B60E3E6554676E6AB
:103C700039462046039D70F099F800287FF46FAE16
:103C8000D6F8C43420210D4CD9615A6822405A60BC
:103C90005823002286F8051503FB058386F80605E0
:103CA00083F8042566E600BF009800FC00200101AF
:103CB000009C00FC0000FF010020000200E800FE64
:103CC000802D0024FF234FF47F00FE224FF08076EA
:103CD000AAF8EC34039BDDF838E01E4358231EF8A5
:103CE00001AB03FB0583DFF850C0D3F8C414C1F85F
:103CF00028A0A3F8EC24B3F8EE24C3F8E8E4013AD2
:103D000092B2A3F8EE244B6803EA0C033343034357
:103D100043F400534B6020E72046554670F046F8C8
:103D200000287FF41CAEABE7013B4FF000769AB25F
:103D3000501CC0B20004CDE7009800FC2DE9F04F04
:103D4000441C85B099469DF83C3000F0968058257B
:103D5000C34C064600FB05F504EB050B9BF8C0A41D
:103D6000BAF1000F00F089802544FF2A90464FEAFF
:103D7000410705F2C44540F08680002B00F08380A7
:103D80009BF80535202B6FD19BF80435012B6BD0A8
:103D90000122D4F8008019234FF400418BF8042548
:103DA0002846CDF80080FEF7E7F900285CD10E9B8D
:103DB000CBF8F804CBF8E83422238BF80535102330
:103DC0008BF80635CBF80805ABF8EE94BBF8EE346B
:103DD0009BB2FF2B00F21081BBF8EE34DBF8C41469
:103DE0009BB2A0484A68ABF8EC34DBB2024047EA29
:103DF000034313439C4A1A434A604FF0580909FB96
:103E00000649B9F8EE349BB2002B00F08481D9F852
:103E1000C4349A69520700F1318142460A2128468A
:103E2000FEF728F9002840F0F480D9F8C4349A69E4
:103E3000910640F1F9809A699A6912F0100200F037
:103E4000F18010222021894DDA610422C9F8082569
:103E5000D9615A682A405A6089F8051589F804051D
:103E600089F8060522689B69B4F8C83530460133E5
:103E70009BB2A4F8C835FFF78DFB4FF0000A5046FF
:103E800005B0BDE8F08F4FF0580B0BFB064B9BF8CD
:103E90000535202BE8D10E9B002B00F0A8809BF865
:103EA0000435012BE0D0236801224FF4004128465D
:103EB0008BF80425039300931923FEF75DF900287E
:103EC000D2D12223DBF8C4140E9A8BF80535402397
:103ED000CBF8E8248BF80635CBF80805ABF8EE9460
:103EE000DFF880914A68CBF8F804284602EA090214
:103EF0003A4342F490324A6003996FF085FF0246DC
:103F0000002840F03481402328461946DBF8C434A9
:103F1000C3F82880039B00930A23FEF72DF900289D
:103F200040F02581BBF8EE349BB2FF2B40F2268196
:103F3000DBF8C414FF234E4AABF8EC344B6803EAB9
:103F400009033B431A434A604FF05808B946039FA0
:103F500008FB064805E0B8F8EE349BB2002B00F0F1
:103F60001F810A230022042128460097FEF704F946
:103F700000287FF479AFD8F8C434596AD8F8E83407
:103F80001970B8F8EE14D8F8E8340139013389B261
:103F9000C8F8E834B8F8EC34A8F8EE14013BB8F8E7
:103FA000EE149BB289B2A8F8EC340029D3D0002BD0
:103FB000D1D102460A23802128460097FEF7DCF87B
:103FC000FF2200287FF450AFB8F8EE349BB2934242
:103FD00040F2BB80D8F8C414A8F8EC244B68254AFA
:103FE0001340254A43EA09031A434A60B3E74FF4F2
:103FF0000073CBF8083537E7DBF8C414FF23194802
:10400000ABF8EC344B681A4A03403B431A434A600E
:10401000F3E6582303FB0643D3F8C4349A692268B5
:104020009B6921E7C9F808252268A2EB08020A2A41
:104030007FF6EFAE9A6912F004027FF4EAAE5821DF
:1040400001FB0641D1F8080581F80425202240F043
:104050002000C1F8080581F805259B6904E700BF29
:10406000802D0024009800FC0024000200E800FEDF
:104070000024FF01009C00FC0000FF015A6AD9F8EF
:10408000E8341A70B9F8EE34D9F8E824013B01326B
:104090009BB2C9F8E824A9F8EE34B9F8EC34B9F8C1
:1040A000EE24013B92B29BB2A9F8EC34002A3FF413
:1040B000A8AE002B7FF4A5AE0A230022802128465B
:1040C000CDF80080FEF758F800287FF4CDAEB9F89F
:1040D000EE349BB2FF2B0CD9D9F8C414FF233B4814
:1040E000A9F8EC344B683A4A03403B431A434A6010
:1040F00087E6B9F8EE34D9F8C4149BB233484A685D
:10410000A9F8EC34DBB2024047EA0343134343F01F
:1041100000734B6075E6414628466FF047FE002865
:104120007FF4A2AED9F8C43420212A4DD9615A684F
:104130002A405A6089F8051589F806055822002397
:1041400002FB064484F8043599E6B8F8EE34D8F852
:10415000C4249BB21D485168A8F8EC34DBB201407E
:1041600049EA03430B4343F000735360F3E65823DB
:10417000002203FB064383F8042575E6BBF8EE3402
:10418000DBF8C4149BB24A68ABF8EC34DBB202EA49
:10419000090247EA034313430F4A1A434A60D3E62E
:1041A000039928466FF002FE034600287FF45CAEB8
:1041B000D8F8C4242020074DD061516829405160AF
:1041C00088F8050588F80635B8E700BF009C00FCB4
:1041D0000000FF0100E800FE002400020348D0F8C0
:1041E000D8300BB1CC301847704700BF0000002416
:1041F0000348D0F8F8300BB1EC301847704700BFD7
:10420000000000240348D0F8183113B100F586707F
:1042100018477047000000240348D0F8383113B124
:1042200000F5967018477047000000240348D0F846
:10423000583113B100F5A6701847704700000024EC
:104240000348D0F8783113B100F5B67018477047BD
:10425000000000240348D0F8983113B100F5C6706F
:1042600018477047000000240348D0F8B83113B154
:1042700000F5D67018477047000000240348D0F8B6
:10428000D83113B100F5E6701847704700000024DC
:104290000348D0F8F83113B100F5F67018477047AD
:1042A000000000240348D0F8183213B100F5037061
:1042B00018477047000000240348D0F8383213B183
:1042C00000F50B7018477047000000240348D0F831
:1042D000583213B100F513701847704700000024DE
:1042E0000348D0F8783213B100F51B7018477047B7
:1042F000000000240348D0F8983213B100F5237071
:1043000018477047000000240348D0F8B83213B1B2
:1043100000F52B70184770470000002400207047FC
:1043200010B41C46436884466FF30F032343436075
:10433000036843F001030360036843F40073036000
:10434000002C3AD040F2E930DCF814309B0748D515
:10435000002A49D012F8013B40F2E9308CF82030B5
:10436000DCF81430DB0720D40138F9D1214B9C450F
:104370000CD0A3F578439C4538D003F580639C4569
:1043800036D003F578439C450BD103201A4A00EB45
:10439000400002EBC002B2F8E03201339BB2A2F857
:1043A000E03200205DF8044B70479CF83000C0B24A
:1043B00009B101F8010B013CC4D1DCF814301B0732
:1043C000FBD5DCF8183001205DF8044B43F01003F6
:1043D000CCF81830DCF8003023F00103CCF80030C2
:1043E00070470138B0D1C1E7FF23B5E70120CDE721
:1043F0000220CBE700300140000000242DE9F04707
:10440000002682B0294F00F10108DFF8A890284C5F
:10441000DFF8A4A00FE0012300220DF10701FFF750
:104420007FFFAB689B0725D59DF80700FF2839D192
:104430000136464536D0D7F8485395F91030AA686A
:1044400003EB4303920709EBC303D3F8CC02E2D496
:104450006B691BB19A88196812048A61D7F84C23DA
:104460006168D200AAFB0232920963685B1A9A4221
:10447000FBD2D0E74FF4FA73D7F84C23616803FB03
:1044800002F2AAFB0232920963685B1A9A42FBD2DB
:104490006B69002BC8D09DF807001A68FF289B881D
:1044A0009361C5D002B0BDE8F08700BF802D002425
:1044B000001000E000000024D34D621070B595227A
:1044C00082B00446002340F040008DF805200A0E1B
:1044D0008DF8041060F3070362F30F230A0C090A36
:1044E00062F3174361F31F6300936FF079FA24B10D
:1044F00080F00100C0B200284AD1274D274AD5F8E4
:10450000484394F91030A16803EB430302EBC30363
:104510008A07D3F8CC0227D506236A460021FFF785
:10452000FFFEA3689B0704D5082002B0BDE87040D9
:1045300064E74FF4FA70D5F84C23194B00FB02F2F4
:104540001849A3FB0232486892094B681B1A9A4229
:10455000FBD26369002BE7D01A6808209B8893611F
:1045600002B0BDE8704049E763691BB11A689B88D7
:104570001B049361D5F84C23094BD2000949A3FBD6
:1045800002324E6892094B689B1B9A42FBD2C3E7EA
:10459000FF2002B070BD00BF802D00240000002469
:1045A000D34D6210001000E070B5044608200D469F
:1045B000FFF724FFFF2823D0FE2801D0022070BD82
:1045C000264E21462B460022D6F8480377F0B6F84F
:1045D000D6F84843224A94F91030A16803EB43030C
:1045E00002EBC3038A07D3F8CC020BD500220223C7
:1045F0001146FFF795FEA3689B0717D5002070BDF5
:10460000012070BD63691BB11A689B881B0493610C
:10461000D6F84C23134BD2001349A3FB02324D684A
:1046200092094B685B1B9A42FBD2DFE74FF4FA70AA
:10463000D6F84C230B4B00FB02F20B49A3FB0232D2
:10464000486892094B681B1A9A42FBD26369002B97
:10465000D4D01A689B889361D0E700BF802D0024D6
:1046600000000024D34D6210001000E070B52F4C04
:1046700000234FF6FF5182B0D4F84853C4F81433E6
:1046800095F910302A4A03EB4303ADF80410A968EA
:1046900002EBC3038A07D3F8CC0233D5022301AA65
:1046A0000021FFF73DFEAB689B0714D50120FFF703
:1046B000A5FEFF2809D0D4F8502309230020C4F810
:1046C000082384F8183302B070BD0423022084F854
:1046D000183302B070BD4FF4FA70D4F84C23154B68
:1046E00000FB02F21449A3FB0232486892094B68AE
:1046F0001B1A9A42FBD26B69002BD7D01A689B8891
:104700009361D3E76B691BB11A689B881B049361A3
:10471000D4F84C23074BD2000749A3FB02324E6862
:1047200092094B689B1B9A42FBD2B7E7802D00246D
:1047300000000024D34D6210001000E0F0B5CF4C13
:1047400085B0D4F8480300284FD094F81803431ECE
:10475000082B40D8DFE813F034010900D4003F00F3
:10476000AD0074005B003F004B00D4F8480308F034
:1047700043F994F80E5300213720A5F10205FFF705
:104780009DFE2920B5FA85F56D09AD072946FFF78D
:1047900095FE0546FCF70AFFADB994F80E33D4F840
:1047A0004803022B00F0AF81D4F8480384F80F537C
:1047B00008F022F900210920FFF780FE002800F010
:1047C0006181FCF7F3FED4F84803022108F0C8F831
:1047D00094F81803431EDBB2022B40F21B81082819
:1047E00018BF04280CBF0120002005B0F0BD6FF0F9
:1047F000F7F8002840F0B481D4F80833D4F85023F7
:10480000FA33934280F02881FCF704FF9DE76FF0B4
:10481000E7F80028F0D0D4F814330022012B84F8F4
:104820000C2340F2BB81D4F81023013B0821013254
:10483000C4F8143384F81813C4F810230120D4E703
:1048400094F8FC028023D4F8F422002102EBC01279
:10485000D4F8480376F072FF94F8FC320133DBB2EF
:10486000042B84F8FC3240F0F7800223844A0021B4
:10487000D4F8480376F062FF012300226946D4F899
:10488000480376F05BFF9DF8003003F01F03052B13
:1048900000F06F81FCF7BEFED4F80053002D3FF40A
:1048A00054AFD4F804330022D4F8F8120120A847FA
:1048B0004BE74FF40071D4F8F402FFF775FE0128BE
:1048C000054600F0B180022800F0B580002840F0D5
:1048D000C380FCF76BFE0423D4F8006384F80C5308
:1048E00084F81833002EA9D0D4F804332846D4F81D
:1048F000F422D4F8F812B04794F81803431E6AE77C
:1049000010216846FFF750FE00287FF45CAF9DF849
:1049100000209DF8031062F307009DF80D30BDF8EC
:10492000012061F30F209DF804101B0152BA61F3BE
:1049300017409DF80510DBB2A4F8202361F31F6037
:104940009DF80E109DF8082043EA111301F00F01A5
:10495000BDF8065003F5FA6384F83013110902F02C
:104960000F02A4F82E33DDF80930C4F822031BBA75
:10497000A4F8265384F82C13C4F8283384F82D2384
:10498000FCF714FE94F80F33D4F8480363B908F029
:1049900033F84FF400711020FFF790FD0546FCF747
:1049A00005FE002D7FF430AF0221D4F8480307F054
:1049B000D7FF00220423C4F8142384F81833C4E674
:1049C000D4F8480308F018F800210846FFF776FDF0
:1049D0000546FCF7EBFD012D7FF4F5AE0026D4F87B
:1049E000480384F80E6308F007F840F2AB11082082
:1049F000FFF764FD05283CD0012800F09C8094F866
:104A00000E53FCF7D3FD002D00F0B080022384F894
:104A100018339AE6D4F85033D4F808239B1AC82BDD
:104A200022D8002005B0F0BDD4F80833D4F85023C4
:104A30006433934210D2FCF7B9FDFCF7EBFDD4F8D8
:104A40000053002D3FF481AE0022D4F80433D4F893
:104A5000F8121046A84778E694F81803431EDBB214
:104A6000022B3FF6BCAED5E7FCF7D4FD94F8180353
:104A7000B5E684F80E53FCF799FDC7E7802D0024B6
:104A800070A10C0810217548FFF78EFD00287FF4F7
:104A900098AE94F8433313F001033FF492AE94F8C8
:104AA0003423921100F08180012A7FF48AAE94F8B9
:104AB0003B2316216A4E02259200D2B2C5F10803AB
:104AC0008B4228BF0B46C3F108059840C91A42FA29
:104AD00005F24FF0000540EA020016F8012FEDD173
:104AE00001308002C4F81C03FCF760FDD4F84803D1
:104AF00007F082FF00210A20FFF7E0FC68BB0323D8
:104B000084F8183321E607F077FF29463A20FFF7AB
:104B1000D5FC2A46054604236946D4F8480376F0B6
:104B20000DFEFCF743FD002D7FF46EAE009D2DBA07
:104B3000C5F3807538E6042332466946D4F8480345
:104B400076F0FCFD9DF80330AB2B7FF458AF0223C9
:104B500084F80E33FCF72AFD58E7FCF727FD53E6EF
:104B6000FCF724FD042384F8183367E684F818530F
:104B700029E60722D4F85033D4F8005384F81823D8
:104B8000C4F80833002D5BD0D4F804330120D4E9F5
:104B9000BD21A84794F81803431E1CE652D00423F5
:104BA00084F81833FCF702FD48E694F839131046F0
:104BB00094F83D53062601F00F022A4FAD0103FA87
:104BC00002F20323EDB2C6F10801994228BF19464B
:104BD000C1F1080688405B1A45FA06F54FF0000659
:104BE00040EA050017F8015FEDD194F83A5302301E
:104BF000DFF874E00C26AD014FF0060CEDB2CCF1FD
:104C000008014FF0000CB14228BF3146C1F108073E
:104C10008B40761A45FA07F543EA05031EF8015F53
:104C2000EDD10133D5178340A3FB022103FB05110E
:104C3000520A42EAC152C4F81C23FCF7B7FC55E7FC
:104C40002846D2E5FFF712FD02287FF405AFFCF7F6
:104C5000ADFC94F81803431EBDE500BFB43000243A
:104C6000BB300024BD300024BA3000242DE9F041CF
:104C7000054682B0884617461E46354C94F8180300
:104C800004280BD0082807D1D4F81033AB423FD00A
:104C9000FFF7ECFC0228F1D0012034E0D4F84833CF
:104CA0001A79022A36D094F80F337BB3294618209C
:104CB000FFF704FC002844D194F81833082B27D0C0
:104CC000FE238DF80530FF2301AA0021D4F8480304
:104CD0008DF80430022376F031FD80234246D4F86B
:104CE0004803002176F02AFD012206230020C4F8A3
:104CF000F482C4F8F852C4F80073C4F8046384F86A
:104D0000FC2284F8183302B0BDE8F0816902CEE7D6
:104D1000FC23D6E79A689207C5D55B691BB19A88D0
:104D2000196812048A61D4F84C330A49DA000A4B34
:104D30004868A3FB023292094B681B1A9A42FBD2C5
:104D4000B1E7FCF733FCFCF765FC0320DBE700BFB1
:104D5000802D0024001000E0D34D621070B51D4C72
:104D600006460D4694F81833042B09D0082B23D19E
:104D7000D4F8103383421DD0FFF778FC02281BD1F2
:104D8000D4F8480307F038FE00213720FFF796FBE0
:104D900029461720FFF792FBB0B994F80F336BB98F
:104DA00071021920FFF78AFB70B90823C4E9C465B2
:104DB00084F81833022070BD012070BD31461920DF
:104DC000FFF77CFB0028F0D0FCF7F0FBFCF722FC9F
:104DD000032070BD802D00242DE9F041294C0746A9
:104DE0008846164694F818C31D46BCF1040F09D036
:104DF000BCF1080F02D00020BDE8F081FFF736FCBF
:104E00000228F8D1D4F848331A79022A22D094F82B
:104E10000F33B3B979021120FFF750FBB8B905225F
:104E2000D4F850330120C4F8F482C4F8F872C4F8FE
:104E30000063C4F8045384F81823C4F80833BDE8A9
:104E4000F08139461120FFF739FB0028E7D0FCF745
:104E5000ADFBD0E79A689207D9D55B691BB19A88F8
:104E6000196812048A61D4F84C330749DA00074BF9
:104E70004868A3FB023292094B681B1A9A42FBD284
:104E8000C5E700BF802D0024001000E0D34D621064
:104E90002DE9F84300242C4E8046036856F8345020
:104EA000AB4209D001340E2CF8D1284A002105204C
:104EB00005F050FD002019E0254B03EB8409D9F8DB
:104EC000CC75AFB198F8051000204B1C01EB4102E6
:104ED00003EB430307EBC202DB00C2F80C80C2E91C
:104EE0000400F854182303FB01700830BDE8F88370
:104EF0000721682005F0B4FD0146C9F8CC05F0B1E2
:104F0000394668227FF0E4FBD9F8CC1506EBC404DF
:104F10003B4689600C6009628963096556F8332055
:104F2000954205D001330E2BF8D14F600F46C9E7EB
:104F3000084F4C2202FB03774F600F46C2E7064A38
:104F4000052005F007FDB5E774A10C08A4550D0870
:104F5000802D002484330024CC550D0830B40C4C33
:104F60000022234603E0013214330C2A0CD093F8BC
:104F700004C08445F7D1DD68294201D10029F2D16E
:104F8000142303FB024000E0002030BC704700BF48
:104F90002C030024F0B54468A37913F002025FD01B
:104FA00002224FF0080C036864795B689B48204438
:104FB00093F83C40012C90F8CC0050D0012483F8A9
:104FC0003C40142848D8DFE810F01500470047009F
:104FD000470084004700470047003B014700470067
:104FE0004700BB00470047004700F200470047006A
:104FF00047004D0018688A4C056A8A4E25F0020564
:10500000B04242EA0502056A25F0010505624768DB
:10501000856904EA050444F0600407D0824DA84283
:1050200004D005F57055A84240F04D8122F00802E9
:1050300047F440774CEA020222F0040247608461A0
:1050400041630262826942F008028261826922F051
:105050000402826182698261002283F83C20F0BDF3
:105060009446A0E718686F4E046AB04224F4001416
:1050700044EA0252046A24F4801404626B4C4568CA
:10508000476D04EA070444F4C0440ED006F5806678
:10509000B0420AD0664F06F58046B04218BFB8420B
:1050A00003D006F58066B04201D145F48025456005
:1050B0004465C1650262426D42F400624265426D20
:1050C00022F480624265426D4265002283F83C20F2
:1050D000C5E71868574C056A524E25F02005B042C6
:1050E00045EA0215026A22F01002026247688269EC
:1050F00004EA020444F4C04400F0DE804A4A9042CC
:1051000000F0DA804A4E4C4A904218BFB04203D0B9
:1051100002F58062904201D147F4406747608461A4
:1051200081630562826942F400628261826922F4CD
:105130008062826182698261002283F83C208EE76E
:105140001868384E046AB04224F4005444EA02322B
:10515000046A24F480540462364C4568C76904EA42
:10516000070444F4C0440ED006F58066B0420AD06D
:105170002F4F06F58046B04218BFB84203D006F55F
:105180008066B04201D145F480454560C461016448
:105190000262C26942F40062C261C26922F48062A2
:1051A000C261C269C261002283F83C2057E71868D7
:1051B0001C4E046AB04224F4003444EA0242046AF9
:1051C00024F4803404621D4C4568476D04EA0704EA
:1051D00044F060040ED006F58066B0420AD0144F49
:1051E00006F58046B04218BFB84203D006F5806687
:1051F000B04201D145F48035456044658165026265
:10520000426D42F008024265426D22F0040242659E
:10521000426D4265002283F83C2020E718A10C086B
:105220008CFFFEFF0000014000040140FF8FFFFEE5
:1052300000400140FF8CFFFE004401408FFFFEFF55
:105240001868264C056A264E25F4007EB0424EEAC8
:105250000225026A22F4807202624768C26904EA87
:10526000020444F0600420D01E4A90421DD01E4E1D
:105270001E4A904218BFB04203D002F580629042AD
:1052800001D147F440574760C461C1630562C269F8
:1052900042F00802C261C26922F00402C261C2691E
:1052A000C261002283F83C20D9E625F4006E4EEA64
:1052B0000C2E2EF48065E4E725F0800545EA0C15F8
:1052C00025F0400528E705F58065A8423FF4AEAE1D
:1052D00005F58065A8427FF4B1AEA7E68CFFFEFF1E
:1052E0000000014000040140004001400044014032
:1052F00042685379032B0FD8DFE803F00B0805024F
:1053000010684030704710683C3070471068383083
:10531000704710683430704700207047D0E90002B1
:10532000064B517992790B44406893F8CC1053079F
:1053300001D577F039BA77F0B3BA00BF18A10C08DD
:10534000F0B54468374A2469C368C4F303245B6832
:1053500052F82460EFF31184102585F31288456814
:10536000314F95F805E0D0F80CC002EB4E02D5F8AD
:1053700000E0158CDEF80C2005F4F05522EA050259
:10538000CEF80C2017F806E0DCF8102053F80E5089
:105390001F2A25F0010543F80E5039D9203A20255F
:1053A000DCF804C005FA02F2CCF80C20E2B282F379
:1053B0001188BA5DDFF874C003EB020E46684569D8
:1053C000DEF8044004EA0C0C4CEA0101CEF80410AB
:1053D0007179032924D8DFE801F018151202316829
:1053E0004031CEF80C500124CEF80810995841F005
:1053F000100199509958214399500474F0BD3168B7
:105400003C31EEE731683831EBE731683431E8E7B9
:105410002025DCF804C005FA02F2CCF80820C5E724
:105420000021DEE718A10C084CA20C080000FFFFC9
:1054300003681A7E012A2ED0002293F83010012929
:1054400009D093F8481001290ED093F86010012973
:105450001BD02ABB7047022142F4806283F83010CF
:1054600093F84810012904D1022142F4006283F824
:10547000481093F86010012907D01B6800211B68B1
:105480005962D9680A43DA607047022142F48052B7
:1054900083F86010F1E702214FF400721976CCE72F
:1054A0004FF40072E9E700BF08B5204B98420ED0D8
:1054B00003F5806398420AD01D4A03F58043984261
:1054C00018BF904203D003F5806398421BD1FCF7CC
:1054D000B7FE1849184BCA69C969C2F30222C1F361
:1054E00002211A4492F8302002F01F02D040114AE3
:1054F0001269C2F3C03241EAC202134493F8D030B9
:1055000003FB00F008BDFCF79BFE0A490A4BCA6981
:10551000C969C2F3021CC1F3021103EB0C0292F839
:10552000302002F01F02D040E1E700BF0000014040
:10553000004001400044025818A10C0870B50E4606
:1055400005EE102AD0E90031013E1A680868B6B2AB
:105550005C681568FFF7A8FF07EE900AB8EE455A99
:105560009FED5D7AF8EE677A87EE850A30EE070ADE
:1055700079F006FD23680138AB4280B268D0C4E9F7
:10558000005000238022E660A360A261C4E90433D6
:1055900094F83D3003F0FF02002B78D00223211D48
:1055A000284684F83D30FBF791FC4C4A0123B5F1C5
:1055B000804FA5EB020284F84830B2FA82F284F8F8
:1055C0003E3084F83F304FEA521284F8403084F87D
:1055D000413084F8423084F8433084F8443084F811
:1055E000453084F8463084F8473084F83D3034D074
:1055F0009ABB3B4B9D420CD003F580639D4208D083
:1056000003F580639D4245D003F578439D4241D028
:1056100070BD94F83C30012BFAD00222314B0121AD
:1056200084F83D20A8680340AB6084F83D1084F8FE
:105630003D206B68A96823F0700321F080010122EE
:105640006B600023A96084F83D2084F83C3070BD75
:10565000636883423AD0606093E794F83C30012B52
:10566000D6D002211F4B002084F83D10A9680B40C2
:105670000121AB6084F83D10022384F83D306B6853
:10568000A9680AB90028D6D023F47003D3E784F8B8
:105690003C2083E794F83C30012BB9D00221114B18
:1056A000114884F83D10A968281A0B40B0FA80F020
:1056B0000121AB600023400984F83D1084F83C30A0
:1056C0000A4B9D42D8D00028D6D170BDE368B342C2
:1056D0007FF457AF70BD00BF0AD7233C00000140E4
:1056E000000400408800CEFF00040140000C004090
:1056F000024B0348D3F8CC15FCF74EB9802D00249B
:1057000000000140034B4FF08040D3F8D015FCF768
:1057100043B900BF802D0024024B0348D3F8D415B1
:10572000FCF73AB9802D002400040040024B0348E6
:10573000D3F8D815FCF730B9802D002400080040BC
:10574000024B0348D3F8DC15FCF726B9802D002462
:10575000000C0040024B0348D3F8E815FCF71CB9D5
:10576000802D002400040140024B0348D3F8F815B3
:10577000FCF712B9802D002400180040024B0348AA
:10578000D3F80416FCF708B9802D0024004001402E
:10579000024B0348D3F80816FCF7FEB8802D00240E
:1057A00000440140024B0348D3F80C16FCF7F4B850
:1057B000802D00240048014010B5064C0648D4F85E
:1057C000E815FCF7E9F8D4F8FC150448BDE81040EA
:1057D000FCF7E2B8802D002400040140001C0040CA
:1057E00010B5064C0648D4F8E815FCF7D5F8D4F8FF
:1057F00000160448BDE81040FCF7CEB8802D002408
:105800000004014000200040BFF34F8F0549064BC4
:10581000CA6802F4E0621343CB60BFF34F8F00BF4E
:10582000FDE700BF00ED00E00400FA0500210120C3
:1058300008B50CF015F872B6FFF7E6FF2DE9F04356
:10584000BFB0BFF35F8FA14C0023626A22F48032A5
:105850006262C4F894309DF843109DF844C0090674
:105860009DF842200F9841EA0C7141EAC2419DF82F
:10587000452041EA82419DF8462041EA42419DF897
:10588000472041EA02419DF8412041EA02219DF86A
:10589000402041EA4201C4F898300133D4F8A020F6
:1058A000112B22F00102C4F8A020C4F89C00C4F817
:1058B000A010F0D10523C4F89430636A43F4803318
:1058C0006362BFF34F8FBFF36F8F8148814A824974
:1058D000121A7DF0D5FA814B5A6D012A00F0DF8053
:1058E000D4F8881000227E4B012041F47001C4F8E6
:1058F000881018601A61196841F0800119601968F0
:1059000001431960196841F480311960196841F444
:10591000805119609A61DA611A629A62DA621A63D6
:105920005A639A63DA631A645A64196821F480210D
:1059300019601A664FF000636A49C1F80801A36054
:1059400078F0C6F8684AD36813F0040FD36840F0C3
:105950009480664B0021644A0591D96A21F00101C7
:10596000D962DB6A03F001030593936943F4404372
:105970009361936903F440430593059B93699804ED
:10598000FCD54C2200210EA8594C7EF0A1FE594AAC
:1059900042F20303A4F110011268B3EB124F4FF06F
:1059A00000024FF0040308BF0C460892E268A3709F
:1059B000002A4FD04D4BD96A21F00101D962DB6A30
:1059C000494903F0010308938B6923F440431343CF
:1059D0008B618B6903F440430893089B424A9369A7
:1059E0009904FCD53E4B4FF4403543480321D3F88E
:1059F000E02042F08002C3F8E0200122D3F8E0303A
:105A000003F080030793079B85610D9BCDE900138D
:105A1000002377F00BFF022301204FF48031A2888E
:105A2000CDE9173304231993A379CDE90E01E07969
:105A3000217A1C900EA81D91CDE91A23082200237B
:105A4000CDE91E23FAF70EFF032800F04982002853
:105A500058D0FEE7244A254B916941F440419161B9
:105A6000926902F440420892DA6A42F00102DA6274
:105A7000DB6A03F001030893AFE723F007031F4C31
:105A800043F00203D360216805E023685B1AB3F595
:105A90007A7F3FF65EAF53689D04F6D559E7104A0A
:105AA000002017495865D2F8F43043F00203C2F8D9
:105AB000F430D2F8F43003F002030E930E9B0B681F
:105AC00083F308884B689847FEE700BF00ED00E0CD
:105AD00000000000603700006CCC0D08004000584A
:105AE0000044025800800051004802580004005849
:105AF0002C0400240010005C001C0258802D00249F
:105B00000098F01F764B1A6812F00E0F0BD11A682E
:105B100022F00F0242F002021A601B6803F00F032A
:105B2000022B40F0DF816F4A936903F070033F2B33
:105B300005D8936923F0700343F040039361694AE9
:105B4000D36903F070033F2B05D8D36923F07003AA
:105B500043F04003D361634AD36903F4E063B3F5D0
:105B6000806F05D2D36923F4E06343F48063D3618B
:105B70005C4A136A03F070033F2B05D8136A23F0C5
:105B8000700343F040031362564B9A69120705D421
:105B90009A6922F00F0242F008029A61514A936911
:105BA00023F47063936113689B0130D5136941F24C
:105BB00088314D4C23F0070343F003031361206841
:105BC00004E023681B1A8B4200F29581136903F0ED
:105BD0003803182BF5D1936903F00F03082B05D96F
:105BE000936923F00F0343F0080393613C4A136861
:105BF00003F00F03022B0BD9136823F00F0343F0BC
:105C000002031360136803F00F03022B00D0FEE7BA
:105C1000344A936903F07003402B05D9936923F04C
:105C2000700343F0400393612E4AD36903F070037D
:105C3000402B05D9D36923F0700343F04003D361AF
:105C4000284AD36903F4E063B3F5806F05D9D369BB
:105C500023F4E06343F48063D361224A136A03F0C0
:105C60007003402B00F23F811E4EFCF7C7FA1F4D18
:105C7000B269B369C2F303221D4B134493F8303069
:105C800003F01F0320FA03F3D5F8A400C5F8A030F1
:105C9000FCF740F9002840F075811023159017900B
:105CA0000EA80E93FAF7DEFD002840F01881336845
:105CB000104A43F080033360D6F8F43043F0020317
:105CC000C6F8F430D6F8F43003F002030493049BD2
:105CD000136A43F001031362074B216811E000BF10
:105CE0000020005200440258802D002400000024AF
:105CF00018A10C080004005880380100013B00F096
:105D0000EF8022689142F9D0226823689B1A0A2BFF
:105D1000FBD900214FF480209B4C4FF44013002608
:105D200000273093CDE90E010EA876F0A5FED4F839
:105D3000EC30964941F2030243F002030EA8C4F886
:105D4000EC30D4F8EC3003F002030393039BD4F857
:105D5000943043F00203C4F89430D4F8943023F024
:105D60000203C4F894300B688949B2EB134F894B96
:105D7000894A28BF0A465A601A6822F47C5242F4C3
:105D800000521A601A6842F060021A60032200236F
:105D9000CDE92C67CDE90E2376F06EFE4FF4E0429C
:105DA00000230EA8CDE9266700270326CDE90E23A0
:105DB0003A9776F061FE182200230EA82F973497A9
:105DC000CDE90E2376F058FED4F8E0304FF4807120
:105DD000724843F00103C4F8E030D4F8E03003F037
:105DE000010309933B46099A0222CDE9006777F047
:105DF0001DFD23694FF40071694823F0FE7343F0E1
:105E000088732361D4F8E03043F00403C4F8E03031
:105E10003B46D4F8E02002F004020692069A0222E1
:105E2000CDE9006777F002FD236923F07E4343F05C
:105E3000FC432361FCF7E2F9C5F8A000BFF35F8FD4
:105E4000584C3E46584D4FF00108636A23F48033A6
:105E50006362C4F8947027E0002A4BD02F686B7AF5
:105E6000103515F8061C1B0643EA017343EA42038A
:105E700015F8052C43EA824315F8042C43EA424303
:105E800015F8032CC4F8986043EA0243D4F8A02024
:105E900043F0010322F00102C4F8A020C4F89C7072
:105EA000C4F8A03046BB01266B682A7A002BD3D0F9
:105EB0002F68002AD3D127F01F02A3EB0209B9F102
:105EC000200F38BF4FF0200948467DF013FB421EDB
:105ED00008FA02F1894508BF0246D2B2BFE7FEE7E1
:105EE000FFF7A4FC93E6136A23F0700343F040032A
:105EF0001362B9E6FEE78AE60523C4F89430636AC4
:105F000043F480336362BFF34F8FBFF36F8FBFF3F0
:105F10004F8FBFF36F8F0022C4F85022BFF34F8F13
:105F2000BFF36F8F636943F400336361BFF34F8F37
:105F3000BFF36F8FC4F88420BFF34F8FD4F8805025
:105F400043F6E0761749C5F34E34C5F3C90564013D
:105F500004EA06002B4640EA8372013BC1F8602246
:105F6000F9D2203C14F1200FF2D1BFF34F8F4B69CF
:105F700043F480334B61BFF34F8FBFF36F8F3FB05C
:105F8000BDE8F08343E600BF004402580010005C07
:105F90007FBB2200008400407FBB223000000258FB
:105FA0000008025800ED00E03C0400242DE9F8430D
:105FB000384E984606EB8003D3F8E040002C66D0BC
:105FC00004F1D20306F580760546B4F8D202A36147
:105FD00004F5E97366601746E3614FF48073261D8C
:105FE000E160C4E904332368C4F8CC30A36300281B
:105FF0004AD194F8D10009F00BFB18F0080F94F87F
:10600000D09034D1BA0723D4FB0711D4052194F8DA
:10601000D6026DF07BFF94F8D63201221E4903F0C0
:106020001F005B09824041F823203046BDE8F88319
:106030000135484609F0ECFAEDB218B140F20663BA
:106040000572C38094F8D422022109F0BFFADDE77B
:106050006B1CDBB218B1037240F20653C38094F894
:10606000D522022109F0B2FAFB07CFD5E0E70135CE
:10607000EDB218B140F206730572C38094F8D522D0
:10608000022109F0A3FAC1E76DF03CFDB1E7264615
:10609000CBE700BF18A10C0800E100E00148FCF7C5
:1060A00055BD00BF600400240148FCF74FBD00BF90
:1060B000380700240148FCF749BD00BF100A00243E
:1060C0000148FCF743BD00BFE80C00240148FCF781
:1060D0003DBD00BFC00F00240148FCF737BD00BF25
:1060E000981200240148FCF731BD00BF7015002450
:1060F00070B52422456B00238168C0F8BC2004469B
:106100002A6800F1340622F001022A602B606B60DD
:10611000AB608279C0F8C43080F8B830C0F8BC30C9
:10612000C364C0F8C0304365C0F8A030C0F8A430E4
:106130009302816303F480534179C363130303F42F
:1061400000530364130203F480634364C36D01F0DE
:106150000200C90745D400287ED1A06412F00802CD
:1061600054D0D4F8BC20002A00F08A802422C4F83D
:10617000BC202A6822F001022A60002B7CD1304624
:10618000FCF7D2F9012812D06B68304623F4904313
:106190006B60AB6823F02203AB60AB6843F008038D
:1061A000AB602B6843F001032B6076F09DFA6279B7
:1061B000D6070DD5D4F8C830196841F4807119603C
:1061C000996841F001019960196841F02001196056
:1061D000950705D5D4F8C820136843F080031360F1
:1061E00070BD0421A16470B30C21D007A164B5D5A2
:1061F0004FF4803143F00203616643F001034FF432
:106200000031E365216612F00802AAD1D4F8BC106F
:1062100009B194F8B82084F8B8202422C4F8BC202E
:106220002A6822F001022A6013BB3046FCF77CF991
:106230000128BCD06B68304623F490436B60AB6898
:1062400023F02A03ACE7D10788D543F002034FF4CB
:106250008031E365616681E70821A164D1077FF59C
:106260007DAF43F001034FF40031E3652166CAE7D7
:106270003046FAF7A1FED8E73046FAF79DFE7EE7F2
:1062800084F8B82072E700BF816031E741712FE7E1
:1062900081712DE710B51C2009F0BAF904461121CF
:1062A00009F072F9204606F0F5FAC8200DF036FA2A
:1062B00014B12368A2889A6110BD00BF2DE9F04F88
:1062C000DFF8B4B38BB0DBF82CAADAF8143013F093
:1062D000010902D00BB0BDE8F08FDAF81420DAF82B
:1062E00018301A42F6D0DAF808280AF50061DAF810
:1062F0001430C2F30D220291CBF8002FDAF81820E7
:1063000013409D0705D5DAF8143003F00203CAF8EC
:106310001430DAF81430DAF818201340DC061BD5F4
:10632000DAF8183023F01003CAF81830DAF8203001
:1063300003F4F01203F00F05B2F5802F00F0498549
:10634000B2F5402F00F02583CDF804A0019A93699F
:1063500043F01003936101E0CDF804A0019A536962
:1063600092691340180300F19C82019A5369926963
:1063700013405F0300F1D281019B5A699B691A4265
:1063800000F1EA80019A5369926913401B0509D50F
:10639000029B9B68DF0700F16485019A536903F44F
:1063A0000063536101994B698A6913401E0116D538
:1063B0004B6903F000634B619BF8F83E002B00F043
:1063C000C282DBF80C3F93F89C22042A04D093F895
:1063D0009C22D2B283F89D22042283F89C22019A47
:1063E000536992691340DD0400F14881019A5369B1
:1063F000926913409C0400F1D780019A5369926915
:106400001340190700F1C38001994B698A69134051
:106410001A067DD44B698A691340DB0228D59BF8A4
:10642000308AB8F1010F1ED9924D0AF51267012684
:1064300004E0013620372435464514D095F83C3029
:106440003A68012BF5D1002AF3DA66F07F0085F86F
:106450003B30C0B26EF066F8EBE7019A536992697F
:106460001340DA0204D5019A536903F4801353618F
:10647000019A5369926913409F0231D59BF8307A93
:10648000012F28D90AF532627A4B012103E0B94283
:1064900003F124031FD093F87C02013114682032E9
:1064A0000128F4D1002CF2DADBF8005F85EA14450C
:1064B000EE07ECD483F87B02DAF8180040F0800095
:1064C000CAF81800DAF814000506E0D4029A5368F6
:1064D00043F400735360019A536903F4001353614A
:1064E000019A5369926913405C0000F1BD800199E3
:1064F0004B698A69134058077FF5ECAE4C68610719
:1065000000F1BF84DBF82C3A5A6814435C60E1E682
:10651000DAF818309BF8308A23F08003B8F1010FC5
:10652000CAF8183099D9534D01262F4603E0013699
:106530002437464507D097F87B32012BF7D1F0B2CC
:106540006DF0F0FFF3E7019B5A699B691340DB0292
:106550008ED59BF8308A68E7029A536823F00103CE
:1065600053609BF8F83E012B00F00182DBF80C3FF2
:1065700093F89C22042A04D193F89D22D2B283F886
:106580009C22019A536903F000435361FAE6DBF859
:106590000C0F90F89C32032B00F0ED81019A5369A7
:1065A00003F0080353612FE7019AD2F800396FF323
:1065B0000A03C2F8003902F50063D2F8042842F455
:1065C00080725A609B68980700F1F78113F0060FFC
:1065D0000CBF00230F238BF8333AFBF731FE9BF8F7
:1065E000336A022E00F06F844FF410530199003E7D
:1065F000DBF80C5FCA6818BF012622F47052CA602B
:10660000CA681343CB600123002185F89C32D5F87A
:10661000B8326960C5F8A41285F8A012C5F89412C2
:106620001BB15B680BB12846984700224024012724
:1066300040231146284675F0EBFC234600228021BA
:106640002846C5F86041A5F8647175F0E1FCDBF8F7
:106650000C3FDBF82C2AAF842C621E745369019224
:1066600003F400535361C8E6019A536903F0804371
:1066700053613CE7AC370024802D0024029A10219E
:106680000198536823F001035360FCF795FD9BF8D4
:10669000300AE0B10AF510634FF67F31996009F1D5
:1066A00001091A682033814522F4001243F8202C96
:1066B000C3F8E811D3F8E02122F40012C3F8E02176
:1066C000D3F8E02142F00062C3F8E021E6D1029A5B
:1066D000D36943F00113D3619BF83B3A002B00F0E0
:1066E0003B81029AD2F8843043F00B03C2F8843025
:1066F000536C43F00B035364DAF80038019C23F425
:10670000FE63B44A2046CAF800389BF8321A75F086
:1067100001FD636903F48053636167E6019AD2F86F
:106720001878D2F81C381F40BFB2002F3FF424AEB7
:106730000AF510614FF00008CDF80CA01346A64DE5
:1067400044468A46CDF8109008E07F0804F1010421
:1067500005F124050AF1200A00F03181FE07F4D585
:10676000D3F8102804F00F01D3F834684FEA441925
:10677000CE40F601F6B2164303F5106202EB441266
:1067800092681640E2B2F007019221D50120029AE8
:10679000DBF80C8F526B00FA01F122EA0102029938
:1067A0004A639BF8321ACAF80800814200F07883E5
:1067B0002B6A0593002C40F0FA82D8F89432022B11
:1067C00000F0E88398F8A03213B1002388F8A032D3
:1067D000320702D50823CAF80830F30602D5102381
:1067E000CAF80830700602D54023CAF80830B1074D
:1067F00000F110813206DBF82C3AA6D5D5E909065E
:106800008642A2D8811BEA6903F5106E8A42CE4403
:1068100028BF0A46DEF81810033289B2B1EB920F96
:1068200031D39BF8328A03F5805C019442460CEB2D
:10683000043C98461346B04240F29083811BEA69BB
:10684000914228BF11462A6A01F103094FEA9909CA
:1068500073B98CB20334A4080AD002EB840452F852
:10686000040BA242CCF80000F9D12A6AD5E9090646
:106870000A440E442A62DEF81820AE6292B29145B4
:10688000D9D9019C4346B0423FF65FAF04F00F02F6
:1068900001219140D3F8342822EA0102C3F83428B8
:1068A00053E70198D0F81838D0F81C2813405FEA55
:1068B00013483FF45AAD484B0AF53066CDF80CA0AA
:1068C00000279A46CDF8149008E05FEA580807F1CF
:1068D000010706F120060AF1240A74D018F0010914
:1068E000F3D0FBB200F530627D01019302EB471358
:1068F0009C68D0F814180C40E1076FD4210700F110
:106900009580E50601D51023B360A0070FD5039B42
:106910005B69190604D5029A536843F48063536097
:106920009AF85732012B00F01C830223B360A206B1
:1069300001D52023B360A30402D54FF40053B36004
:10694000DBF82C0AC1E701238BF8F83E4B6DC3F34B
:106950008303CBF8FC3E42E5029942F22B034A69DD
:1069600013434B610B6943F00B030B61C4E6002337
:106970008BF8F83E05E6D0F8B832002B3FF40EAEA7
:10698000DB69002B3FF40AAE9847DBF82C3A019301
:1069900004E605EBC5020AF58051C3F30A130BEBBD
:1069A0008202D2F8940C03440868CBF8C80E096838
:1069B000C2F8943CCBF8CC1EC6E402230BE6DDE91A
:1069C00003A90193D8E4DDF80CA0DDF81490019040
:1069D000CBE400BF483C0024AC3700240121B16067
:1069E0009BF8321AD0F840E00129D3F808C000F033
:1069F000A582B6498E4500F09B83DBF8903C3B4373
:106A000000F04984DAF860220199DBF80C0F75F088
:106A1000B3FD73E721460398FCF7CEFBEB7D012B1A
:106A200000F091830223CAF80830E3E6DBF82C2A51
:106A30000823B36002F53063126C2B4410460492B5
:106A4000A34A9968904204D90A0402D54FF400423F
:106A50009A60DBF80C5F01219BF8C83E05F2AA2082
:106A600085F8AA329BF8C9EE079085F8ABE2BBF82F
:106A7000CA2EA5F8AC22BBF8CCCE0692A5F8AEC2C1
:106A8000BBF8CE2EC5F8941203F01F01A5F8B02272
:106A90000129C5F8982200F0A582022900F0078399
:106AA000002940F0DE8203F06003202B00F0E98330
:106AB000402B00F0E683A3B9BEF1090F11D8DFE83F
:106AC0001EF0E800C1001000D80010007D00640036
:106AD00010003E002300D5F8B4325B69002B40F073
:106AE000C285284675F0D8FB794B049A9A427FF606
:106AF00008AF9BF8321A01297FF403AF754ADBF81F
:106B00002C0A75F007FBFCE69DF81890B9F1010F0F
:106B10008BF8109FE5D895F89C32DAB2022B0692DA
:106B200000F00385032A00F0D784284675F0B4FBF3
:106B3000D5F8B832494628465B689847D4E7012A19
:106B4000CFD195F89C120229CBB200F2A684002B7B
:106B5000C7D0D5F8C832002128464FF0020C40F8C3
:106B6000081FC5F894C2C5E90622C3E909211862C5
:106B70004FF4807203F114019A829A79012A08BFB6
:106B80001863186875F0C2FBAEE7069B00221B0A6B
:106B9000ADF82620013B062BA3D801A252F823F022
:106BA000816D0408656D04083B6D0408E36A040800
:106BB000E36A0408D96C0408936D040852EA0C0CCB
:106BC0008FD1069B7F2B8CD895F89C32032B88D0D5
:106BD0000698D5F8C8325FFA80F985F89E9293F846
:106BE0009424012A12D01A684FF0000C83F81190F7
:106BF000D2F8001821F4FE61C2F80018D2F800188B
:106C000041EA0011C2F8001883F894C4042200205D
:106C100003F11401C5F894224FF48072A8619A829E
:106C20009A799862012AC3E9080008BF18631868B6
:106C300075F06CFBB9F1000F40F07284012385F808
:106C40009C3251E795F89C32013B022B3FF649AF4D
:106C5000069B012B7FF448AF0020D5F8C832C5F859
:106C6000A402A8610422C5F894229862C3E908002E
:106C70007EE7069B012B00F06F84069B022B7FF4BE
:106C800030AF4FEA1C2CD5F8C832002085F8A0C2DE
:106C9000E7E795F89C32013B022B3FF622AF022A30
:106CA0007FF41FAFD5F8A4322846002B18BF4FF051
:106CB000030940F80C9FD5F8C832C5F89422C5E9FD
:106CC0000622C3E9080200229A6251E70A31544FB2
:106CD0000A30544F483C00242B7C002B7FF401AF3A
:106CE000D5F8B8320DF126005B6B98470346B5F82E
:106CF000B002002800F03884BDF82620002A3FF4B6
:106D0000F0AE82424FF0020128BF0246D5F8C80219
:106D1000C5F8941200F11401C5E90622C0E9083251
:106D2000002282624FF4807282828279012A08BF37
:106D30000363006875F0EAFAD6E69DF818000528A6
:106D40003FF6CFAE01A353F820F000BF9F760408B2
:106D5000917604088376040875760408D76A0408D7
:106D60005B7604082A7CD5F8B832002A40F0728499
:106D70009B6A0DF126009847022203464270B6E74F
:106D8000D5F8B4320DF12601287C1B6898470346DC
:106D9000ADE72B7C002B7FF4A4AED5F8B8320DF113
:106DA00026001B6B98470722034642709FE798F81E
:106DB0009C32032B7FF40CADD8F8B8325B69002B02
:106DC0003FF406AD002240460199C8F8D422984706
:106DD000FEE447F6F07213423FF4B6AA05EBC50293
:106DE000C3F388144FEA131CC3F301130BEB8202A5
:106DF000EE00D2F88C7C002C00F000830AF5805E57
:106E0000002239460132DEF80000944241F8040BBA
:106E1000F8D107EB8404002B00F0BC810AF5805206
:106E200023441068002220FA02F1083204F8011B02
:106E30009C42F8D173190BEB8303D3F88C7CDBF8FD
:106E40002C3A01937319CCF30A0C0BEB83036744C0
:106E5000D3F8942CC3F88C7C6244C3F8942CFFF7CD
:106E600075BADBF80C3F93F89C22042A04D093F8FF
:106E70009C22D2B283F89D22042283F89C22FFF741
:106E80008CBADBF80C0F0122D0F8B83280F89C22C3
:106E9000002B3FF437AB5B6801799847FFF732BBB3
:106EA000D5E9070202442A62002C80D1DBF84C0AA3
:106EB000DBF8502A0590002A7FF47FAC1846B74AC9
:106EC00075F028F979E4B64BB64A0344934240F290
:106ED0005281B54BB54A0344934240F25781B44BBB
:106EE000B44A0344934240F23582B34BB34A03445D
:106EF0009342C0F06B82B24BB24A0344934240F2D9
:106F00009182B14BB14A03449342C0F08F82B04B9F
:106F1000B04A03449342FFF467ABAF4BAF4A03441C
:106F20009342C0F0D582AE4BAE4A034493422CBF8D
:106F30004FF4C0534FF4E053FFF758BB1CF0080F59
:106F400000F01D81A84A96457FF6D8AC1CF4004F8E
:106F50003FF4D4AC4FF400429A60CFE4019C434626
:106F600094E400238AF85732DBF80C0FD0F8D432BF
:106F7000AE3350F82330002B3FF4D7AC90F89C226E
:106F8000032A7FF4D2AC5B6A002B3FF4CEAC0199AC
:106F90009847CAE4D8E90732934200F2278100F00B
:106FA000988198F89C32032B00F0C88180214046DC
:106FB00075F036F905230020C8F89432D8F8C832A5
:106FC0009A7903F51571C3F86802012AA3F85402EF
:106FD000C3E9980008BFC3F87002186875F096F905
:106FE000FFF7F0BB03F060025B0602D5402A7FF496
:106FF00078AD95F89C32013B022B3FF672AD5FFAFB
:107000008CFCBCF1030F3FF66CADD5F8B8329B6831
:10701000002B3FF469AD4FF0000907992846C5F8E9
:10702000D4929847B5F8B022002A7FF45DAD0028CD
:107030007FF45AAD0422D5F8C832C5F81890C5F8C7
:1070400094224FF4807203F11401C3F828909A82BD
:107050009A79012AC3E908997FF493ADC3F8309077
:107060008FE51B06D5F8C85200F12D81002385F865
:10707000553205F5157301224FF000099A7083F817
:10708000009095F8941491423FF42EAD286885F84D
:1070900094245A781978069075F088F8069805F2C5
:1070A0009C42A97975F036F885F894941CE503F0B4
:1070B0006003202B00F07C81402B00F07981002BB5
:1070C0007FF40FADBEF1010F5FFA8CF100F0468145
:1070D000BEF1030F00F07E81BEF1000F7FF401AD21
:1070E00095F89C32022BDAB200F0A481032A7FF4D7
:1070F000F8AC01F00F0314221CF0800F02FB0353C5
:1071000040F0B281B3F86431002B3FF4EAAC02FBEB
:10711000015202F5AA70002940F02B82002303607F
:10712000D5F8C8320222C5F89422C5E90622C8E57E
:107130001CF4004F7FF40EAF1CF0200F3FF462AC44
:1071400020229A605EE40023EB75DBF80C0FD0F888
:10715000D432AE3350F82330002B3FF463AC90F8B8
:107160009C22032A7FF45EAC1B6A002B3FF45AACCE
:107170000199984756E44FF47053FFF737BA1CF063
:10718000200F60D020229A60FFF7B8BB4FF4605305
:10719000FFF72CBACDF804A054E600BF483C002409
:1071A000405327FFFF340C00401E1BFF3F420F00DF
:1071B00000DC0BFF7F4F1200808CF9FE20D61300FD
:1071C00060B6E5FE5FE3160000D3CEFE40771B00FD
:1071D000C05BB3FEC091210000CA91FE207538004B
:1071E000E05459FEE09C41000A30544F9A1AD8F8F6
:1071F000C832C8E906225A6203F11401059A1A62DC
:1072000000229A624FF480729A829A79012A01D1FF
:10721000059818631868CDE9050375F077F8069BA3
:1072200000209A7903F51571C3F86802012AA3F8C2
:107230005402C3E9980008BFC3F87002059875F0BE
:1072400065F8FFF7BFBAC64A964503D91CF4004F4C
:107250007FF480AE1A69DAF87432C2F312029B1A14
:10726000CAF86832002F7FF4CDABDBF8902C002AEF
:1072700000F0D280DBF88C2C1A44CBF88C2CFFF772
:10728000C1BBD5F8D43228460799AE3355F8233020
:107290009B68984728E4016CB14B994203D9136865
:1072A000002BFFF6AFAB00231361136943F40023F7
:1072B0001361136943F018031361136943F0C0436A
:1072C0001361FFF79FBB4FF001036B7505F11403CA
:1072D000D1E6D8F8182093423FF663AED8F898323A
:1072E0009A42BFF45EAED8F8C83200204FF48072E4
:1072F000C8F8180003F114019A829A799862012A59
:10730000C3E9080008BF18631868CDE9050374F0E5
:10731000FDFF069B4FF0000C059803F51571C8F8AA
:1073200098C29A79C3F868C2012AA3F854C2C3E983
:1073300098CC7FF453AEC3F870C24FE6D8F8B83299
:10734000DB68002B3FF432AE00224046C8F8D4225E
:1073500098472BE64FF45053FFF748B995F89C3205
:10736000022BDAB24CD0032A7FF4BBAB069B002B76
:107370007FF4BAAB4806D5F8C89240F006810422E3
:10738000002309F11401D9F80000C5F894224FF444
:107390008072AB61A9F8142099F80620C9F828304A
:1073A000012AC9E9083308BFC9F8303074F0AEFFCC
:1073B000D5F8B83200229B68C5F8D422002B3FF4E0
:1073C00093AB079928469847FFF78EBB4FF440537D
:1073D000FFF70CB995F89C32022B5FFA83FC0FD0B3
:1073E000BCF1030F7FF47DAB480603D0069B13432B
:1073F00000F0C780D5F8C832002032E43C460AE5E8
:107400004B0628463FF46EAB74F00AFF28468021F5
:1074100074F006FFFFF768BB524A012174F07AFE50
:10742000FFF7F0BA4FF43053FFF7E0B84FF42053B2
:10743000FFF7DCB84A067FF454AB1CF0800FD5F898
:10744000C8324FF002024FF0000114BF05F11400E2
:1074500005F5AA700160C5F89422C5E90622C3E9C2
:1074600009211862FFF784BB9B8C002B3FF439ABDA
:1074700001F07F01481C00EB800005EB8000002933
:107480003FF44CAE2422D5F8C83202FB01318A7D8C
:10749000003A18BF0122026044E6032B7FF421ABBF
:1074A000D5F8C8320221C5E90622C5F89412043580
:1074B0005A62002203F114011D629A624FF4807235
:1074C0009A829A79012A7FF45CAB1D63FFF759BB5E
:1074D0004FF40053FFF78AB8B9F1000F00F0AE8007
:1074E0006968012986D0D5F8B832C9B228465B68E8
:1074F00098479BF8101FD5F8B8326960002B3FF40D
:1075000079AF1B682846984700283FF473AF284698
:1075100074F0C2FED5F8B832297928465B689847DE
:10752000022385F89C32FFF7DFBAB9F1000F3FF470
:1075300081AD0121D5F8B8326960002B5AD01B68A3
:1075400028469847002855D0284674F0A5FE069B8B
:1075500085F89C32FFF7C8BAC5F8A4324AE700BFE5
:107560000A30544F483C0024D5F8C832A861FFF7D0
:1075700079BB2422D5F8C83202FB013191F856229A
:1075800086E7284674F04CFE34E701F00F0199F8C5
:1075900004308B42FFF4F3AE01EBC1031CF0800F0B
:1075A0004FEA830341D103F51573002209EB030C65
:1075B000242303FB019383F855224FF000038CF83A
:1075C00000108CF8023099F89434012B3FF4D7AEB8
:1075D0000123D9F8000089F894349CF804309CF811
:1075E00001209CF8001074F0BBFD4FF0000389F8F7
:1075F0009434C4E60422D5F8C8320020C5F8942299
:107600004FF48072A86103F114019A829A7998620A
:10761000012AC3E9080008BF1863186874F076FEF1
:10762000032385F89C32FFF75FBA1433012209EB7C
:10763000030C242303FB01935A75BEE7022349463A
:107640002846C5F8049085F89C32D5F8B8325B68B6
:107650009847EFE4DB6AFFF78CBBD5F8B4329B693F
:10766000002B3FF43EAA0DF12601287C98470346E3
:10767000FFF73DBBD5F8B4321B69002BF3D1FFF700
:1076800030BAD5F8B432DB68002BECD1FFF729BA59
:10769000D5F8B4329B68002BE5D1FFF722BAD5F8B4
:1076A000B4325B68002BDED1FFF71BBA2DE9F0473F
:1076B0004A4FD7F85453EE682C69A30701D5B00799
:1076C00036D4610701D572072AD4230701D53007C4
:1076D0001ED4E10601D5F20612D4E30701D5F00766
:1076E0003BD414F4025F2BD031066CD4600601D574
:1076F00071066ED4A20601D5B30629D4BDE8F08781
:107700006FF010032B610023EA6987F87033E4E718
:107710006FF008032B610023EA6987F87033D8E71C
:107720006FF004032B610023AA6987F87033CCE75C
:107730006FF002032B610023AA6987F87033C0E75A
:10774000E305D3D53706D1D56FF480732B61CDE730
:107750006FF020032B61BDE8F0876FF001032B6110
:107760001F4B9D42BDD1D7E9B9839845B9D098BF89
:10777000A3EB0809D7F8DC321A4A88BFC8F580594C
:1077800007EB83034244D3F8C832002BA9D0D3F8C7
:1077900014A2C3F80822C3F81092BAF1000FA0D1C6
:1077A0000121C8441048C3F814124B468121C7F880
:1077B000349074F0BBFEB8F5805F14BF4346534667
:1077C000C7F8E4328DE76FF40253E2052B618DD5E3
:1077D000BAE76FF040032B618CE700BF802D0024D7
:1077E00000140040944C0024882D002470B4154DE2
:1077F00000202B4693F82A4014B1DE698E4205D052
:10780000013010330828F5D170BC7047AAB1AB69BC
:1078100003EB40239A4201D1022C07D095F8B831EE
:1078200013B9012385F8B83101236B7005EB0015FE
:10783000012385F82A3070BC704705EB001585F8E8
:107840002A20E1E7A05C002430B40023184C204635
:1078500084F8A43003E001331030082B1AD0C56936
:107860008D42F8D190F82AC0BCF1030FF3D19AB140
:10787000A16901EB43218A4207D094F8B82112B9DB
:10788000012284F8B8210122627004EB0314012361
:1078900084F82A3030BC7047D4F8A02004EB0313DE
:1078A0000421013283F82A10C4F8A020F2E700BFB7
:1078B000A05C0024A0B183681BB10C4B07229A7016
:1078C00070470A4A04211078137503289170C2E9A1
:1078D000033314BF4FF480738023C2E90133704730
:1078E000024B012283F8B8215A707047A05C002433
:1078F000234910B54C8891F800C0644530D96346DF
:10790000E646624603E0944238D991F800E07144BB
:10791000724491F801E092B2BEF1050FF3D191F8F3
:1079200002E0BEF1810FEED1154A03E0A3421BD263
:1079300092F800C06244634492F801C09BB2BCF16B
:10794000050FF3D192F802C0BCF1010FEED119B1CD
:10795000002402230C714B71002102231171537119
:1079600020230380064810BD0029F9D002230022FD
:107970004B7120230A710380014810BD0021D3E719
:1079800048180024234910B54C8891F800C064457C
:1079900030D96346E646624603E0944238D991F80E
:1079A00000E07144724491F801E092B2BEF1050F1B
:1079B000F3D191F802E0BEF1810FEED1154A03E058
:1079C000A3421BD292F800C06244634492F801C003
:1079D0009BB2BCF1050FF3D192F802C0BCF1010FCC
:1079E000EED119B1002440234C710B7100214023CA
:1079F0005171137120230380064810BD0029F9D06E
:107A0000402300220B7120234A710380014810BDDE
:107A10000021D3E748180024234910B54C8891F879
:107A200000C0644530D96346E646624603E09442AE
:107A300038D991F800E07144724491F801E092B2B3
:107A4000BEF1050FF3D191F802E0BEF1810FEED146
:107A5000154A03E0A3421BD292F800C0624463447B
:107A600092F801C09BB2BCF1050FF3D192F802C0AD
:107A7000BCF1010FEED119B1002440234C710B7100
:107A8000002140235171137120230380064810BD4B
:107A90000029F9D0402300220B7120234A71038072
:107AA000014810BD0021D3E74818002403460A22EC
:107AB00001481A80704700BF68180024D0F8D4220B
:107AC00000EB82022DE9F041D2F8C0420646002CBC
:107AD0004ED0B4F8643204F11007D4F8705208465E
:107AE000D2F8C422394603FB05F5D2F81080B5F56B
:107AF000007FD4F86C2228BF4FF40075B5FBF3F378
:107B00009BB2C04700281BDB2B463A4681213046FA
:107B100074F00CFDB4F86422B5FBF2F2D4E99B13C7
:107B200011449B1AD4F83822521BC4E99B13C4F8A1
:107B3000382213B10020BDE8F08103232372F9E756
:107B4000D6F8D432B03356F823208AB192F8613295
:107B50000424112003F148010133DBB202F8314063
:107B600002EBC101A342888008BF002382F8613282
:107B70004FF0FF30DFE700BF38B5084BD3F82832AD
:107B800053B1DB6914460D4698474FF40073026801
:107B900000202A60238038BD1B68FFDEA05C002423
:107BA00008B5064BD3F8283223B11B699847013832
:107BB00040B208BD4FF0FF3008BD00BFA05C0024FC
:107BC0000020704700207047DFED0A7AB7EE007A98
:107BD0000023C0ED020A20EE270A0360C7EE007AF8
:107BE00030EEA77AC0ED017AC0EE877AC0ED037A55
:107BF000704700BFDB0FC940704700BF704700BF30
:107C000003685A1C02601970704700BF03685A1C51
:107C100002601970704700BF024BD3F82C02036852
:107C20001B681847A05C00242DE9F0413A4E3378D8
:107C30007E2B03D000273846BDE8F08108214FF4A1
:107C4000FC4341F221041AB25B00002A84EA42009C
:107C50009BB2B8BF83B20139F5D1B6F80140002C10
:107C600037D02E4A2E4DAA42E4D2052CA2F10602AC
:107C70008CBF002701271444AC4228BF47F00107FE
:107C8000002F47D141F2210EA24214D0501E04F120
:107C9000FF3810F8011F082283EA012319B25B00A4
:107CA00000298EEA410C9BB2B8BF1FFA8CF3013A4F
:107CB000F4D14045EDD1218861B1A21DAA42BAD2CA
:107CC000052904EB01002246B5D9A842B3D20446E7
:107CD000DAE7144C671E41F22105BC4617F8012F64
:107CE00083EA0223082219B25B00002985EA4100D9
:107CF0009BB2B8BF83B2013AF5D16445EDD1678834
:107D0000094AFF1A231DB7FA87F79B1B7F09A2F8C0
:107D1000303290E70F468EE70000020807000208A5
:107D20000000040801000208A05C002470B51C4E8D
:107D30000D2300223621022008F0BCFD706558B3E7
:107D4000002104F00DFE0BF0BBFC04460D460BF0C9
:107D5000B7FC001B61EB0501B0F57A7F71F1000102
:107D6000F5D3726D536913B119689B888B6192F9D1
:107D7000101000220B480A2301EB410150F831009A
:107D80001146FCF7CDFA084B012100221B6886F84A
:107D900024103276736170BD86F8240070BD00BF78
:107DA00074300024CC020024D0300024F8B51F4FDA
:107DB000D7F84025B7F84415D7F8283291614BB36E
:107DC0009B69984730B30026D7F8283213B11B6956
:107DD000984790B9B6F57A7F24D00BF071FC013644
:107DE00004460D460BF06CFC001B61EB0501B0F581
:107DF0007A7F71F10001F5D3E6E7B6F57A7F4FF0AF
:107E0000FF3018BF0020B7F84435D7F840251B04D1
:107E10009361F8BD064B03F12C02DB6AC7F82822F8
:107E20009847D0E74FF0FF30EDE700BFA05C00249B
:107E3000481800242DE9F0472F4E90469A46B6F890
:107E40005025D6F84C451304A361BAF1000F46D073
:107E50008946C24441F28937D6F828225AB1002314
:107E60005468494640461A46A047A8B9D6F8283271
:107E70000BB11B699847013F35D00BF021FC04463C
:107E80000D460BF01DFC001B61EB0501B0F57A7F80
:107E900071F10001F5D3DFE741F28937D6F82832D6
:107EA00013B11B69984780B9013F1CD00BF008FC47
:107EB00004460D460BF004FC001B61EB0501B0F518
:107EC0007A7F71F10001F5D3E8E708F1010809F5BF
:107ED0000079D045BED1D6F84C45B6F850250020E3
:107EE000A261BDE8F087D6F84C354FF0FF30B6F808
:107EF00050259A61BDE8F087A05C00242DE9F04789
:107F0000314E90469A46B6F85025D6F84C451304A3
:107F1000A361BAF1000F4AD08946C244D6F828229C
:107F20000AB341F289370023D468494640461A46CD
:107F3000A047D6F82832B8B10BB11B699847013F6A
:107F400039D00BF0BDFB04460D460BF0B9FB001B0E
:107F500061EB0501B0F57A7F71F10001F5D3D6F838
:107F60002822002ADFD1002341F2893713B11B698F
:107F7000984790B9013F1ED00BF0A2FB04460D4676
:107F80000BF09EFB001B61EB0501B0F57A7F71F1F0
:107F90000001F5D3D6F82832E8E708F1010809F521
:107FA0000079D045BAD1D6F84C45B6F85025002016
:107FB000A261BDE8F087D6F84C354FF0FF30B6F837
:107FC00050259A61BDE8F087A05C0024D0F8D43237
:107FD000B03370B550F823402CB30026124B054641
:107FE00084F83C12C4F8303204F50C7226720D236A
:107FF000812104F5047474F099FAD5F8C8321F226F
:108000000121C3F88C62A3F8781203F51E71186879
:10801000C3E9A1429A79012A08BFC3F89442BDE896
:10802000704074F073B970BD55534253D0F8D422E8
:1080300000EB82022DE9F041D2F8C0420646002C46
:1080400067D0B4F8643204F11007D4F870520846CF
:10805000D2F8C422394603FB05F5D2F81480B5F5F1
:10806000007FD4F86C2228BF4FF40075B5FBF3F302
:108070009BB2C047002834DBD4F83802B4F864223D
:10808000401BB5FBF2F5D4E99B13C4F83802294430
:108090005B1BC4E99B13FBB1D6F8C80202FB03F3D8
:1080A00001220021B3F5007FC0F88472A0F8782285
:1080B000827928BF4FF40073C0F88C1200F51E714E
:1080C000012AC0F8883208BFC0F89472006874F0C2
:1080D0001DF90020BDE8F08119463046FFF776FF14
:1080E000F7E7D6F8D432B03356F823208AB192F8A5
:1080F00061320424032003F148010133DBB202F8AA
:10810000314002EBC101A342888008BF002382F8FE
:1081100061324FF0FF30DDE7D0F8D43200EB83035B
:108120002DE9F043D3F8C04283B0002C00F0B780B3
:108130001646127805460F465A2A5FD85A2A00F288
:108140009B80DFE812F04701990099005B019900DC
:108150009900990099009900990099009900990057
:10816000990099009900990099008F019900990050
:1081700099009900990099009900AD01CE019900EC
:1081800099003E0199009900990099001102990007
:10819000370299009900FA0099005F02990099004E
:1081A00099009900E20199009900990099009900BD
:1081B00099009900990099009900990099009900F7
:1081C00099009900990099009900990099009900E7
:1081D00099009900990099009900990099009900D7
:1081E00099009900990099009900990099009900C7
:1081F00099009900990099009900F101A82A53D09B
:10820000AA2A00F065829E2A36D1D3F8C4320846E5
:1082100004F5197204F51A715B6898470146002845
:1082200040F0098394F86232022B00F00483D6F800
:108230000A301ABAE2601BB104F110007CF048FA6F
:10824000D4F868320022013B190E61F30702190CC1
:1082500061F30F22190A61F31742B4F8641263F351
:108260001F624BBA6383002362612383D6F80A300E
:108270001BBAE360002014E094F861220526202553
:108280000221531C4832DBB204F8326004EBC20016
:10829000042B858008BF0023617284F861324FF09F
:1082A000FF3003B0BDE8F08394F80880B8F1000F08
:1082B0007DD194F91C22002A80F2058394F8622271
:1082C000022A00F08083D3F8C43208469B6898479E
:1082D000002840F0DE82D6F80230D5F8D4121BBA5E
:1082E000B031C4F86C32D6F8062055F8211012BA15
:1082F000C4F870220029D2D01344D1F86802834216
:1083000000F24783B4F8643202FB03F3D4F8182276
:108310009A424AD091F861320524202003F14802A4
:108320000133DBB201F8324001EBC202042B908032
:1083300008BF002381F86132B1E794F80880B8F1F2
:10834000000F34D194F91C22002A80F2BC8294F8E8
:108350006222022A00F03783D3F8C43238469B6881
:108360009847002840F09582D6F80220D5F8D4121C
:1083700012BAB031C4F86C22B6F8073055F82110A3
:108380005BBA9BB2C4F87032002988D01A44D1F885
:108390006862B24200F27383B4F8642202FB03F312
:1083A000D4F818229A4240F0E182022323724FF45B
:1083B000007339462846E36003B0BDE8F043FFF799
:1083C0007DBB337900229B1AE26018BF012384F839
:1083D00062324FE7D4F81822002A40F0388294F82D
:1083E0006212022900F04583D3F8C43238469B68F4
:1083F0009847002840F0D282E0603BE7D4F818327A
:10840000002B00F024827021002294F86032217445
:108410000C21C4F81520E17594F86112C4F81120FC
:108420009942C4F81920C4F81D2084F8212011D0E5
:1084300004EBC30191F84012A17404EBC3010133B2
:10844000B1F84412DBB2A183042B14BF84F860326C
:1084500084F860221223E36032799A4298BF13466F
:10846000E36007E7D4F81822002A00F0F081727860
:10847000D20740F1B081B378002B00F0CE81802B81
:1084800040F0DF810821CC4A04F1180304F1100008
:10849000E16012F8011D03F8011D8342F9D1E9E6FC
:1084A000D3F8C4323846DB689847002840F074811E
:1084B0003279042A134628BF0423E360002A3FF4DC
:1084C000D9AE013BBC4A04F1100099B201F111038D
:1084D0000A44234412F8011903F8011D8342F9D11B
:1084E000C8E694F862223379012A03F0030300F00E
:1084F0006981012B00F06B81022B00F06981032B55
:1085000000F065810023E360B4E6737813F00203A2
:1085100040F09781D4E99B210A44D4F868128A423A
:1085200000F2E481E360A5E6D3F8C4323846DB68A4
:108530009847002840F03881337A082B194628BF25
:108540000821E160002B3FF495AE9C4A01F1100335
:1085500004F110000A4454FA83F312F8011D03F8E1
:10856000011D9842F9D185E6D3F8C4320DF102021B
:10857000384601A95B689847002840F06E8194F85E
:108580006232022B00F06981BDF8022008212061CF
:1085900052BA019BA061013B62830C22E174E37536
:1085A000190EE2601A0C1B0A217562750222A3756E
:1085B000227676E6D3F8C43204F51972384604F50B
:1085C0001A715B689847002840F0358194F8623250
:1085D000022B00F03081D4F868320822A082013BDF
:1085E000E260190E1A0C61F30700190A62F30F20FA
:1085F000B4F8642261F3174052BA63F31F60E28259
:10860000206137E694F80890B9F1000F40F0FF8040
:10861000D4F81822002A00F0898194F91C22002A3B
:10862000C0F21482D3F8C43238469B68984780461B
:10863000002840F0F081D5F8D432384605EB8303AA
:10864000D3F8C432DB6898470146002840F08181A6
:10865000D6F80220D5F8D40212BAB030C4F86C2291
:10866000B6F8073055F820005BBA9BB2C4F87032F8
:1086700000283FF414AE1A44D0F86862B24200F207
:10868000C581B4F8642202FB03F3D4F818229342A4
:1086900040F0EB80B3F5007F4FF0010004F11004CF
:1086A00028BF4FF4007304F8080C1A46D5F8C832F6
:1086B000C3F888229A79C3F88C1203F51E7182429E
:1086C000C3F88442A3F8780262D1C3F894425FE011
:1086D000227A002A40F09B80D4F81812002900F07A
:1086E000828194F91C120029C0F22081D3F8C4328F
:1086F00038469B689847D5F8D432002840F0598115
:1087000005EB83033846D3F8C432DB68984700286A
:1087100040F0F180D6F80230D5F8D4121BBAB0314F
:10872000C4F86C32D6F8062055F8211012BAC4F8F5
:10873000702200293FF4B3AD1344D1F8680283429C
:1087400000F22781B4F8643202FB03F3D4F8182254
:1087500093427FF4DFADB3F5007F4FF0010104F1E8
:10876000100028BF4FF40073217200241A46D5F878
:10877000C832C3F888229A79A3F8781203F51E71DB
:10878000012AC3F88402C3F88C4208BFC3F89402DC
:10879000186873F0BBFD6DE5094A92F85E3063F02E
:1087A0007F0382F85E3083E6054A92F8633063F017
:1087B0007F0382F86330BFE6A4180024A8180024C1
:1087C00048180024022B3CD0012B7FF498AE0023E4
:1087D00084F8623296E6D3F8C43207EBC7013279E7
:1087E000D86900EB810003790533934228BF134613
:1087F000E360002B3FF43EAD03F11002034422443A
:1088000013F8011D834202F8011DF9D132E5394602
:10881000284603B0BDE8F04308E406219A4A04F173
:10882000160304F11000E16012F8011D03F8011DA8
:108830008342F9D11EE53A220221284673F01AFA42
:108840002DE524220521284673F014FA27E520227D
:108850000521284673F00EFA21E528463A22022126
:1088600073F008FA4FF0FF301BE590F861320525F0
:10887000202403F148020133DBB200F8325000EB50
:10888000C202042B948014BF80F8613280F8611218
:1088900005E5D5F8D432B03355F82320002A3FF44B
:1088A000FEAC92F8613202243A2003F14801013310
:1088B000DBB202F8314002EBC101042B888075D095
:1088C00082F86132EBE494F861320520202103F153
:1088D00048020133DBB204F8320004EBC202042B7D
:1088E00091807FF4DAAC84F86182D8E421220521FA
:1088F00073F0C0F9D3E4D5F8D432B03355F823205F
:108900008AB192F861320225272003F14801013330
:10891000DBB202F8315002EBC101042B888008BFA2
:10892000002382F8613205232372B8E494F861329F
:108930000525202003F148010133DBB204F8315052
:1089400004EBC101042B88807FF4A7AC84F861227A
:10895000A5E4D5F8D432B03355F82320002A3FF4EB
:108960009EAC92F86132022427209EE791F8613292
:108970000525202403F148020133DBB201F832500F
:1089800001EBC202042B94807FF4D4AC81F8610225
:1089900085E491F8613205242120BFE43A220221C6
:1089A000284673F067F90523237278E482F8618220
:1089B00075E4B03355F82320002AB4D092F8613220
:1089C00002253A20A1E794F8613203F1480101330E
:1089D000DBB204F8312004EBC1013A22042B8A8077
:1089E0007FF45BAC7FE794F861320525202003F12A
:1089F00048020133DBB204F8325004EBC202042B0C
:108A000090807FF44AAC84F8611248E490F86132B7
:108A1000052521242DE7D5F8D432B03355F823208D
:108A2000002A3FF43CAC92F8613202243A2003F170
:108A300048010133DBB202F8314002EBC101042BE3
:108A400088807FF43DAF82F8619228E494F8613227
:108A50000520202103F148020133DBB204F8320083
:108A600004EBC202042B91807FF417AC84F861926E
:108A700015E43A2273F0FEF8052323720FE491F80F
:108A800061320525212475E79A180024D0F8D432E4
:108A9000B03350F82330CBB110B51A7A022A07D080
:108AA000033A012A02D80021FFF790FA002010BDF6
:108AB00003F21F2293F81D120446FFF72DFB002836
:108AC000F4DA01212046FFF781FAEFE70020704732
:108AD0002DE9F04104464FF41D707BF003FF05467D
:108AE00000285BD0D4F8D47204EB8707C7F8C00223
:108AF000237CC4F8BC02002B45D040230222012174
:108B0000204673F085FA012240234FF001082046E9
:108B1000A4F8782181210222002673F079FAA4F8C2
:108B20003880D7F8C43230462E81A5F8606285F8C7
:108B300062621B689847D4F8C84294F89434276856
:108B4000434508D03846FAF75FFB41463846FAF706
:108B500033FB84F8946405F504751F22002338461E
:108B600004F51E71C4F88C320123C4E9A152A27924
:108B7000A4F878329A4208BFC4F8945273F0C6FB46
:108B80000020BDE8F0814FF400730222012120464D
:108B900073F03EFA01224FF40073B6E7D4F8D432F2
:108BA0000220B03344F82350EBE700BFF8B5D0F80B
:108BB000C85201260446002295F89434A5F878623C
:108BC000B34227D03146286885F89464002773F0B3
:108BD0002DFD40F20113A4F8787132463146286821
:108BE00085F894642B8773F021FD85F89474D4F88C
:108BF000D4320025B033258754F8230040B17BF0F0
:108C000079FED4F8D432B03344F82350C4F8BC52BF
:108C10000020F8BD40F20113A0F878212B87E6E789
:108C200038B5D0F8D432B03350F823507DB195F830
:108C30001C32044623B9D5F818320BB16B7A8BB1CC
:108C40008121204673F0ECFA6B7A022B00D038BDFC
:108C50002046812173F0E4FA20460121BDE8384026
:108C600073F0DEBA012173F0DBFA20468121BDE802
:108C7000384073F0D5BA00BFD0F8D432B03370B5F5
:108C800050F8235025B12B7A044683B1012B01D033
:108C9000002070BD05F21F2295F81D12FFF73CFA67
:108CA0000028F5DA01212046FFF790F9F0E7D5E931
:108CB0008523C5F83832D0F8C832C5F83422D3F845
:108CC0008C321F2B04D12F4BD5F810229A421AD088
:108CD00095F861324FF0050C2021204603F148023F
:108CE0000133DBB205F832C005EBC202042B9180E0
:108CF0004FF0020208BF00236A7285F86132FFF765
:108D00008FFF002070BD95F81D120129E0D895F85D
:108D10001E32013B0F2BDBD805F21F22FFF7FCF9B7
:108D200000282B7A22DB013B022BB1D9EE681EB35F
:108D3000D4F8D432B03354F823100029A8D02046F8
:108D4000D1F83842D1F8183205F11002A41BB34211
:108D5000C1F838424FF0000428BF334681F83C4246
:108D600004240C72812173F0E1FB91E7052B99D06B
:108D70002046FFF755FF8BE731462046FFF726F9DF
:108D800086E700BF55534243F0B5002383B0ADF8EA
:108D90000630D0F8D43200EB8303D3F8C0524DB183
:108DA0000A78044612F0600036D0202805D020460C
:108DB00073F072FA032003B0F0BD4878FE2849D062
:108DC000FF28F4D14B88002BF1D1CE88002EEED1B4
:108DD0001006ECD44FF4807381212B8105F50475C6
:108DE000D4F8C842204674F0C7FC2046012174F034
:108DF000C3FC1F22012304F51E712068C4F88452AD
:108E0000A4F87832C4E9A226A2799A4208BFC4F82D
:108E1000945273F07BFA46E04B780B2BC7D801A233
:108E200052F823F0AB8E04081B8F0408AF8D0408A2
:108E3000AF8D0408AF8D0408AF8D0408AF8D040812
:108E4000AF8D0408AF8D0408AF8D0408E38E0408CD
:108E50009B8E04084E88002EA9D1CF88012FA6D161
:108E60001206A4D5D3F8C4329B6998470223286020
:108E70004FF48071C4F89432D4F8C832C4E906774C
:108E80009A79998203F11401012A5F621D629E6240
:108E900041D0186873F03AFA05E094F89C32032B3D
:108EA00085D18B786B60002085E794F89C32032B8A
:108EB0007FF47DAF0222D4F8C8320020C4F8942297
:108EC00003F11401C4E906220DF106049862C3E916
:108ED00008424FF480729A829A79012AD9D11C6390
:108EE000D7E794F89C32032B7FF461AFD4F8C832F3
:108EF0000122022104350020C4F894124FF480713D
:108F0000C4E90622C3E908529A79998203F114014F
:108F1000012A9862BDD11D63BBE794F89C32032BF4
:108F2000C1D14B88002BBED1D4F8C8628F8896F887
:108F30009434012B0AD001233906306886F8943422
:108F400010D4FAF761F9002386F894346B7A022B77
:108F50000DD03A06A7D5012BA5D001212046FFF759
:108F600035F8A0E707F00F01FAF726F9EBE72046FE
:108F7000812173F055F90121204673F051F992E7F0
:108F80002DE9F8430D46D0E9003113448B4220D837
:108F90000446AE18076BCAB14FF0000900F10C0887
:108FA00001E0AE4212D0E36A5A1C2344E262202A56
:108FB00015F8011B1973F4D14146204617B9FAF789
:108FC0006FF90746AE42C4E90B97ECD13846BDE8CD
:108FD000F8834FF0FF37F9E702784368022A0FD091
:108FE0000B490269D1F81C02023A184010B4400A39
:108FF000D1E9841404FB02005DF8044B0844704777
:10900000034AD2E9812102EB410202EB532070476F
:10901000A05C00242DE9F04F83B002F002077D4DE3
:10902000019308B9002F65D1D5F80C42002C4FD11F
:109030004FF0FF3E774C4FF0000CF146F046F24601
:10904000E36994F82A60984200F09580C6B3012E37
:1090500005EB0C1B0AD19BF82B60F30706D416F026
:109060007E0F03D1F60900F08980E0460CF1010C77
:109070001034BCF1080FE3D1BEF1000F04DAB8F1EF
:10908000000FC0F28D80C646D5F89C4005EB0E1C43
:109090000EF102060134CCE9070405EB061CC5F805
:1090A0009C40CCF804400024CCF8084005EB0614A2
:1090B000A47A042C1ED8DFE804F0274119414300AC
:1090C000E6460CF1010C1034BCF1080FB8D1D3E71F
:1090D000D5E9843606FB0434A042A9D395F8B8310B
:1090E00013B9012385F8B83101236B70002003B058
:1090F000BDE8F08F95F8B831002B4DD00123022048
:109100006B7003B0BDE8F08F12F00104D5F818C001
:109110006CD105EB0610019B4FEAE20C90F80B8036
:10912000032B6CF3C71880F80B805DD94FF6FF70E6
:10913000834228BF034605EB06100381002F41D16F
:10914000500705D505EB0610C37A43F00103C3723F
:10915000D30608D505EB0616F37AC3F345020132B0
:1091600062F34603F372AB69012003EB4E230B60FD
:1091700003B0BDE8F08FC6B9E64685E7666A1034ED
:10918000B24588BFE1460CF1010C88BFB246BCF184
:10919000080F7FF455AF6FE7012385F8B831ADE7CD
:1091A000B9F1000FA2DBCE466EE7D5F89C400CF17A
:1091B0000206E646013405EB061CC5F89C40CCF8D7
:1091C000044073E7D5F8A000D5F89C300130013396
:1091D000C5F8A00005EB0E10C5F89C30036205EB46
:1091E000061304209872ABE72346A4E7D5F828328B
:1091F000002B3FF47BAF5C680CEB4E210023064A4A
:10920000A04700283FF472AF05EB06160223B372A5
:109210006CE700BFA05C0024ED77040870B5104D2A
:1092200082B00E462B78022B15D1020AC4B2D5F8B3
:109230000402002301A910440322FFF7EBFE0128DA
:1092400007D12B78019A022B0CBF22F8146042F848
:10925000246002B070BDC0F3D41200F07F04E6E7D2
:10926000A05C00242DE9F04F434E0D4683B0174615
:1092700031782B6803293DD002295FD14FEA1329A9
:109280004FF4807A5FFA83F8421E012A23D84FF008
:10929000010B9F421AD901288CBF00240124D6F863
:1092A0007C211AB1D6F8981199424AD0D6F8040216
:1092B0000023092201A94844FFF7ACFE012822D06F
:1092C000022813D020B12B689F42E8D803202F60DA
:1092D00003B0BDE8F08FB8F1000F12D096F8B831A6
:1092E00013B9012386F8B83101237370022003B04B
:1092F000BDE8F08F4FF0800AC3F3D41903F07F0864
:10930000C2E7D346C5E73178022913D00329EDD14E
:10931000019B53F8282022F07042B2FA82F22B68A7
:109320005209A2421FD0D8445B44D0452B601DD2C5
:109330000229EDD1019B33F81820EEE74FF4807A33
:10934000DAE7D6F81412013A02EB41224902B2FBE5
:10935000F1F21344B3FBFBF20BFB12320AB15B4494
:109360009B1A2B60B0E79F42B2D8AFE709F1010921
:109370004FF00008A8E700BFA05C00242DE9F04FE3
:10938000DFF884918B4685B0174699F800C00968CC
:10939000BCF1020FD9F8045240F08280CEB24FF4F3
:1093A000807305EB1125A6EB010890449844B9425F
:1093B00008F1FF38B8FBF3F84AD200F00103A844E3
:1093C0006FF0404A0193BCF1030F07EB0604A8EBD2
:1093D0000503284614BF4FF480728022641A03A943
:1093E000944228BF1446944228BF002E14BF012285
:1093F00000220A32FFF70EFE01282AD199F800C098
:10940000DBF800E0BCF1020F0EF1010324D0B442FE
:1094100055D9039806EB0A02011F00EB820201EB0B
:10942000840142F8043F8A4203F10103F9D1DBF8D9
:109430000030A11B19448F42CBF8001002D1019BD0
:10944000002B48D18F4205F101054FF00006BAD834
:10945000012005B0BDE8F08FB44246D903986FF003
:109460000042811E324401EB440100EB420222F82B
:10947000023F914203F10103F9D1A11B71448F42D4
:10948000CBF80010DED1019B002BDBD086466FF0BD
:1094900000434FF6FF72012023442EF81320D8E733
:1094A00001F07F06C1F3D413BCF1030FA6EB010852
:1094B0001D4414BF4FF480738023904476E7AEEBD5
:1094C000060E0EEB04018F42CBF80010BAD1019BBF
:1094D000002BB7D003986FF040434FF0FF32234486
:1094E00040F82320DBF80010ACE7AEEB060E0EEBE5
:1094F00004018F42CBF80010A4D1019B002BA1D016
:10950000DDF80CE0C3E700BFA05C002430B50446E2
:10951000C06983B010B9012003B030BD0D460023EF
:10952000032201A9FFF776FD0128F5D1B4F9202027
:10953000002A19DB019B012D4FEA421103EB421275
:1095400003D0022D1AD1E5205854A368D3612378A3
:10955000032B04D10023137753779377D377636A70
:10956000190C53839182D6E7054A92F8B81109B9CC
:1095700082F8B801012302205370CDE7E368E5E7E4
:10958000A05C00242DE9F041044682B00D4694F819
:109590003C30042B7DD8DFE803F02A03684839000B
:1095A0003D4E4FF6F777DFF8F48016E0BA425AD80E
:1095B0006AF0EAF901284FF0000133D1206BFFF780
:1095C0002DFE01282ED1019AD6F81812531E2263BF
:1095D0008B4228BF0B46C6F81832327801A9236B9C
:1095E000032A18469AB2E1D14345E1D93BE069002C
:1095F000204601F0FE01FFF789FF01283FD1636B90
:10960000002B18BF022084F83C00C0E794F82830F3
:10961000042B02D1002384F82830A36B0BB1204621
:109620009847012002B0BDE8F0811B4E0021E26A9C
:10963000D6F8983106F5BA70C6F898219B1AD6F874
:10964000142202FB03F3D6F87C2102EB4322C6F876
:109650007C21D6F8802102EB4322C6F88021FFF757
:1096600055FF01280BD10420CDE7626B04F13001D6
:109670000020FFF783FE012801D10320C3E7022861
:10968000D0D194F82830042BCCD1002384F8283092
:10969000C8E70220F5E700BFA05C0024F7FFFF0F3A
:1096A00038B5044694F83430052B60D8DFE803F071
:1096B00031251D130D0394F82830082B3FD02D4B76
:1096C0000122022083F8B92138BD94F82830082BF4
:1096D00030D0012038BD00212046FFF717FF0128B8
:1096E00045D1042084F83400DCE7D4E90B01FFF70E
:1096F00095FD01283BD10320F4E74FF0FF31206BAB
:10970000FFF78CFD012832D1E36A002BF3D0022051
:10971000E8E7184D04F130010120D5F80C2202329F
:10972000FFF7A0FD012813D00238C0B201281ED8CF
:109730000520D7E70023012084F82830CAE700235A
:109740000122022084F828300A4B83F8B921BBE7B4
:10975000E368D5F81412226B03EB4123C5F81822F5
:10976000C4E90332E36A002BBCD16262BAE700208D
:1097700038BD00BFA05C0024F8B5044694F838302A
:10978000032B4BD8DFE803F021180B020021204601
:10979000FFF7BCFE431EDBB2012B40D9F8BD012010
:1097A000626B04F13001FFF7E9FD01284FF003037C
:1097B000F0D184F83830E1E700211E48FFF7A6FE1B
:1097C00001284FF00203F4D0E4E71B4BE6681A7857
:1097D000D3F81412032AD3F87C51D3F8980114BF9C
:1097E0004FF480728022206102FB01F1871A02444B
:1097F000A5EB412506EB4126E660C3F87C51D3F882
:109800008051C3F89821A5EB4121C3F88011E36A88
:10981000C4E90C025BB960620123CAE7022094F834
:109820002830062BBAD1002384F82830F8BD2763EE
:10983000F2E700BF145E0024A05C00244368C3F379
:1098400008020A44B2F5007F2DE9F041054682B0D6
:109850000C4605D223446B60012002B0BDE8F081C4
:1098600090F91A20501C09D04449023201EB02122F
:10987000D17A21F00101D172FF22AA7695F91B203D
:10988000511C13D03D4E023206EB0211C97AC1F3CE
:109890004501012941D9013901F03F0106EB0212CE
:1098A000FF26D07A61F34600D072EE762A78022A3B
:1098B000D0D0324ED6F81422B4EB422F4FEA4228D1
:1098C0002DDCD6F81C721F407A42A24227DCE21936
:1098D0002869424513D32A7E12072BD5D6F8982142
:1098E000411C8A421DD300D100214344A4EB080847
:1098F00068610846DB1B08EB070429616B600028E0
:10990000AAD03278032A33D080B24FF6F772904251
:10991000A2D81A4614446C609EE70021BEE70020DE
:109920009BE796F8B82102BB012386F8B831737023
:109930006B68DAE701A96AF027F80128EFD16B68B4
:10994000A4EB080428699844297868613C44A8EB92
:109950000703019802291A466B602861CFD1D6F817
:109960002412B3EB412FD5D376E701227270BCE706
:10997000034A90423FF670AFCBE700BFA05C0024E3
:10998000F7FFFF0F2DE9F0474FF0010882B00446C2
:1099900094F83830032B00F2A580DFE803F0551768
:1099A0000C020020236C84F8280003B198470220A1
:1099B00002B0BDE8F0870022236C84F828200BB1A8
:1099C00020469847012002B0BDE8F08723786768F9
:1099D000022B03D0444BD3F81C321F40C7F34F2750
:1099E0002046FFF7F9FA404E3F1A0546BFB207EB93
:1099F000050C022201A9002328461FFA8CF9FFF763
:109A000009FB01284FF400724FF00001D0D10198FA
:109A10007AF05EFEE3694FF4007120460BB1636893
:109A2000EBB1D6F814325A1E914547D20135FFF7F3
:109A300005FF0028DBD196F8B83113B9012386F869
:109A4000B83186F80180D2E72046FFF729FE0128C9
:109A500002D0022846D1032084F8380098E7019B01
:109A60004FF020324FF0100E4FF02E0C42F62E6ABF
:109A7000C3F80120C3F80520A3F8092083F800C02B
:109A8000D4F824C0A3F820A083F80BE0C3F8222068
:109A9000C3F8262083F82A20E26BA3F81AC02CFA18
:109AA0000EFC5A8722FA0EF2A3F814C09A8683F8A5
:109AB0002BE0D6F814325A1E9145B7D3C3EBC353EB
:109AC0002046590201F50071FFF7B8FE20B996F85B
:109AD000B8311BB1012373700220BDE7012386F862
:109AE000B831F7E7002063E7A05C0024B1F9043047
:109AF0000F2B2DE9F0410D4682B00446164631D0B9
:109B00002046FFF769FA94F91B80B8F1FF3F3AD07D
:109B1000584F07EB0813DB69984211D097F8B8311A
:109B2000002B6BD001237B702378022B5CD0226941
:109B3000002A71D100230120336002B0BDE8F0811A
:109B4000B96901EB4821002964D0AB882046013374
:109B50001BB201EB4311AB803160FFF73DFA286087
:109B60000120EAE74FF40071FFF768FE002841D0BA
:109B70004FF6FF732046AB80FFF72EFA94F91B8057
:109B8000B8F1FF3FC4D12378022B3BD02269002AD1
:109B9000D0D0384F3B78032B62D093B24FF6F77199
:109BA0008B4294BF00230123002BC1D128B997F821
:109BB000B831002B47D001237B700023112201A96B
:109BC000FFF728FA012825D10199BB69CB1A48BFB4
:109BD00003F2FF13B3F5805F4FEA63222AD24FFAF4
:109BE00082F884F81B80AEE7D7F824226368B3EBD1
:109BF000422F9FD2002002B0BDE8F081012387F8F8
:109C0000B8318FE71B4F6368D7F82422B3EB422F9C
:109C1000CCD38FE7237888E73B78032B17D093B218
:109C20004FF6F772934294BF00230123002B81D19A
:109C30000020E0E797F8B83113B9012387F8B8316D
:109C400001237B70CDE7012387F8B831B3E70A4BD6
:109C50009A4294BF00230123002B7FF46BAFE7E708
:109C6000054B9A4294BF00230123002B7FF460AF81
:109C70009CE700BFA05C0024F7FFFF0F70B50378DE
:109C8000044690F818C0023B012B02D91CF0060FC5
:109C900066D11CF0200F3FD194F91A30591C09D01D
:109CA000364A0233FF2102EB0313DA7A22F0010273
:109CB000DA72A17694F91B305A1C13D02F48023364
:109CC00000EB0312D27AC2F34502012A45D9013AC8
:109CD00002F03F0200EB0313D97A62F34601FF2240
:109CE000D972E2761CF0080F0DD0244890F89C3110
:109CF000072B05D090F8B831002B39D001234370E1
:109D0000002380F89C310023E26A237084F8283015
:109D10002AB3BDE87040104718480023E5690246A1
:109D2000D16910328D4206D00133082BB4D0D169ED
:109D300010328D42F8D1023300EB0312D27AC2F313
:109D40004502012A18D9013A02F03F0200EB031341
:109D5000D97A62F34601D9729EE70022BAE770BD54
:109D60000121FFF7D3FB0128F9D194F818C090E73F
:109D7000012380F8B831C1E70022E7E7A05C0024A6
:109D800038B5194C94F8E4312BB970B190F828200B
:109D90001AB1184638BD002038BD0146442204F5EA
:109DA000DE7079F06DF8012038BD04F5DE750146EE
:109DB000442228467AF08CFC237803224FF6FF7168
:109DC000022B2846A4F8D61118BF1346D4F8201247
:109DD00084F8D421102284F8BC31C4F8E01184F84E
:109DE000D5216AF075FEDEE7A05C0024F8B54FF0DF
:109DF000FF312C4C002322460D4603E00133103284
:109E0000082B14D092F82A000428F7D104EB031091
:109E100090F82B00C707F1D46E1C106A01D0814264
:109E2000ECD91D46013301461032082BEAD1002D32
:109E300001DA0120F8BDAE1CD4F8282204EB061389
:109E40001989D1B92F012744A169D4F82832F869BA
:109E500001EB4521CBB1DD680023134AA847A0B12F
:109E6000022808D1D4F8A03004EB06160122013BE9
:109E7000B272C4F8A0300020F8BD04EB05132F0126
:109E8000D86912B193689847DDE7D4F8A03004EBA5
:109E9000061603210122013BB17284F8A420C4F804
:109EA000A030E8E7A05C002449780408704700BFB0
:109EB00010B54FEA511E024400EB8E0C624529D9C1
:109EC00001F01F034FF0FF3450F82E1004FA03F393
:109ED0000B4093FAA3F3B3FA83F3DBB2202B16D132
:109EE0000CF104018A4202D817E08A4212D98C464A
:109EF0000431DCF8003093FAA3F3B3FA83F3DBB256
:109F0000202BF2D0ACEB000C03EBCC0010BD03EB2C
:109F10004E1010BD4FF0FF3010BD204610BD00BFE9
:109F20000369416853EA0102F0B43B4E5DD0C56A53
:109F3000013390ED067A6A1C876830EE077A036178
:109F4000012AC26280ED067A42D090ED075A07EEF0
:109F5000902AD0ED096A70EE455A3468B8EEE76A87
:109F6000611AC5EE867AB94277EE857A30EE670AD5
:109F7000C0ED087AC0ED077AF0EE667AE5EE807AF9
:109F8000C0ED0A7AC0ED097A01D8F0BC7047012A09
:109F900028DD06EE905AF8EEE66A87EEA66AB5EE80
:109FA000C06AF1EE10FA1DDBF1EEC67AF4EE677AC4
:109FB000F1EE10FA16D6D0ED056AF4EEE76AF1EE8E
:109FC00010FA15D5037BFBB10323F0BC0370704777
:109FD000326880ED080A521A002180ED070ABA4261
:109FE0004162D2D9DFED0D7AE5E7316841609EE745
:109FF00007EE903A0223F8EE677A0370F0BCC7EEE2
:10A00000276AC0ED066A7047316800220361C362A7
:10A0100041608261B9E700BFD03000240000000039
:10A0200010B5DFED4F4A844600F1480E0346DA6A68
:10A03000B1EC017AD3ED067A013277EE877A012A04
:10A04000DA62C3ED067A71D093ED075A07EE902AD3
:10A0500093ED096A77EE455AF8EEE77AC5EEA76AFE
:10A0600076EE857AF0EE466A37EE677AC3ED087AC7
:10A07000E5EE876AC3ED0A6AC3ED077A1833C3EDCC
:10A08000036A7345D3D1374C416822680369521A79
:10A09000816801338A42036147D990ED056A002245
:10A0A000DFED2F5ADCF82C10F0EE657ADCED0A6A51
:10A0B000012901F1FF3E11DD07EE90EAF8EEE77AA3
:10A0C00086EEA77AB5EEC07AF1EE10FA45DBF1EE36
:10A0D000C77AF4EE677AF1EE10FA3ED6B4EEE76A8C
:10A0E00001320CF1180CF1EE10FA26D4022AD9DD57
:10A0F000B4EEE76AF1EE10FA1FD407EE903AD0ED15
:10A10000066A90ED0C7A0223F8EE677AD0ED125AC7
:10A11000037086EEA76AC7EE276A85EEA77A80ED00
:10A12000066AC0ED0C6A80ED127A10BDF0EE477A37
:10A1300083ED087AF0EE646A9EE7037B13B1032394
:10A14000037010BD002221680361C3624160826117
:10A15000026343648264C36510BDDFED017ABDE72D
:10A1600000000000D0300024B0EEC06AF0EEE05AEB
:10A17000F0EE407AF4EEC65AF1EE10FA0EDCB5EECF
:10A18000400AF1EE10FA4AD0F4EEC65AF0EE466AF2
:10A19000F1EE10FA4FD5B0EE655A03E0F0EE656AC5
:10A1A000B0EE465A85EE267A9FED242A9FED243A9A
:10A1B0009FED244ADFED244ADFED242ADFED243A27
:10A1C000B7EE005ADFED236AF4EEC65AF1EE10FA4C
:10A1D000A7EE023AE7EE223AA7EE034AA7EE235A89
:10A1E000E7EE044AE7EE246AB1EE667A87EE050AE6
:10A1F00010D4F5EEC00AF1EE10FA03D59FED167AF1
:10A2000037EE400AF5EEC07AF1EE10FA48BFB1EE33
:10A21000400A70479FED117A37EE400AE9E7F5EE04
:10A22000C00ADFED0F7A9FED0F0AF1EE10FA58BF6A
:10A23000B0EE670A7047B0EE465AB3E739094E3DB3
:10A24000E3B59EBE88FA16BE45FE7FBF99FB243F4C
:10A2500069A2163EA7DFA8B4DB0F4940DB0FC93F58
:10A26000A7DFA834DA0F4940D1ED007AF7EE002AD3
:10A27000D0ED043A90ED054AE7EEA73AD0ED064A54
:10A2800090ED075AD0ED085A90ED096AD0ED0A6AB0
:10A2900090ED0B7AC0ED043A91ED003AD1ED013A20
:10A2A000D0ED0C7AA3EE234A80ED054AD1ED003AB9
:10A2B00091ED024AE3EE844AC0ED064AD1ED004A30
:10A2C00035EE245A80ED075AD1ED014A91ED005A3E
:10A2D000E4EE855AC0ED085AD1ED015AA5EEA56A03
:10A2E00080ED096AD1ED015A91ED026AE5EE866AC8
:10A2F000C0ED0A6AD1ED016A37EE267A80ED0B7A5D
:10A30000D1ED026A91ED007AE6EE877AC0ED0C7A23
:10A3100091ED027AD1ED017A90ED0D3AD0ED0E3A41
:10A32000A7EE273A90ED0F4AD0ED104A90ED115A62
:10A33000D0ED127AD0ED135A90ED006A80ED0D3A0F
:10A3400075EEA25A91ED023AD0ED016AE3EE033ABE
:10A3500090ED027AC0ED0E3AD1ED023A34EE234A86
:10A3600080ED0F4A91ED004A74EE844AC0ED104A28
:10A37000D1ED014A35EE245A80ED115A91ED025A81
:10A38000C0ED135A77EE857AC0ED127AD1ED017ADD
:10A39000D1ED005A67EEA77A91ED025AE5EEA57A63
:10A3A000E5EE057AA5EEA76A80ED006A91ED016AF7
:10A3B000E6EE276AC0ED016AD1ED026AA6EEA77A41
:10A3C00080ED027A90ED037A77EE277AC0ED037A7A
:10A3D000704700BF2DE9F04F4FF00009864600F1AD
:10A3E00010050646034689B000F130080746484686
:10A3F0002C468B469C46B246CDF80CE000283CD15A
:10A400000CF1040CA445FBD1032800F1010151D04B
:10A410009C46AA46029398B1DCED047AAAEB0903A4
:10A42000B64601927246F3EC016A0EF1100E92EDFF
:10A43000007A5345E6EEC77ACCED047AF2D1019A60
:10A44000DCED046A0CF1100C15ED047A0AF1100A27
:10A45000C445C6EE877ACCED007ADCD1029B043687
:10A46000084608F10408143314351034103709F184
:10A4700004099C46B2460028C2D0DCED007AD646DC
:10A48000394601927246F1EC016A0EF1100E92ED1E
:10A49000007A9942E6EEC77ACCED007AF2D10CF15F
:10A4A000040C019A0AF1040AA445E6D1032800F13C
:10A4B0000101ADD1DDF80CE00023594604AD76462C
:10A4C000774600200493059306930793F2EC017AF4
:10A4D000E5EC017AB0B104AC3B46B4EC017AF3ECA4
:10A4E000016AE6EEC77AB34245ED017AF5D1013053
:10A4F00004280BD0F2EC017A10371436E5EC017A1F
:10A500000028E8D1103714360120DFE708AD1031FC
:10A510000EF1400E042875ED017AA1F10402744693
:10A5200041ED017A1ED07346F3EC016AB1EC017A79
:10A53000A342E6EEC77AC2ED007AF5D15EED016A7C
:10A54000013887EEA67A82ED007A17D0AEF1140EAC
:10A55000103C114675ED017A0428A1F1040241ED89
:10A56000017AE0D15EED016A103CAEF1140E0320D9
:10A5700087EEA67A01ED017A1146EBE709B0BDE856
:10A58000F08F00BF60EEA00AE0EE000AF5EEC00A10
:10A59000F1EE10FA07DBB1EEE00AB4EE400AF1EE9C
:10A5A00010FA00D670479FED010AFBE7000000009B
:10A5B00060EEA00AE0EE000AE1EE010AF5EEC00A44
:10A5C000F1EE10FA07DBB1EEE00AB4EE400AF1EE6C
:10A5D00010FA00D670479FED010AFBE7000000006B
:10A5E000DFED297AB4EEE70AF1EE10FA28DD9FEDEF
:10A5F000277A30EE470AB4EEE70AF1EE10FAF8DCFB
:10A60000DFED237AB4EEE70AF1EE10FA2FDD30EE3B
:10A61000670A37EEC00A60EE007ADFED1E5A9FED42
:10A620001E6ADFED1E6AA7EEA56A9FED1D7A60EE39
:10A63000275AE7EE866AA7EEA67AA5EE870A704744
:10A64000DFED187AB4EEE70AF1EE10FAD8D59FEDF7
:10A650000F7A30EE070AB4EEE70AF1EE10FAF8D4FA
:10A66000DFED0B7AB4EEE70AF1EE10FACFDC9FEDE6
:10A670000E7AB4EEC70AF1EE10FACCD530EE270A06
:10A6800037EE400AC7E700BFDB0F4940DB0FC94088
:10A69000DB0FC93F9A7C2E36FAAF4FB93587083C9D
:10A6A000A4AA2ABEDB0F49C0DB0FC9BF10B5404CBE
:10A6B000B4FBF2F4A14219D3DFED3E7AF7EE005A73
:10A6C000B0EE677AB0EE676AF0EE676A0023C0ED1D
:10A6D000005AC0ED017A80ED027A80ED036AC0ED88
:10A6E000046A836143610362C36110BD07EE902A6F
:10A6F000DFED315AB7EE006ADFED306AB8EE677A07
:10A7000007EE901AB0EE405AF8EE677A27EE257AF7
:10A7100067EEA67AC6EE076AC7EEA64AFDEEE47AB1
:10A7200017EE902A2032402A3FD8B0EE640AFFF795
:10A7300057FFB0EE404ADFED227A34EEA70AFDEE75
:10A74000C07A17EE902A2032402A29D8FFF748FF16
:10A75000F8EE006A60EE266A012B1CD0B7EE006AA4
:10A76000F6EE004A36EE406A66EE244A35EE055AA9
:10A77000F7EE007A84EE057A77EE275A37EEC75A5D
:10A7800084EEA57AC6EE257A86EEA56AC5EE256A20
:10A79000F0EE475A9AE7F7EE004AB0EE666AE5E750
:10A7A000DFED086A9FED030AD6E79FED024AC2E794
:10A7B00020A1070000000000BD378635DB0FC9402F
:10A7C000DB0FC93F00000080DFED077A30EE270A7B
:10A7D000FDEEC07A17EE903A2033402B00D8FFE60A
:10A7E0009FED020A704700BFDB0FC93F0000000069
:10A7F0002DE9F84F9DF828408946DDF82CB0054634
:10A80000002C17461BF8011B0CBF4FF020084FF01F
:10A8100030081C1E08463ADB00295CD0002C53D0BF
:10A820004FF0000A5B4600E064B313F8016B013C93
:10A83000002EF9D1BAF1000F2FD1264644B14D4573
:10A840004146284600D2B847013CF8D10B9B187806
:10A850000146A0B14FF0FF344FF0000A00E09B46E4
:10A860004D45284600D2B8475B4613F8011B002926
:10A87000F5D10B9BF61A5E44BAF1000F10D13046A9
:10A88000BDE8F88FBAF1000F1BD15646E0E76342EE
:10A8900029B31C464FF0010AC4E70028E0D1064660
:10A8A000002C04F1FF3AEADD54464D454146284666
:10A8B00000D2B847013CF8D2013656443046BDE8D4
:10A8C000F88F30B12646CBE726464FF0FF34B2462C
:10A8D000C6E70646D3E72646002CB0D1CFE76FEA9D
:10A8E000040A0E46E0E700BF0FB430B583B00C4C4D
:10A8F00006ABD4F8E015D4F8DC0553F8042B01932B
:10A900006CF02EFA0546D4F82C0203685B69984770
:10A910000028F8D0284603B0BDE8304004B07047A6
:10A92000A05C00240EB410B583B00446084905AB02
:10A9300001A853F8042BCDE900346CF011FA002281
:10A94000019B1A7003B0BDE8104003B0704700BF10
:10A950000D7C04080CB4F0B53C4CADF5277DD4F863
:10A96000E435002B6DD094F8EC3599420BD90123D6
:10A97000D4F8F0258340134205D10DF5277DBDE8BD
:10A98000F04002B07047324B4FF47A71314A1B6885
:10A99000A2FB030206A8920901FB12332E49FFF71E
:10A9A000C1FF06ABAC9A064603442C4901A80193AB
:10A9B000ADAB00936CF0D4F9019B0A2100225D1C21
:10A9C00001951970019BD4F8E455591C01911A7036
:10A9D000ADB12B685B6A1BB128469847D4F8E455A3
:10A9E0009DF818100029C8D00DF119042B682846CD
:10A9F0001B68984714F8011B0029F7D1BDE7D4F86C
:10AA0000E875002FB9D0304426ABFD2206A9841C7E
:10AA10001846ADF810202246CDF81250ADF8165069
:10AA200078F02EFA02220346044402A93846CDE902
:10AA3000023434F02BFC0DF5277DBDE8F04002B068
:10AA40007047D4F8E835002B8DD196E7A05C002440
:10AA5000D0300024D34D6210E8550D08017C040865
:10AA600038B5184C0330D4F8F42502EB9003B3F555
:10AA7000007F18D804EB810104F5BF6520F00300C6
:10AA8000C4F8F43505EB8205D1F8F82DC3F5007351
:10AA900010440D4A9B00C1F8F80D04210020FFF777
:10AAA00059FF284638BD0021084A00250846FFF70F
:10AAB00051FFD4F8803E284643F00073C4F8803E2E
:10AAC00038BD00BFA05C0024F4550D0818560D08D1
:10AAD00003685A1C02601878704700BF03681A4662
:10AAE000591C016012F8021B0260587841EA0020EC
:10AAF000704700BF02681346511C016013F802CB77
:10AB00000360D31C5178036093781B0443EA01234C
:10AB1000111D43EA0C030160D07843EA00607047DE
:10AB200012B370B50446864604E0981B17D114EBA7
:10AB30000C0C15D01EF8013BA3F14100A2EB0E0C4A
:10AB4000192811F8010BA0F1410598BF203300F13D
:10AB50002006192DE9D91B1A04D10028E7D170BDB0
:10AB6000604670BD184670BD1046704703880021CE
:10AB7000184AA3F5FA6C70B503F0030490F802E0EC
:10AB8000154E40F2B5550EF1FF3E04EB44044FEA7A
:10AB90009C0C0EEB8403C47836F81330013C05FBA3
:10ABA0000C3390F804C02344847903EB430322441C
:10ABB0004FF47A740CEBC30C43790089CCEB0C1C7A
:10ABC00003EB8C03C3EB031302EB8302C2FB040110
:10ABD00070BD00BF80436D3888A20C082DE9F0419C
:10ABE00016461F46404D0446394630464FF47A72A9
:10ABF00000237CF05DFD3D4B05443D4F3D4E83FB06
:10AC00000510E9172844C1EB601183FB0103C81745
:10AC10000B44C0EB631087FB003CC317C3EBAC03D2
:10AC200086FB03764FEAE37ECEEBE61EC1EB011610
:10AC3000A5EB860CC0EB00154FEA8E0684F806C023
:10AC4000A1EB8501617103EB4301A0EBC10040F270
:10AC5000B55101FB1E332071B3F5896F33DA40F231
:10AC6000DA218B4237DCB3F5B77F234FB4BF4FF007
:10AC7000000E4FF0010E0EEB4E0175464FEA4E08E6
:10AC800007EBC101C88A08EB0E0C0B2107EBCC0CBB
:10AC90000CF1160C01E03CF8020D984210DD013970
:10ACA000F9D1F044012137F8380006F5FA6E013386
:10ACB000A17075441B1A22812580E370BDE8F081E4
:10ACC0000131C9B2F1E7032540F296500A4F4FF027
:10ACD0000608AE46D7E7022540F22940064F4FF05E
:10ACE0000408AE46CFE700BF80BC92C78988888839
:10ACF000ABAAAA2A73B06D1688A20C0830B5304CE6
:10AD00008DB086460D46EC461EF0030F0FCCACE826
:10AD10000F000FCCACE80F0094E80F008CE80F0098
:10AD20000FD1284B284A03FB0EF3B2EBB30F44D3E9
:10AD3000264AB2EB331F34BF01220022C2F11D02AA
:10AD400000E01C220EF1FF33019240F26D12204808
:10AD5000002B194602FB0EF21E4CB8BF0EF1020189
:10AD6000EE4602EBA10280FB0310DB17ADF10401FC
:10AD700001EB8501A3EB6015C3EBE0132A441A44F1
:10AD8000253284FB0230D3171044C3EBA003C3EB7E
:10AD9000C303D31A5EF8040FC218714584FB023C4A
:10ADA0004FEAE2739444C3EBAC03C3EBC303A2EBDF
:10ADB0000303EFD1C01A0DB030BD1D22C2E700BFA2
:10ADC000E8A20C08295C8FC2285C8F020AD7A30076
:10ADD0001F85EB51932449920D4B10B553E9024363
:10ADE00054EA03020AD10146002340F20112184638
:10ADF0000B80C1F802208B710B8110BD054A1268CF
:10AE0000121943F10003FFF7E9FE012010BD00BF56
:10AE1000306B0024D030002430B5144D83B004468C
:10AE2000D5F8881ED5F88C3E51EA03020AD10023DA
:10AE300040F2011218462380C4F80220A371238136
:10AE400003B030BD0A4A1268521843F10003FFF7FD
:10AE5000C5FEB5F8903E20460DF106022146ADF83C
:10AE6000063068F0F1FC012003B030BDA05C002486
:10AE7000D03000242DE9F047044688B094F83030F3
:10AE8000042B11D8DFE803F04C135D035600237E3A
:10AE90009A0640F1F0800023112204A9E069FEF730
:10AEA000B9F8012800F0E78008B0BDE8F087C94D87
:10AEB00003AE04F11C0705F5DE79324639464846F3
:10AEC000FEF714FE012800F0F1800228ECD195F97C
:10AED000D6315F1C09D00233FF2205EB031385F83E
:10AEE000D621DA7A22F00102DA7295F9D7315E1CA6
:10AEF00014D0023305EB0312D27AC2F34502012AC1
:10AF000040F25081013A02F03F0205EB0313D97A77
:10AF100062F34601FF22D97285F8D721042306E0A7
:10AF2000AD4869F0D5FD4FF6FF720123228484F805
:10AF30003030A3E70020E36A207008B0BDE8F04796
:10AF40001847A44D95F8E431002BADD104F11C074E
:10AF500003AE05F5DE78324639464046FEF7C6FDBB
:10AF6000012840F00D81039B002B00F0E8801A7847
:10AF70000AB1E52AEFD1AA699A1A48BF02F2FF1274
:10AF8000B2F5805F4FEA622180F041810901934A66
:10AF90000A44917B04290CD0D5F89C100131C5F8E6
:10AFA0009C10516004219173D5F8A0200132C5F89E
:10AFB000A02095F9D621501C09D0023205EB0212CF
:10AFC000D17A21F00101D172FF2285F8D62195F9BD
:10AFD000D721511C14D0023205EB0211C97AC1F3FA
:10AFE0004501012940F25681013901F03F0105EB8D
:10AFF0000212FF2085F8D701D07A61F34600D072A3
:10B0000020220021184679F063FBD4F83110034662
:10B01000D4F8352005A819605A6094F83B20B4F89C
:10B0200039109A721981627E0193DA72FFF7F4FE89
:10B03000019B002800F0D4809DF816009DF8172091
:10B040009DF8191042EA4012BDF814004901A0F21F
:10B05000BC7042EA40229DF81A0041EA50019DF876
:10B06000180092B241EAC02188B2D9811A821A83AB
:10B07000D88203235BE7204669F02AFD2369002B71
:10B0800000F08380237E03F0F70213F0040322769E
:10B0900040F08A80122A00F0A6800022E36A20464F
:10B0A00084F8282008B0BDE8F0471847DDF80C8088
:10B0B000B8F1000F00F0B68098F80030002B00F0D7
:10B0C000B18098F80BA01AF0080F7FF4F6AE0B22AF
:10B0D00004F13101404678F013FA00287FF4EDAE18
:10B0E000637E8AEA0303DF0640F1D88095F9D63102
:10B0F0005E1C09D00233FF2105EB031385F8D6113E
:10B10000DA7A60F30002DA7295F9D721511C3FF424
:10B1100005AF023205EB0213DB7AC3F34503012BC3
:10B1200040F2FB80013B03F03F0305EB0212D17AB2
:10B1300063F34601FF23D17285F8D731EEE695F827
:10B14000BC310922022B3FF4E9AE95F8E431002B23
:10B150007FF4E4AE85F8F43185F8F0311E4885F8C7
:10B16000E421C5E97E33D5F8D031C5F8E831D5F80A
:10B170001832C5F8EC31FEF705FC01283FF4EBAEC0
:10B1800002287FF491AE0423D1E6237E1B0784D5E9
:10B19000104B93F89C21002A7FF486AE072283F897
:10B1A0009C217AE70022B0E60023A5682046E66AE3
:10B1B000294684F82830FEF741FB002864D194F832
:10B1C0002830002B7FF470AE0223C4E90B6584F8AD
:10B1D000283069E6A05C00245C5E0024BC5C00248E
:10B1E00044F2817242E7E06A0421626AA063204669
:10B1F00084F83C3084F8281063636362C4E90B224E
:10B20000C4E9023308B0BDE8F04769F061BC95F8C5
:10B21000B82112B9012285F8B82101226FF00F017F
:10B220006A70B4E695F9D631591C09D00233FF2271
:10B2300005EB031385F8D621DA7A22F00102DA72DF
:10B2400095F9D7315A1C13D0023305EB0312D27A89
:10B25000C2F34502012A1FD9013A02F03F0205EB71
:10B260000313D97A62F34601FF22D97285F8D721F8
:10B27000237EDB067FF552AE2A4869F029FC4FF6A3
:10B28000FF720223228452E6002E3FF40DAE2046C8
:10B29000334652E60021AAE60022E0E7B8F814207F
:10B2A000B8F81A3043EA0243D5F814226362520216
:10B2B000D8F81C30B3FBF2F102FB1131A36009B1E5
:10B2C00013445B1AE36084F819A095F9D6315A1C2F
:10B2D00009D00233FF2205EB031385F8D621DA7A71
:10B2E00022F00102DA7295F9D721531C3FF4C1AE66
:10B2F000023205EB0213DB7AC3F34503012B0ED9AF
:10B30000013B03F03F0305EB0212D17A63F34601E0
:10B31000FF23D17285F8D731ABE6002305E7002380
:10B32000F1E700BF5C5E00242DE9F04390F828307F
:10B3300083B00446013B082B0BD8DFE803F0393D0E
:10B340001F24052A0A2F34000121FEF71BF90128CA
:10B3500002D003B0BDE8F08300222378216C84F88A
:10B360002820002BF5D00322E162D4E9010384F800
:10B370002820834238BF03462046A36003B0BDE8BF
:10B38000F043FEF77BBC002103B0BDE8F043FEF7BD
:10B39000F9B803B0BDE8F043FEF7EEB903B0BDE87D
:10B3A000F043FEF77DB903B0BDE8F043FEF7EABA1B
:10B3B00003B0BDE8F0435DE5DFF830914368D9F8AC
:10B3C0001C62026B19461E40D9F8140294F800C0A2
:10B3D000B5184702B5EB402F41D34FF6F778BCF1D3
:10B3E000020F14D025692846002D5AD16168A36840
:10B3F0000020E26A8B4284F8280038BF0B46A36025
:10B40000002AA6D0204603B0BDE8F043104761688B
:10B41000D9F82402B1EB402F5CD22069217E0907C4
:10B4200032D5D9F89811451CA9422AD299F8B811F9
:10B43000002943D1012389F8B83189F80130226B02
:10B44000636894F800C0D21B3B4432449B1B002627
:10B450009742194663602263C4E90450BFD9BCF126
:10B46000020F37D02569002DC1D099F80030032B89
:10B4700036D0ADB24FF6F7739D42B8D81144616033
:10B48000B5E7E0D10025DEE701A968F07DFA0128E3
:10B490007FF45FAF2069019D94F800C06368226B60
:10B4A000D1E799F8001003290ED0A9B2414594BF05
:10B4B000002101210029B1D06168D4E7012189F878
:10B4C000011094F800C0BEE707498D4294BF0021E7
:10B4D0000121EFE7D9F82432B1EB432FCED386E731
:10B4E000014B9D4283D8C9E7F7FFFF0FA05C002402
:10B4F00088422DE9F04198464FF0010439D301FB11
:10B5000004F4B0FBF4FC8C45F9D264B30025BCF123
:10B51000000F04FB1C00B4FBF1F7D4BF002601268A
:10B520006DB966B9A142354619D9C6460CF1300C41
:10B530000EF801CB00238EF80030BDE8F081BCF19D
:10B54000090F18DD002A0CBF57233723C646634472
:10B55000A14205F101050EF8013BF046EAD83C4650
:10B56000B0FBF7FCD3E7C64600238EF80030BDE8F9
:10B57000F0818446CAE73023E8E700BF2DE9F041B7
:10B580000446154608469442B4FBF2F607D205FB82
:10B590001644134B1B5D00F8013BBDE8F081964259
:10B5A000B6FBF2F70CD20E4B05FB176705FB1644F2
:10B5B000DA5D1B5D00F8012B00F8013BBDE8F0816E
:10B5C000BA42B7FBF2F807D905FB1878044B13F819
:10B5D000082000F8012BE7E74046FFF7CFFFF3E72D
:10B5E00028560D08B5EEC00ADFED357A0023F1EEDE
:10B5F00010FA30B5C8BF30EE270A87B0D8BF30EE9A
:10B60000670ADFED307A054603A9029320EE270A88
:10B61000CDE90033FDEEC07A17EE904A84EAE4707B
:10B62000A0EBE47068F0D6FF002C03A8B4BF2D2374
:10B6300020238DF800307BF003F901282AD002285E
:10B6400034D003281ED003A968467BF039F8684639
:10B650007BF0F6F8044669462846033CE4B22246ED
:10B6600077F00EFC002328462B557BF0E9F82E22BC
:10B67000431C0DEB04012A54E8187BF041F82846DE
:10B6800007B030BD302303A968468DF801307BF048
:10B6900017F8DCE743F23002302303A96846ADF81F
:10B6A00001208DF803307BF00BF8D0E743F2300334
:10B6B00003A96846ADF801307BF002F8C7E700BF88
:10B6C0006F12033A00007A440378202B03D110F85C
:10B6D000013F202BFBD0092BF9D02D2B63D02B2B36
:10B6E000B7EE000A08BF01300278A2F13003D9B2E8
:10B6F000092961D8F2EE046ADFED4D7A07EE103ABF
:10B7000010F8012FB8EEC77AA2F13003D9B2A7EE34
:10B71000A67A0929F0EE477AF0D92E2A50D003787C
:10B7200003F0DF03452B3BD110B442782D2A73D0B0
:10B730002B2A62D0A2F130030130092B63D80024F8
:10B74000002303EB830302EB430310F8012FA2F164
:10B750003001303B0929F4D9B3F59A7F1A46B7EE88
:10B76000007A28BF4FF49A72072B09D91346DFEDF0
:10B77000316A083B27EE267A072BFAD802F0070237
:10B780002AB1F2EE046A013A27EE267AFBD1002CA8
:10B790003BD0C7EE877A5DF8044B20EE270A70474E
:10B7A00020EE270A704742780130BFEE000AA2F16E
:10B7B0003003D9B209299DD92E2ADFED1D7AAED1E9
:10B7C00043780130A3F13002D1B20929A8D8B2EEF2
:10B7D000047AF0EE475A06EE902A10F8013FB8EED0
:10B7E000E66AA3F13002D1B2C6EE076A092927EE54
:10B7F000257A77EEA67AEED992E782780230A2F126
:10B800003003092B9BD9B7EE007A67EE877A5DF893
:10B81000044B20EE270A704782780230A2F13003F1
:10B82000092B01D801248BE7B7EE007AB1E700BFFE
:10B830000000000020BCBE4C0378092B01D0202B57
:10B8400005D110F8013F202BFBD0092BF9D02D2B6F
:10B8500009D001784FF0010CA1F13002D3B2092BCD
:10B860000AD900207047417801304FF0FF3CA1F128
:10B870003002D3B2092BF4D8002310F8011F03EBD8
:10B88000830302EB4303A1F13002D1B20929F4D9B9
:10B890000CFB03F0704700BFAB4BAC4A2DE9F04FF7
:10B8A0004FF0000A97B09E1A41F221051F462C2244
:10B8B00000210DEB020078F00BFFA44AA44B089284
:10B8C000CDE90976DA68D10707D5A24A5A6002F1B4
:10B8D00088325A60DB68DC070DD49D4BD3F80C210D
:10B8E000D20708D59B4AC3F8042102F18832C3F875
:10B8F0000421D3F80C31002101227E2308A81491E1
:10B9000005A98DF854208DF81430FDF739FB002877
:10B91000C0F2298108214FF4FC4303E05B000139A8
:10B920009BB207D01AB2002AF8DA85EA420201393E
:10B9300093B2F7D1884AADF81630884B934280F025
:10B94000518198460DF11809CDE902A7B8F80220F7
:10B950004FF0000CB8F80030C2F30B0B10048DF858
:10B960001DC00BF10601ADF81810C3F30B014FEA2F
:10B970001333ADF81A108DF81C3000F191800622B7
:10B98000494608A8FDF7FCFA0028C0F2FD80BDF882
:10B99000164049460DF11E0011F8013B082284EAC9
:10B9A000032403E06400013AA4B207D023B2002BC1
:10B9B000F8DA85EA4303013A9CB2F7D18842EBD129
:10B9C0005A46D8F8041008A8FDF7DAFA0028C0F2A1
:10B9D000DB80D8F8041001EB0B00814215D001394F
:10B9E000013811F8013F082284EA032403E06400CF
:10B9F000013AA4B207D023B2002BF8DA85EA430358
:10BA0000013A9CB2F7D18142EBD1ADF8164008F172
:10BA10001408514B984599D3DDE902A7002302226F
:10BA2000494608A8ADF81830FDF7AAFA0028C0F278
:10BA30009A80BDF816300DF11A0041F2210119F873
:10BA4000012B082483EA022303E05B00013C9BB244
:10BA500007D01AB2002AF8DA81EA4202013C93B216
:10BA6000F7D14845EBD102220DF1160108A8ADF837
:10BA70001630FDF785FA002875DB1398002840F092
:10BA80008980149800286EDB9DF85420002A40F02D
:10BA9000978000280DBF012200220123002364E0CB
:10BAA000E2466746019601370622494608A8FFB2DA
:10BAB0008DF81D70FDF764FA002851DBBDF81640C3
:10BAC00049460DF11E0011F8013B082284EA0324C7
:10BAD00003E06400013AA4B207D023B2002BF8DAE5
:10BAE00085EA4303013A9CB2F7D18842EBD1D8F8FA
:10BAF00004105A4608A801EB0A063146FDF740FA41
:10BB000000282DDB06EB0B00864215D0711E013894
:10BB100011F8013F082284EA032403E06400013A9B
:10BB2000A4B207D023B2002BF8DA85EA4303013A26
:10BB30009CB2F7D18142EBD1032FDA44ADF8164025
:10BB4000B1D1019E63E700BF0000040800000208B5
:10BB5000002000522301674580090E08CC030E081F
:10BB6000DDE9016A039F012300220AF1010ABAF10B
:10BB7000020F02DC002B7FF49AAE12B1FCF754F8EE
:10BB800028B9052007F0F8FDDDE902A7EBE717B0BB
:10BB9000BDE8F08F089B099A03449342E3D80BABAE
:10BBA000C0F120022146184478F092FD149818B98B
:10BBB0000BA908A8F7F774FB00221490139261E711
:10BBC0000A4AD16841F00101D160D168C9077FF507
:10BBD00060AFD2F80C1141F00101C2F80C11D2F89B
:10BBE0000C2156E70DF1180918E700BF002000529C
:10BBF000007970470079C0F3401070470079400920
:10BC0000704700BF90F83C20034602F0FF0012B1DD
:10BC1000002283F83C2070474FF400638381704713
:10BC200031B10A4BD3ED077AFDEEE77AC1ED007A28
:10BC300052B1064B9FED067AD3ED087A67EE877A0C
:10BC4000FDEEE77AC2ED007A0120704700E800249B
:10BC50000000C842012070470E4B10B40E4C1B6808
:10BC6000606A1B1AFA2B09D809B1E36A0B600AB1A2
:10BC7000236B136001205DF8044B7047074A0021D5
:10BC80001368084684F8281023F004035DF8044B79
:10BC900013607047D030002400E8002490B50024E1
:10BCA00001207047044B0022002101205A639A634F
:10BCB000DA631964704700BF00E80024104B114993
:10BCC0001A680346086C121AFA2A16D8D1ED0D6AC2
:10BCD000012091ED0E7AFDEEE66AD1ED0F7ABDEE10
:10BCE000C77AFDEEE77A16EE902ADA8617EE102A6A
:10BCF0001A8717EE902A5A8770470020704700BFB6
:10BD0000D030002400E800240F4B70B593F8443085
:10BD100082B00191ABB90D4B1D6895B12B681A68C3
:10BD20007AB19B686BB104462846984748B101999F
:10BD300022462E6828460B46316802B0BDE87040A6
:10BD4000084702B070BD00BF00E80024F8B9002425
:10BD50000B4B70B51E688EB133681A6872B19B6860
:10BD600063B1054630460C46984738B131682A46DB
:10BD7000234630460968BDE87040084770BD00BFE3
:10BD800010BA0024014B9B6C5B68184700E8002444
:10BD9000024B08309B6C9B68184700BF00E80024EA
:10BDA0000120704701207047012070470120704733
:10BDB0000120704731B10B4BD3ED137AF8EEE77ADF
:10BDC000C1ED007A6AB10749074B096DDFED076ADB
:10BDD0000B4407EE903AF8EEE77A87EEA67A82ED0A
:10BDE000007A704700E800244D95FFFF0000C8422C
:10BDF00001207047012070477A4A0146002394468B
:10BE0000104610B490F904400C30012C4DD0013391
:10BE1000082BF7D1734C002394F904000C3402284A
:10BE200058D00133082BF7D16E4C002394F904004D
:10BE30000C3403286BD00133082BF7D1694C002355
:10BE400094F904000C34042877D00133082BF7D17F
:10BE5000644C002394F904000C34062800F083801D
:10BE60000133082BF6D1002392F904000C32072885
:10BE700000F093800133082BF6D15B4B1B68D8038D
:10BE800040F1A180594B086803F1F00403E014333A
:10BE9000A34200F098801A689042F8D1DA68D20183
:10BEA000F5D501205DF8044B704703EB43035CF8C4
:10BEB000233023B34E480B7990F8D14090F8D0004E
:10BEC000984218BF9C420CBF01200020A2D15DF80F
:10BED000044B704703EB43035CF823308BB14548B8
:10BEE0000B7990F8D04090F8D100984218BF9C424E
:10BEF0000CBF0120002097D15DF8044B7047394CEE
:10BF00008AE7384C94F904000C34032893D103EBEE
:10BF100043035CF82330002B3BD037480B7990F873
:10BF2000D04090F8D100984218BF9C420CBF01202D
:10BF3000002083D15DF8044B704703EB43035CF8AA
:10BF4000233043B32D480B7990F8D04090F8D100BE
:10BF5000984218BF9C420CBF012000207FF478AFAC
:10BF60005DF8044B704703EB43035CF82330002B70
:10BF70003FF47AAF22480B7990F8D04090F8D10086
:10BF8000984218BF9C420CBF012000208AD0034673
:10BF90006AE7144C54E7134C5CE703EB43035CF88B
:10BFA0002330002B3FF469AF164A0B7992F8D10089
:10BFB00092F8D0209A4218BF98420CBF012000206E
:10BFC0007FF45BAF6EE70A79203AD2B2152A06D821
:10BFD0000D4B5DF8044BD34003F001007047002087
:10BFE00060E700BF189A0024FC6B00242C03002497
:10BFF000340700240C0A0024E40C0024BC0F0024A5
:10C00000941200246C150024010033000B4B84466D
:10C01000002010B503F1F00E02E014339E450BD062
:10C020001A686245F9D1DA68441C8A42F5D0D960B1
:10C030001433E0B29E45F3D110BD00BF2C030024A1
:10C04000704700BF40F2FF72044B914203EBC00304
:10C05000A8BF1146A3F85810704700BF00E800249D
:10C06000112807D8044B03EB8003D3F8B4300BB18D
:10C070009B68196028F088BF00E80024112807D8C1
:10C08000044B03EB8003D3F8B4300BB19B68196009
:10C09000704700BF00E800240C4A13787BB10C4BBA
:10C0A00093F8FC1059B193F8FD1059B15068002273
:10C0B000FA2883F8FD20A8BF4FF0FF3070476FF0DB
:10C0C000010070476FF00200704700BF041B00249E
:10C0D00000E8002438B505680446EB69E3B19878B8
:10C0E00000B938BDB3F90420012007EE902AF8EE1C
:10C0F000E77AC4ED047AB3F9062007EE902AF8EE49
:10C10000E77AC4ED057AB3F9083007EE903AF8EE15
:10C11000E77AC4ED067A38BD09211420FEF7A0FCA9
:10C120000346E861DBE700BF70B506680D461446BC
:10C13000F069A0B3D0F80130CDB1D0F80520B7EE4A
:10C14000006A9FED1A7A07EE902ADFED195ADFEDAB
:10C15000196AF8EE677A77EEC77A77EEA77A87EEF4
:10C16000A57A77EE467A67EEE67AC5ED007AACB14D
:10C1700007EE903A9FED107ADFED105AF8EEE77A6D
:10C180009FED0F6ADFED0F6A67EE877A87EEA57A7B
:10C1900077EE467A77EEA67AC4ED007A70BD092173
:10C1A0001420FEF75DFCF061C4E700BF9AC9CC44DF
:10C1B0009AC94C460E76D7450000484300E0FF443C
:10C1C000000048423393884370B5066882B00D463C
:10C1D0001446F06900284AD0D0F80530F3EE096A19
:10C1E000DFED265AB2EE047A07EE903A9FED246A0C
:10C1F000D0F80130F8EE677A77EEE57A67EE867A66
:10C2000067EEA67AF4EEC77AF1EE10FA20DCBAEE09
:10C21000047AF4EEC77AF1EE10FA19D42DB19FED3D
:10C22000197A67EE877AC5ED007A7CB107EE903A0D
:10C230009FED156ADFED156AB8EE677ADFED147AC7
:10C24000E7EE067A77EEA67AC4ED007A02B070BD0A
:10C2500017EE900A7AF048FD04460D460D4A042177
:10C260000320CDE90045FEF775FB02B070BD092142
:10C270001420FEF7F5FBF061AEE700BF00000046BA
:10C28000000080380AD778430319C83D33938843A8
:10C29000000048C23C5A0D0890F91030F0B503EB8D
:10C2A0004303264E154683B056F833600446836830
:10C2B0009A0715D501230DF106028DF806103046B8
:10C2C0000DF10701F8F72CF801230022294630462A
:10C2D000F8F726F8A3689B0716D5012003B0F0BD38
:10C2E00043691BB19A88186812048261144B154A7D
:10C2F0001868154BC0005768A3FB003080095368CD
:10C30000DB1B9842FBD2D5E70D4A4FF4FA700E4B77
:10C3100012680C4900FB02F24868A3FB0232920942
:10C320004B681B1A9A42FBD26369002BD5D01A685E
:10C3300001209B88936103B0F0BD00BFCC020024B4
:10C34000CC300024001000E0D34D6210F0B504465C
:10C3500083B00D461746061D20680379012B19D0BE
:10C36000022B02D0002003B0F0BD83683246FF21CB
:10C37000DB075CBF3246FF21FFF78EFF0028F1D0BC
:10C3800015B12379DB07E7D4002FECD023793B707C
:10C3900003B0F0BD8268417C02F0010C90F91000FE
:10C3A000FF22CDE9006CF7F7C9FCE7E770B504465A
:10C3B000051D82B020680379012B16D0022B02D014
:10C3C000002002B070BD83682A46FF21DE075CBFF3
:10C3D0002A46FF21FFF760FF0028F1D02379DB0711
:10C3E000EFD520680379012BE8D18668FF22417CD4
:10C3F00006F0010690F91000CDE90056F7F79EFC13
:10C40000EAE700BF024630B5044652F8040B83B099
:10C410000379012B0ED0022B01D0002008E0FF2170
:10C42000FFF73AFF0028F8D02079C04300F0010060
:10C4300003B030BD8568417C05F0010590F910001E
:10C440000092FF220195F7F779FCEBE72DE9F04127
:10C450004FF0B046D6F88050D6F888301D4010D046
:10C46000DFF824800127B5FA85F4C4F11F0458F8D9
:10C47000240007FA04F403689847A543C6F88840E7
:10C48000F1D1BDE8F08100BF046C002438B514463A
:10C49000002944D0344B0D469FED344A93ED407A49
:10C4A000D3ED436AB8EEC76AB3F91C21B8EEE60AC9
:10C4B000D3ED417A04EE902AB3F91821C6EE046A4E
:10C4C00093ED447A05EE902AB3F91A2105EE102A6D
:10C4D000B3F91621B3F91431F8EEE44A06EE102A46
:10C4E000F8EEE55AF8EEE77AB8EEC55AB8EEC77A34
:10C4F000C7EE843A07EE903AB8EEC66AE6EEA45A62
:10C50000F8EEE77AA6EE856AA6EEA57AE6EE867ADA
:10C51000A6EE870AA3EEA70A72F032FD28600CB3DC
:10C52000114BF6EE005A9FED115AD3ED416AB3F963
:10C530000A21F8EEE66AB3F9083107EE102A9FEDFA
:10C540000C6A07EE903A86EE850AB8EEC77AF8EEE6
:10C55000E77A20EE070AA7EEA50A20EE060A72F097
:10C560000FFD2060012038BD00E800240000F04AE3
:10C570000000C8420B4B03EBC00310B55C6D82B0EA
:10C5800001916CB107EE901A94ED047A94ED030AD0
:10C59000F8EEE77AA7EE870A72F0F2FCA36818605B
:10C5A00002B010BD00E80024174B70B5D3F820612D
:10C5B00026B1164A03213046F8F7C0FF0021304665
:10C5C000F8F7E8FC72680023114915695A0101EB7C
:10C5D000431401338A586A4012F47C5F07D0102B51
:10C5E000F4D100220B4BF2607361002070BD094949
:10C5F000F4607161237F002BF7D1304640F62B4267
:10C60000BDE8704067F0AEBC00E80024009F240045
:10C61000CC0000243C07003038B50E4DD5F8204141
:10C6200024B10D4A64212046F8F788FF00212046F6
:10C63000F8F7B0FC2046F8F771FE2368586890F8C8
:10C640003D30012B01D170F0CFF9012385F8243161
:10C6500038BD00BF00E80024009F2400F8B5544B0B
:10C660000D4614462DED048B1B7F022B18D09FED39
:10C67000510A7DB120EE000ADFED4F7ADFED4F6AFF
:10C680009FED4F7A20EE270AC0EE267A77EE877A62
:10C69000C5ED007A0CB14B4B2360BDEC048BF8BDAB
:10C6A000494B4A4E1B6896F8251103F00202C1B9A6
:10C6B0005B0516D4B2B1464BB3F9182001EE102A2F
:10C6C000B3F91620B3F9143000EE902AB8EEC11A6F
:10C6D00000EE103AF8EEE00AB8EEC00AFDF768FF87
:10C6E000C7E722B9D6F8343193ED330AC1E7D6ED66
:10C6F0004A8A96ED4B9AF0EE680AB0EE490AFDF7C9
:10C7000033FDB5EEC00AB0EE408AF1EE10FA47D420
:10C71000B0EE680A2F4FF0EE490AFDF733FFDFED68
:10C720002E7ADFED2E6AF0EE408A28EE278AD7F8BF
:10C73000EC239FED2B6A9FED2B7AC8EE267AFCEE58
:10C74000E77A17EE903A9BB29B1A07EE903AF8EE12
:10C75000E77A67EE867AA7EEA67AFDEEC77AB0EEA4
:10C76000470A17EE903A2033402B1ED8FDF738FFCA
:10C77000F0EE407A1C4BB97CA3F12C021846443BE6
:10C78000D6ED4C0A90ED000A002918BF1346A8EE1A
:10C79000E70AD3ED057A70EEA70AFDF7F3FE68E726
:10C7A000DFED127A30EE278AB2E7DFED027AE1E7B9
:10C7B00010B6002400000000CDCC9C3F00409C46F9
:10C7C00082E6C547331390432071002400E800241B
:10C7D000B89A0024E89A00240000C84235FA8E3C3A
:10C7E0000AD7233CDB0FC93FE89E0024DB0FC9407A
:10C7F00070B545880B4604460021C5F30B05184665
:10C800002A4677F065FF0A4A21690346914206D31A
:10C81000084A914206D31846BDE8704008470029EF
:10C82000F9D170BD2A46BDE8704076F029BB00BF43
:10C8300080090E08AF0E0E0810B5037982B08E463F
:10C84000012B0DD0022B02D0002002B010BD836856
:10C85000DB0758BF41F0800102B0BDE810401BE586
:10C86000816814467246009401F00104417C90F9FD
:10C8700010000194F7F762FA02B010BD10B504463B
:10C88000C06900B110BD09211420FEF7E9F8E0618C
:10C8900010BD00BF18B1838802681B049361704704
:10C8A000184B03EB8000D0F8380138B300EB4000A0
:10C8B00003EB800292F949C1BCF1FF3F1FD092F80F
:10C8C0005101D8B103EB0C00002310B590F89CE1A6
:10C8D0008C2092F85011142200FB0CFC0A4C0CEB3B
:10C8E0000100013A714434F8100013FA80F3F6D1D4
:10C8F000064AA2FB0320C0F30F1010BD70470020B2
:10C90000704700BF00E8002400000030CDCCCCCC44
:10C9100030B50D4683B003201446FFF7C1FF0190E8
:10C920009DB107EE900ADFED0B5AB0EE006ADFED25
:10C930000A6AF8EE677AB8EE047A67EEA57AA7EE8F
:10C94000867A67EE267AC5ED007A0CB1034B236038
:10C9500003B030BD6740533A00007A44331390432C
:10C960000379022B00D0704790F9102008311E483F
:10C9700002EB420210B44FF4807483B050F83220BE
:10C98000ADF800406944194C8DF80230A24211F80C
:10C9900008CC24D016498A4223D001F580618A420E
:10C9A00005D0144B9A420CBF03234FF0FF3311689C
:10C9B00003EB430321F0010100EBC30011600169A7
:10C9C000936851F82C1023F0E0430B4393601368F5
:10C9D00043F00103136003B05DF8044B704700237C
:10C9E000E5E70123E3E700BFCC020024003001406B
:10C9F00000380040003401400379022B00D070471A
:10CA000083689B07FBD543691BB19A881968120498
:10CA10008A61074A074B12680749D2004868A3FB9E
:10CA2000023292094B681B1A9A42FBD2704700BF30
:10CA3000CC300024D34D6210001000E090F910308B
:10CA4000F0B503EB4303284E154683B056F8336028
:10CA5000044683689A0719D501230DF106028DF863
:10CA6000061030460DF10701F7F75AFC01230DF1CE
:10CA700006020DF1070130468DF80650F7F750FC1D
:10CA8000A3689B0716D5012003B0F0BD43691BB115
:10CA90009A88186812048261144B154A1868154B5D
:10CAA000C0005768A3FB003080095368DB1B984225
:10CAB000FBD2D1E70D4A4FF4FA700E4B12680C49C5
:10CAC00000FB02F24868A3FB023292094B681B1A72
:10CAD0009A42FBD26369002BD5D01A6801209B884B
:10CAE000936103B0F0BD00BFCC020024CC30002421
:10CAF000001000E0D34D621010B5037984B0844675
:10CB00008E46012B0DD0022B02D0002004B010BDA8
:10CB10008368DB0758BF01F07F0104B0BDE8104017
:10CB20008CE781680DF10F001446724601F0010197
:10CB30008DF80F40CDE900019CF811109CF9100010
:10CB4000F6F7E0FE04B010BD70B5B42282B0044622
:10CB5000FF210068FFF7D0FF10B9002002B070BDC0
:10CB60002068251D0379012B13D0022BF5D1836892
:10CB70002A46FF21DE075CBF2A46FF21FFF78CFB18
:10CB80000028EAD02379DB07E8D520680379012B58
:10CB9000EBD18668FF22417C06F0010690F9100077
:10CBA000CDE90056F7F7CAF8EAE700BF70B50A46C4
:10CBB00082B00446A5210068FFF79EFF10B900204F
:10CBC00002B070BD2068251D0379012B13D0022B04
:10CBD000F5D183682A46FF21DE075CBF2A46FF2184
:10CBE000FFF75AFB0028EAD02379DB07E8D5206855
:10CBF0000379012BEBD18668FF22417C06F0010608
:10CC000090F91000CDE90056F7F798F8EAE700BF71
:10CC1000002A34D0F0B5044683B00E46051D8F18A7
:10CC200016F8012BA5212068FFF766FF90B90020B8
:10CC300003B0F0BD8268417C02F0010C90F9100055
:10CC4000FF22CDE9005CF7F779F80028EFD02379CF
:10CC5000DB070FD520680379012BEBD0022BE6D13F
:10CC600083682A46FF21DB075CBF2A46FF21FFF7C6
:10CC700013FBEAE7B742D3D1012003B0F0BD012096
:10CC8000704700BFF0B5962283B00E460446FF21E0
:10CC90000068FFF731FF10B9002003B0F0BD251D7B
:10CCA00020680379012B1DD0022BF5D183682A4619
:10CCB000FF21DF075CBF2A46FF21FFF7EDFA0028BE
:10CCC000EAD02379DB07EBD4E12220681146FFF795
:10CCD00013FF0028E0D03246FF21206803B0BDE8F2
:10CCE000F040A9E58768FF22417C07F0010790F931
:10CCF0001000CDE90057F7F721F8E0E7002A42D00D
:10CD0000F0B5044683B00E46051D8F189622FF210C
:10CD10002068FFF7F1FE90B9002003B0F0BD8268F3
:10CD2000417C02F0010C90F91000FF22CDE9005C7B
:10CD3000F7F704F80028EFD02379DB070FD5206838
:10CD40000379012BEBD0022BE6D183682A46FF2121
:10CD5000DB075CBF2A46FF21FFF79EFAEAE7E122E4
:10CD600020681146FFF7C8FE0028D5D03246FF21C3
:10CD70002068FFF761FD0028CED00136B742C5D14B
:10CD8000012003B0F0BD0120704700BFF0B50B4695
:10CD900005461646044683B087211A4655F8040B0B
:10CDA000FFF7AAFE20680379012B19D0022B02D0CD
:10CDB000002003B0F0BD83682A46FF21DF075CBF77
:10CDC0002A46FF21FFF768FA0028F1D02379DA0715
:10CDD000E8D4002EEDD0C3F34013337003B0F0BDA0
:10CDE0008768FF22417C07F0010790F91000CDE928
:10CDF0000057F6F7A3FFE7E7F0B5782183B01646B2
:10CE0000044600220068FFF777FE10B9002003B047
:10CE1000F0BD251D20680379012B13D0022BF5D11D
:10CE200083682A46FF21DF075CBF2A46FF21FFF700
:10CE300033FA0028EAD02379DA07EBD45B093370A0
:10CE400003B0F0BD8768FF22417C07F0010790F92D
:10CE50001000CDE90057F6F771FFEAE770B5CC2274
:10CE600082B00446A5210068FFF746FE10B90020F5
:10CE700002B070BD2068251D0379012B13D0022B51
:10CE8000F5D183682A46FF21DE075CBF2A46FF21D1
:10CE9000FFF702FA0028EAD02379DB07E8D52068FB
:10CEA0000379012BEBD18668FF22417C06F0010655
:10CEB00090F91000CDE90056F6F740FFEAE700BF11
:10CEC00070B5B42282B00446FF210068FFF714FE5B
:10CED00010B9002002B070BD251D20680379012B18
:10CEE00021D0022BF5D183682A46FF21DE075CBFE3
:10CEF0002A46FF21FFF7D0F90028EAD02379DA0784
:10CF0000EBD4CC212046FFF751FE0028E1D002E00F
:10CF10002379DB07DED52A46FF212068FFF78CFC4A
:10CF20000028F5D1D5E78668FF22417C06F001068E
:10CF300090F91000CDE90056F6F700FFDCE700BFDE
:10CF400070B582B00446CDE90023FFF7FDFD10B9AE
:10CF5000002002B070BD5522A5212068FFF7CCFD4E
:10CF60000028F5D0251D2A46FF212068FFF764FC24
:10CF70000028EDD02379DB07F5D40DF1FF350DF155
:10CF8000070615F8011F2046FFF710FE0028DFD026
:10CF9000B542F6D1DDE700BF2DE9F04F82468DB0F6
:10CFA000002090460AF10407089106900A93079022
:10CFB000069B5046DC0008EBC3030593FFF7C4FD56
:10CFC00028B941E09AF8043013F0010208D03A463B
:10CFD000FF21DAF80000FFF72FFC0028F2D133E040
:10CFE00003929A070B9040F1CC80F0215046FFF756
:10CFF000DDFD48B3083CDDF80C9008EB0403012488
:10D0000009932546089B003B18BF01230493049B0A
:10D01000082D8CBF002303F001039B46002B5DD03D
:10D020006E1E089B43FA06F606F00106F20178210F
:10D03000DAF80000FFF760FD30B1DAF8000003799C
:10D04000012B3FD0022B07D000220A9B10460699E5
:10D0500019700DB0BDE8F08F83683A46FF21DB07F9
:10D060005CBF3A46FF21FFF717F90028ECD09AF889
:10D07000043013F00102E0D199094FEA531E4FEA40
:10D08000D31C01EA5313DB074BD4664502D0BBF136
:10D09000000F73D1BCF1000F2DD0059911F80930A4
:10D0A000234301F809306400013514F0FF04EDB2A8
:10D0B000ADD109F101095FFA89F9B9F1080F30D052
:10D0C0000124A4E78268417C02F0010C90F9100071
:10D0D000FF22CDE9007CF6F731FEC6E7069BD3B10F
:10D0E000079BAB4217D9099B13F809301C4214BFA8
:10D0F000012600269AE74EEA0101039B11F0010F79
:10D10000059908BF2B46039311F8093023EA04035D
:10D1100001F80930C7E7079B5E1BB6FA86F6760969
:10D1200084E7402D07D80A9B069A1B7893423FF666
:10D130003FAF024689E7059BDD795C1E9E1D14F812
:10D1400001CF082182EA0C0301394FEA5C0C43F35A
:10D15000000311F0FF0123F0730383EA5202D2B2FD
:10D16000F0D1A642EBD19542DDD1069B0133DBB273
:10D170000693039B002BDCD00793D4E70B9E32462B
:10D1800063E70646324660E72DE9F0430768642608
:10D1900089B0B6227E2180463846FFF7ADFC06F006
:10D1A0008FFA04460D4606F08BFA001B61EB050171
:10D1B000B0F57A7F71F10001F5D3013EEFD1022184
:10D1C0003846FFF7CDFB7B691BB19A8819681204BA
:10D1D0008A6106F075FA04460D4606F071FA001BE6
:10D1E00061EB0501B0F57A7F71F10001F5D37B6940
:10D1F00013B11A689B8893610A2606F061FA044607
:10D200000D4606F05DFA001B61EB0501B0F57A7F73
:10D2100071F10001F5D3013EEFD132467C21384651
:10D22000FFF76AFC06F04CFA04460D4606F048FA91
:10D23000001B61EB0501B0F57A7F71F10001F5D3B8
:10D24000002259213846FFF757FC06F039FA044608
:10D250000D4606F035FA001B61EB0501B0F57A7F4B
:10D2600071F10001F5D397F910305E21A34A03EB69
:10D2700043038DF81F1052F83340BB689A0740F102
:10D28000108101230DF11F0200212046F7F748F815
:10D290004FF4A4739A4A20460021F7F741F8BB687F
:10D2A0009B0740F112810A2606F00AFA04460D4651
:10D2B00006F006FA001B61EB0501B0F57A7F71F10B
:10D2C0000001F5D3013EEFD1012259213846FFF785
:10D2D00013FC06F0F5F904460D4606F0F1F9001BC3
:10D2E00061EB0501B0F57A7F71F10001F5D38C2275
:10D2F00040213846FFF700FC06F0E2F904460D46EF
:10D3000006F0DEF9001B61EB0501B0F57A7F71F1E3
:10D310000001F5D3032241213846FFF7EDFB06F06B
:10D32000CFF904460D4606F0CBF9001B61EB050171
:10D33000B0F57A7F71F10001F5D3724D4FF448607A
:10D34000D8F83810704A98F8353002F1120E1446A9
:10D35000B5FBF1F5ADB202E00632724516D0117898
:10D3600084460029F8D1291AB2F802900029A5EBC9
:10D370000906B8BF4942002EB8BF7642B142EBDD84
:10D38000144606324846CC467245E8D1CDF808C06E
:10D390000120009561795D4A0491217903912178FA
:10D3A00001910321FDF7D6FA6288564B4221384697
:10D3B000B3FBF2F3C8F84030227942F0C002FFF725
:10D3C0009BFB06F07DF904460D4606F079F9001B3B
:10D3D00061EB0501B0F57A7F71F10001F5D3082208
:10D3E00043213846FFF788FB06F06AF904460D46EC
:10D3F00006F066F9001B61EB0501B0F57A7F71F16B
:10D400000001F5D3042258213846FFF775FB06F0DA
:10D4100057F904460D4606F053F9001B61EB050170
:10D42000B0F57A7F71F10001F5D30A225321384615
:10D43000FFF762FB06F044F904460D4606F040F99A
:10D44000001B61EB0501B0F57A7F71F10001F5D3A6
:10D4500000227C213846FFF74FFB06F031F90446E5
:10D460000D4606F02DF9001B61EB0501B0F57A7F42
:10D4700071F10001F5D306227D213846FFF73CFB10
:10D4800006F01EF904460D4606F01AF9001B61EB82
:10D490000501B0F57A7F71F10001F5D309B0BDE85F
:10D4A000F0837B691BB11A689B881B049361184B3E
:10D4B00018491A68184BD2004868A3FB0232920937
:10D4C0004B681B1A9A42FBD2DBE6114A4FF4FA7002
:10D4D000114B12680F4900FB02F24868A3FB0232AD
:10D4E00092094B681B1A9A42FBD27B69002B3FF4CE
:10D4F000DAAE1A689B889361D5E600BFCC0200249F
:10D50000E0AB0C0840420F00CCAB0C08605A0D0891
:10D51000CC300024001000E0D34D6210F0B583B091
:10D5200015461C4606460DF107020F46FFF784F923
:10D530009DF8072005EA0203A34201D103B0F0BD24
:10D5400022EA050239463046224303B0BDE8F040E6
:10D55000FFF7D2BAF8B50526782200210746006801
:10D56000FFF7CAFA06F0ACF804460D4606F0A8F834
:10D57000001B61EB0501B0F57A7F71F10001F5D375
:10D58000013EEFD10526202201213868FFF7B4FAC9
:10D5900006F096F804460D4606F092F8001B61EB83
:10D5A0000501B0F57A7F71F10001F5D3013EEFD1AD
:10D5B0003246642602213868FFF79EFA06F080F8AA
:10D5C00004460D4606F07CF8001B61EB0501B0F542
:10D5D0007A7F71F10001F5D3013EEFD10120F8BD52
:10D5E00070B52422044641210068FFF785FA90B9FE
:10D5F000052606F065F804460D4606F061F8001BA6
:10D6000061EB0501B0F57A7F71F10001F5D3013EC0
:10D61000EFD1012070BD202230212068FFF76CFA85
:10D620000028E5D0062231212068FFF765FA00289E
:10D63000DED0002234212068FFF75EFAD8E700BF71
:10D64000F8B5052607220A2107460068FFF754FAB5
:10D6500006F036F804460D4606F032F8001B61EB82
:10D660000501B0F57A7F71F10001F5D3013EEFD1EC
:10D670000526242241213868FFF73EFA06F020F8FB
:10D6800004460D4606F01CF8001B61EB0501B0F5E1
:10D690007A7F71F10001F5D3013EEFD10526C0225A
:10D6A00042213868FFF728FA06F00AF804460D46CA
:10D6B00006F006F8001B61EB0501B0F57A7F71F109
:10D6C0000001F5D3013EEFD10120F8BD10B50446AD
:10D6D000002221210068FFF70FFAFC222021206898
:10D6E000FFF70AFA402224212068FFF705FA0C22EE
:10D6F00023212068FFF700FA002222212068FFF78B
:10D70000FBF9012010BD00BFF8B50122074610212A
:10D710000068FFF7F1F900B9F8BD142605F0D0FF55
:10D7200004460D4605F0CCFF001B61EB0501B0F58A
:10D730007A7F71F10001F5D3013EEFD13868A02264
:10D740001121BDE8F840FFF7D7B900BF2DE9F0413E
:10D7500080220B2107460068FFF7CEF91E2680467F
:10D7600005F0AEFF04460D4605F0AAFF001B61EB75
:10D770000501B0F57A7F71F10001F5D3013EEFD1DB
:10D78000B8F1000F02D10020BDE8F0810622292166
:10D790003868FFF7B1F90028F5D008220B21386866
:10D7A000FFF7AAF90028EED03868CF220A21BDE899
:10D7B000F041FFF7A1B900BF10B5044694220B2138
:10D7C0000068FFF799F9712201212068FFF794F9A9
:10D7D000002204212068FFF78FF9C8220521206864
:10D7E000FFF78AF9002206212068FFF785F9C82291
:10D7F00007212068FFF780F9002208212068FFF741
:10D800007BF9C82209212068FFF776F9012010BDB5
:10D810000A4600212DE9F041DFF8B08084B042F0E3
:10D8200001020446274EFFF767F9D8F80070264D2D
:10D83000C6F8A07118E0022B4FF000000BD1A368CE
:10D840000DF10F0213212046DB0702D40DF10F0268
:10D850009321FEF721FD9DF80F30287013F0070388
:10D8600018D1D6F8A4212ABB2379012BE3D1A268D1
:10D870000DF10F0102F00102009101921322617C6F
:10D8800094F91000F6F75AFA9DF80F30287013F04B
:10D890000703E6D001220B212046FFF72DF90022D5
:10D8A00020461146FFF728F901232870184604B0D6
:10D8B000BDE8F081D8F8001089B2C91B8A42D3D2E2
:10D8C000F4E700BF00E80024041B0024D03000244B
:10D8D00000680379012B0AD0022B01D00020704789
:10D8E0008368F022DB0718D5FF21FFF7A7B882680D
:10D8F00090F910C002F00102417C60464FF0F00C3C
:10D9000010B584B00DF10F040192FF228DF80FC005
:10D910000094F5F7F7FF04B010BD7F21FFF78EB834
:10D9200070B5056884B004460E462B79012B16D0DD
:10D93000022B02D0002004B070BDAB68E122DB07EF
:10D940001DD528461146FFF779F80028F2D0324657
:10D95000FF21206804B0BDE87040FEF76DBFAA68E3
:10D96000697C02F0010295F910000DF10F0501929A
:10D97000E12200958DF80F20F5F7C4FFE5E761215E
:10D980002846FFF75BF8E0E770B5056884B0044609
:10D990000E462B79012B17D0022B02D0002004B0A9
:10D9A00070BDAB68C3222846DB074CBFE121612173
:10D9B000FFF744F80028F1D03246FF21206804B078
:10D9C000BDE87040FEF738BFAA6895F9100002F074
:10D9D0000102697C01920DF10F020092C3228DF8C1
:10D9E0000F20E122F5F78EFFE4E700BF0068CA438D
:10D9F000037941EA0211012BCAB209D0022B01D0EE
:10DA0000002070478368DB0716D5D221FFF716B8D0
:10DA100010B584B0846890F910C08DF80F200DF116
:10DA20000F0204F00104417C0092D222604601946E
:10DA3000F5F768FF04B010BD5221FEF7FFBF00BF2D
:10DA400070B5056884B004460E462B79012B1BD0B7
:10DA5000022B02D0002004B070BDAB68F022284633
:10DA6000DB074CBFE1216121FEF7E8FF0028F1D080
:10DA70002246FF2152F8040BFEF7DEFE0028E9D013
:10DA80002379337004B070BDAA6895F9100002F0D4
:10DA90000102697C01920DF10F020092F0228DF8D3
:10DAA0000F20E122F5F72EFFE0E700BF00680379C1
:10DAB000012B0AD0022B01D0002070478368B422CA
:10DAC000DB0718D5FF21FEF7B9BF826890F910C0B7
:10DAD00002F00102417C60464FF0B40C10B584B0F6
:10DAE0000DF10F040192FF228DF80FC00094F5F79D
:10DAF00009FF04B010BD7F21FEF7A0BF00680379C5
:10DB0000012B0AD0022B01D00020704783680A46FF
:10DB1000DB0716D5A521FEF791BF10B584B0846848
:10DB200090F910C00DF10F0204F001048DF80F10F0
:10DB3000417C60460092A5220194F5F7E3FE04B013
:10DB400010BD2521FEF77ABF00680379012B0AD0AA
:10DB5000022B01D00020704783689622DB0718D57E
:10DB6000FF21FEF76BBF826890F910C002F001023E
:10DB7000417C60464FF0960C10B584B00DF10F0457
:10DB80000192FF228DF80FC00094F5F7BBFE04B0A0
:10DB900010BD7F21FEF752BF00680379012B0AD028
:10DBA000022B01D00020704783680A46DB0716D598
:10DBB0008721FEF743BF10B584B0846890F910C088
:10DBC0000DF10F0204F001048DF80F10417C604646
:10DBD000009287220194F5F795FE04B010BD07214D
:10DBE000FEF72CBF0068C9010379CAB2012B06D029
:10DBF000022B01D0002070477821FEF71FBF10B51F
:10DC000084B0846890F910C08DF80F200DF10F02D8
:10DC100004F00104417C0092782260460194F5F7FB
:10DC200071FE04B010BD00BF00680379012B0AD05B
:10DC3000022B01D00020704783685522DB0718D5DE
:10DC4000A521FEF7FBBE826890F910C002F0010228
:10DC5000417C60464FF0550C10B584B00DF10F04B7
:10DC60000192A5228DF80FC00094F5F74BFE04B089
:10DC700010BD2521FEF7E2BE00680379012B07D015
:10DC8000022B01D0002070471A460821FEF7D6BEAD
:10DC9000826890F910C002F00102417C60464FF0AA
:10DCA000020C10B584B00DF10F04019208228DF81A
:10DCB0000FC00094F5F726FE04B010BD006803798C
:10DCC000012B07D0022B01D0002070470122082130
:10DCD000FEF7B4BE8268417C02F0010210B590F9F3
:10DCE000104084B020460DF10F04019208220094E8
:10DCF0008DF80F30F5F706FE04B010BD10B50446E0
:10DD0000006884B00379012B12D0022B02D00020CE
:10DD100004B010BD01220B21FEF790FE0028F6D0C2
:10DD20001D220921206804B0BDE81040FEF7E4BEC2
:10DD3000826890F910C002F00102417C60468DF8C3
:10DD40000F3001920DF10F0200920B22F5F7DAFD70
:10DD5000E4E700BF2DE9F04105461F462848164676
:10DD600095F9103082B003EB430350F83380AB6871
:10DD70009A0716D501230DF106028DF806104046CC
:10DD80000DF10701F6F7CCFA3B463246002140463A
:10DD9000F6F7C6FAAB689B0718D5012002B0BDE8BC
:10DDA000F0816B691BB19A88186812048261154B67
:10DDB0001868154BC000A3FB0030144B80095A684B
:10DDC0005C68A4EB020C6045FAD2D3E70D4A4FF42D
:10DDD000FA700D4B12680D4900FB02F24868A3FB74
:10DDE000023292094B681B1A9A42FBD26B69002BD4
:10DDF000D3D01A6801209B88936102B0BDE8F081FE
:10DE0000CC020024CC300024D34D6210001000E07E
:10DE100030B5057983B084468E46012D0DD0022D94
:10DE200002D0002003B030BD8468E40758BF41F041
:10DE3000800103B0BDE830408CE7806814460A4694
:10DE4000009400F001049CF811109CF9100001945A
:10DE5000F5F758FD03B030BDF0B5002383B01426AC
:10DE600007468DF8023005F02BFC04460D4605F000
:10DE700027FC001B61EB0501B0F57A7F71F1000111
:10DE8000F5D3013EEFD131460DF102023868FEF7BD
:10DE9000D3FC0DF1020280213868FEF7CDFC4FF46F
:10DEA000F8428DF806601426ADF80420032301AA79
:10DEB00060213868FFF7ACFF05F002FC04460D4610
:10DEC00005F0FEFB001B61EB0501B0F57A7F71F1F7
:10DED0000001F5D3013EEFD131460DF10302386860
:10DEE0008DF80360FEF7A8FC4CF26243142601AAE9
:10DEF0006021ADF80430042338688DF80630032320
:10DF0000FFF786FF05F0DCFB04460D4605F0D8FB65
:10DF1000001B61EB0501B0F57A7F71F10001F5D3CB
:10DF2000013EEFD131460DF1030238688DF80360F0
:10DF3000FEF782FC4FF4E853142601AA6021ADF8E5
:10DF40000430082338688DF806300323FFF760FF9C
:10DF500005F0B6FB04460D4605F0B2FB001B61EB75
:10DF60000501B0F57A7F71F10001F5D3013EEFD1E3
:10DF70000DF10302314638688DF80360FEF75CFC52
:10DF80000DF102021E213868FEF756FC012003B095
:10DF9000F0BD00BF10B5164C82B0037984F8AA21F9
:10DFA0000022012B84F8A91184F8A82110D0022B9B
:10DFB00003D06FF00C0002B010BD032304F5D4723F
:10DFC000FF21FFF7C7FE0028F3D0002002B010BDEC
:10DFD000816804F5D4740323FF2201F00101CDE927
:10DFE0000041417C90F91000F5F78CFCEBE700BF95
:10DFF00000E800242DE9F04105461F462848164652
:10E0000095F9103082B003EB430350F83380AB68CE
:10E010009A0716D501230DF106028DF80610404629
:10E020000DF10701F6F77CF93B46002231464046E8
:10E03000F6F776F9AB689B0718D5012002B0BDE86A
:10E04000F0816B691BB19A88186812048261154BC4
:10E050001868154BC000A3FB0030144B80095A68A8
:10E060005C68A4EB020C6045FAD2D3E70D4A4FF48A
:10E07000FA700D4B12680D4900FB02F24868A3FBD1
:10E08000023292094B681B1A9A42FBD26B69002B31
:10E09000D3D01A6801209B88936102B0BDE8F0815B
:10E0A000CC020024CC300024D34D6210001000E0DC
:10E0B00030B5057983B084468E46012D0DD0022DF2
:10E0C00002D0002003B030BD8468E40758BF41F09F
:10E0D000800103B0BDE830408CE7806814460A46F2
:10E0E000009400F001049CF811109CF910000194B8
:10E0F000F5F724FE03B030BD10B582B00821044608
:10E1000000686A46FEF798FB9DF80030DB0602D4F3
:10E11000002002B010BD06236A4600212068FFF7E8
:10E12000C7FF0028F4D09DF801209DF800101202CE
:10E130009DF80230DFED496A02EB01429DF80410C0
:10E1400014024FEA01219DF8034013449DF8052075
:10E1500001EB044148BF03F17F430A44090207EE83
:10E16000903A3F4B48BF02F17F42F8EEE77A93EDD9
:10E17000026A07EE102AB3F90C20F8EEC65AB3F97A
:10E180001210B8EEC77A93F8A84204EE901AB3F9C9
:10E190001610112CC7EE263A87EEA67A06EE902AC4
:10E1A000B3F90E20D3ED017A06EE102AB3F9102050
:10E1B00005EE102AB3F91420F8EEE66A04EE102AF0
:10E1C000F8EEE77AB8EEC66AB3F91820B8EEC55A89
:10E1D000F8EEE44AB8EEC44A66EEA36A27EE232AB4
:10E1E00023D0A7EE045AA7EE246AE5EE075AE5EE1F
:10E1F000877A77EEA67AE6EE027AB3F90220F6EE97
:10E20000006AC3ED077A07EE902AB3F90010F8EE22
:10E21000E77A07EE101AB8EEC77A67EEA37AE7EE50
:10E22000267AC3ED087A02B010BD03EE102AF8EE8C
:10E23000C32A03EE101AB8EEC33AA7EE224AE7EE5D
:10E24000034AA4EE075AA4EE876AE5EE075AE5EE04
:10E25000877A77EEA67AE6EE027ACEE70000784873
:10E2600000E80024F0B5142683B000220A210746F6
:10E270000068FEF741FC05F023FA04460D4605F060
:10E280001FFA001B61EB0501B0F57A7F71F1000107
:10E29000F5D3013EEFD10A260F220A213868FEF796
:10E2A0002BFC05F00DFA04460D4605F009FA001B9B
:10E2B00061EB0501B0F57A7F71F10001F5D3013E04
:10E2C000EFD10A26032301AA10213868FFF7F0FED8
:10E2D00005F0F6F904460D4605F0F2F9001B61EB76
:10E2E0000501B0F57A7F71F10001F5D3013EEFD160
:10E2F0009DF804209DF805009DF806108032194B0A
:10E3000080308031A3F8AC2232460A26A3F8AE0250
:10E31000A3F8B0120A213868FEF7EEFB05F0D0F939
:10E3200004460D4605F0CCF9001B61EB0501B0F584
:10E330007A7F71F10001F5D3013EEFD10DF10302B7
:10E3400002213868FEF778FA0DF1030209213868D6
:10E35000FEF772FA11220A213868FEF7CDFB012080
:10E3600003B0F0BD00E80024026830B5137985B031
:10E370000446012B61D0022B03D00025284605B0AE
:10E3800030BD916802AD1046C9072A464CBF1946F8
:10E390008221FDF781FF0028EFD09DF80830DA07D1
:10E3A000EBD52A46072303212068FFF781FE0546A7
:10E3B0000028E2D011220A212068FEF79DFB9DF87B
:10E3C0000E301B07D9D42A49BDF80830B1F8AC2269
:10E3D00013FB02F3274A93423EDBB3F5000F39DA11
:10E3E000002BB8BFFF331B125B421BB2BDF80A20E3
:10E3F000E386B1F8AE3212FB03F31E4A93422FDBE1
:10E40000B3F5000F30DA002BB8BFFF3343F30F2210
:10E41000BDF80C30B1F8B012228713FB01F3154A96
:10E4200093421BDBB3F5000F1CDA002BB8BFFF33A0
:10E430001B125B421BB26387A0E7517C02AD92F9CD
:10E4400010009268009502F0010201920222F5F795
:10E4500075FCA0E7084BC9E7084BC7E7074BEAE79D
:10E46000064AD5E7044BE6E747F6FF72D0E700BF60
:10E4700000E8002401FF7FFF0180FFFF0080FFFF15
:10E48000F0B5142683B000220A2107460068FEF783
:10E4900033FB05F015F904460D4605F011F9001B94
:10E4A00061EB0501B0F57A7F71F10001F5D3013E12
:10E4B000EFD10A260F220A213868FEF71DFB05F06E
:10E4C000FFF804460D4605F0FBF8001B61EB050163
:10E4D000B0F57A7F71F10001F5D3013EEFD10A2644
:10E4E000032301AA10213868FFF7E2FD05F0E8F8E0
:10E4F00004460D4605F0E4F8001B61EB0501B0F59C
:10E500007A7F71F10001F5D3013EEFD132460A2640
:10E510000A213868FEF7F0FA05F0D2F804460D46F5
:10E5200005F0CEF8001B61EB0501B0F57A7F71F1C3
:10E530000001F5D3013EEFD10DF10302022138684D
:10E54000FEF77AF90DF1030209213868FEF774F934
:10E5500001220A213868FEF7CFFA012003B0F0BD8E
:10E5600030B5002385B004460221C0F836300DF1E5
:10E57000070243870068FEF75FF918B19DF807307E
:10E58000DB0703D40025284605B030BD062302AAC8
:10E5900003212068FFF78CFD0DF107020921206897
:10E5A000FEF74AF905460028ECD09DF8073013F035
:10E5B0000C0FE7D1BDF80820BDF80C30BDF80A10EB
:10E5C000C2EB8232C3EB8333206889009B00920048
:10E5D000218763870A21E2860122FEF78DFA284609
:10E5E00005B030BD10B50446006882B003796A46B4
:10E5F000022B4FF006030CBF43210321FFF758FD08
:10E6000068B1BDF80010BDF80220BDF8043049BA69
:10E6100052BA5BBAE1866287238702B010BDC4F8A4
:10E620003600608702B010BD10B5002386B00446E6
:10E6300000688DF80F300379012B31D0022B02D006
:10E64000002006B010BD83680DF10F02D9074CBF42
:10E650002721A721FDF720FE0028F1D09DF80F30DB
:10E660001B07EDD5062304AA28212068FFF720FD0B
:10E6700028B3BDF91030002BB8BF03339A10BDF991
:10E680001230002BE286B8BF03339A10BDF9143064
:10E69000002B2287B8BF03339B10638706B010BDE1
:10E6A0008268417C02F0010290F910C001920DF1E4
:10E6B0000F02604600922722F5F740FBCCE7C4F832
:10E6C000360060870020BCE730B54FF0000C0446F0
:10E6D000006887B0C4F836C0A4F83AC00379012BAB
:10E6E0002AD0022B02D0002007B030BD83680DF184
:10E6F0000F02D9074CBF61468021FDF7CDFD0028F0
:10E70000F1D09DF80F301B07EDD5062304AA012197
:10E710002068FFF7CDFC0028E5D0BDF81430BDF827
:10E720001010BDF812205BBA49BA52BA5B42E186BA
:10E730002287638707B030BD85686246417C05F05B
:10E74000010590F9100001950DF10F050095F5F701
:10E75000F5FAD4E710B500230446006886B0C4F883
:10E76000363063870379012B23D0022B02D000209F
:10E7700006B010BD83680DF10F02D9074CBF06210A
:10E780008621FDF789FD0028F1D09DF80F30DB07C9
:10E79000EDD5062304AA00212068FFF789FC002894
:10E7A000E5D0049ABDF81430C4F83620638706B06B
:10E7B00010BD8268417C02F0010290F910C0019204
:10E7C0000DF10F02604600920622F5F7B7FADAE77C
:10E7D00010B500230446006886B0C4F8363063875D
:10E7E0000379012B29D0022B02D0002006B010BDE6
:10E7F00083680DF10F02D9074CBF09218921FDF76C
:10E800004BFD0028F1D09DF80F30DB07EDD5062336
:10E8100004AA01212068FFF74BFC0028E5D0BDF8D1
:10E820001210BDF81020BDF81430494252425B422C
:10E83000E1862287638706B010BD8268417C02F0C2
:10E84000010290F910C001920DF10F026046009292
:10E850000922F5F773FAD4E710B5002304460068DF
:10E8600086B0C4F8363063870379012B12D0022BAF
:10E870000DD183680DF10B02DB074CBF3421B421AD
:10E88000FDF70AFD18B19DF90B30002B11DB0020BC
:10E8900006B010BD8268417C02F0010290F910C000
:10E8A00001920DF10B02604600923422F5F746FA10
:10E8B000E8E7092303AA24212068FFF7F9FB0028D1
:10E8C000E5D09DF810209DF80F109DF8133012042C
:10E8D0001B0442EA01629DF8121043EA01639DF8AD
:10E8E0000C10C2F30F42C3F30F43228763879DF8D6
:10E8F0000D301B0443EA0163C3F30F43E38606B004
:10E9000010BD00BF70B5066882B00446F569002DE1
:10E910005CD0002204233046FF212A700DEB030255
:10E92000FFF7C6FB10B9002002B070BD04236A4691
:10E93000FF212068FFF7BCFB0028F4D09DF80430CD
:10E940009B09023B012BEED9BDF8043043F6FF7C56
:10E95000BDF806205BBABDF80010BDF80240C3F355
:10E960000D066645DFD0002EDDD053BA40F2FF7EA3
:10E97000C3F34A1272451346D5D0002AD3D049BA00
:10E98000C1F30D0262451146CDD0002ACBD064BA46
:10E99000C4F34A1272451446C5D0002AC3D0721A75
:10E9A000002AB8BF5242FF2ABDDC1A1B002AB8BF9A
:10E9B0005242FF2AB7DC23440E445B107610C5F8A0
:10E9C00001300123C5F805602B70ADE70921142043
:10E9D000FCF746F8F061054626689AE770B50668C8
:10E9E00082B0F469F4B100210423304621700DEBAC
:10E9F0000302FF21FFF75CFB10B39DF804309B0975
:10EA000019D1BDF804200121BDF8063052BA217099
:10EA10005BBA92B2C3F34A13C4F80520C4F80130BC
:10EA200002B070BD054609211420FCF719F8F06109
:10EA300004462E68D7E7044A04210320FBF78AFF27
:10EA4000002002B070BD00BF9C5A0D08F0B5484DC3
:10EA500083B095F8FC303BB195F8B2620446012EC4
:10EA600038D0022E54D00EB103B0F0BD0122802167
:10EA70000068FEF741F80122FF212068FEF73CF80C
:10EA8000324631462068FEF737F895F8B3229121D7
:10EA90002068FEF731F8314601222068FEF72CF895
:10EAA0003246FF212068FEF727F832468021206891
:10EAB000FEF722F8314601222068FEF71DF82D4BA3
:10EAC0002D4901221B68087085F8B222C5F8A031D3
:10EAD00003B0F0BD01AA00210068FDF7ADFE9DF86E
:10EAE0000430254FDA07387039D5D5F8A431002B1A
:10EAF000BAD0204AD5F8A011126892B2521A9342A5
:10EB0000B2D24FF0FF3200237A6085F8B232ABE721
:10EB100001AA13210068FDF78FFE9DF80430164FFF
:10EB20005B073870E1D0334601AA1E212068FFF749
:10EB3000BFFABDF80430206801225CBA0B21FDF752
:10EB4000DBFF0E4BA4B201223870A3FB0434002378
:10EB500085F8FD20E40885F8B2327C6084E7054B37
:10EB600002221B6885F8B222C5F8A0317CE700BFFD
:10EB700000E80024D0300024041B0024CDCCCCCCF1
:10EB800070B5066882B00546F469002C3ED0337932
:10EB9000E21C012B2DD0022B26D1B368304613F096
:10EBA000010F4FF00D0314BF0C218C21FFF722FA47
:10EBB000A070D8B1B4F90A3007EE903AF8EEE77ACF
:10EBC000C5ED077AB4F90C3007EE903AF8EEE77A23
:10EBD000C5ED087AB4F90E3007EE903AF8EEE77A10
:10EBE000C5ED097A02B070BD0023A370002002B009
:10EBF00070BDB368717C03F0010396F910000092B8
:10EC00000C2201930D23F5F799F8D1E7092114207F
:10EC1000FBF726FFF06104462E68B8E7006810B5E0
:10EC2000037984B00C46012B1AD0022B02D00020AD
:10EC300004B010BD836803AA13F0010F4FF0030363
:10EC400014BF2221A221FFF7D5F90028EFD0BDF98A
:10EC50000D3003EB83031B12E633238004B010BD99
:10EC6000836803AA417C03F0010390F9100000922D
:10EC7000222201930323F5F761F8E6E7006810B557
:10EC8000037984B0012B28D0022B01D0002022E090
:10EC9000836803AA13F0010F4FF003030CBF832115
:10ECA0001946FFF7A7F90028F0D09DF80C309DF920
:10ECB0000C109DF80D201B0400299DF80EC043EA9E
:10ECC00002230D4AACBF00214FF07F4143EA0C0301
:10ECD0000B43C2F8043104B010BD826803AC0323B7
:10ECE000417C02F0010290F91000CDE900421A4681
:10ECF000F5F724F8D7E700BF00E80024006810B556
:10ED0000037984B0012B28D0022B01D0002022E00F
:10ED1000836803AA13F0010F4FF0030314BF00210F
:10ED20008021FFF767F90028F0D09DF80C309DF99D
:10ED30000C109DF80D201B0400299DF80EC043EA1D
:10ED400002230D4AACBF00214FF07F4143EA0C0380
:10ED50000B43C2F8003104B010BD826803AC417CA3
:10ED6000032302F0010290F91000CDE900420022D5
:10ED7000F4F7E4FFD7E700BF00E8002410B504462D
:10ED8000006884B00379012B43D0022B07D0002206
:10ED900013461046C4F83620638704B010BD83685C
:10EDA00002AA13F0010F4FF0060314BF11219121A5
:10EDB000FFF720F90028EAD0BDF90C20B7EE086A69
:10EDC000BDF90A3007EE902ABDF908205B4206EE35
:10EDD000902AF8EEE77A07EE103AF8EEE66AB8EE17
:10EDE000C77A67EE867A66EE866A27EE067AFDEEC9
:10EDF000E77AFDEEE66ABDEEC77A17EE903A16EEB8
:10EE0000902A1BB2E28617EE102A6387228704B08D
:10EE100010BD836802AA417C03F0010390F9100041
:10EE20000092112201930623F4F788FFC2E700BF86
:10EE300010B500230446006884B0C4F836306387F8
:10EE40000379012B22D0022B01D000201CE0836823
:10EE500002AA13F0010F4FF0060314BF0321832110
:10EE6000FFF7C8F80028F0D0BDF90A30BDF8081047
:10EE7000BDF80C205B4201EB410102EB420203EBC7
:10EE80004303E1866287238704B010BD836802AA2A
:10EE9000417C03F0010390F91000009203220193DA
:10EEA0000623F4F74BFFDDE710B54FF0000C0446E6
:10EEB000006884B0C4F836C0A4F83AC00379012BC6
:10EEC00018D0022B01D0002012E0836802AA13F0B0
:10EED000010F4FF0060314BF61468021FFF78AF847
:10EEE0000028F0D0029ABDF80C30C4F836206387B1
:10EEF00004B010BD83686246417C03F0010390F9C1
:10EF000010E0019302AB704600930623F4F716FF5E
:10EF1000E6E700BF10B5002384B004460068029302
:10EF2000CDF80B300279012A1ED0022A19D183684C
:10EF300002AA13F0010F4FF0070314BF4E21CE2198
:10EF4000FFF758F8BDF80910BDF80B20BDF80D30DB
:10EF5000C9BAD2BADBBA0120E1862287638704B03E
:10EF600010BD1A461946F6E7826802AB90F910C048
:10EF700002F00102417C00936046019207234E2279
:10EF8000F4F7DCFEDEE700BF006810B5037984B05B
:10EF9000012B0BD0022B06D1012303AAFF21FFF77F
:10EFA00029F804B010BD002004B010BD826803AC85
:10EFB000417C02F0010290F9100000940192FF22BE
:10EFC000F4F7BCFE04B010BD0368DA6B10B504465C
:10EFD00082B012B1904740B123685B6B1BB12146F0
:10EFE00001A8984718B9FF23E38202B010BDBDF80D
:10EFF0000630013B9BB2F7E7F0B50D4683B00446FF
:10F00000184616461F4677F01BFC2844E67329462F
:10F01000A0732046256800243B46324600946C6964
:10F02000A04703B0F0BD00BF38B58B68044601604F
:10F030000D46984700230B4A237522612B6B13B1B1
:10F04000204698472075084B93F8B4321BB1237DB6
:10F0500023F00103237500232046E382BDE83840F6
:10F06000B2E700BF0001FF0000E80024144B30B5F8
:10F070001C6885B084B12379012B10D0022B0BD1F1
:10F08000A1680246204611F0010118BF802105B099
:10F09000BDE83040FDF7D2BC002005B030BDA2680D
:10F0A0000DF10F05617C8DF80F0094F9100002F04E
:10F0B0000104802200950194F4F724FC05B030BDD2
:10F0C000C8720024F0B5274D85B02868002846D0C6
:10F0D000B0228021FDF710FD286800283FD0402293
:10F0E0008021FDF709FD2868002838D00022802102
:10F0F000FDF702FD286890B310228021FDF7FCFC8B
:10F1000028684FF4806400270DF10F0670B1037971
:10F11000012B10D0022B09D183680022402113F06B
:10F12000010304BF1A464021FDF788FC013CA4B24C
:10F130009CB12868EAE78268013C90F910E002F08F
:10F14000010CA4B2417C402270468DF80F70CDE9CD
:10F15000006CF4F7D7FB002CEBD105B0F0BD00201C
:10F16000CFE700BFC872002410B50C4C2368A3B1D0
:10F17000A0F1500280211846D2B2FDF7BDFC2068F4
:10F1800058B100228021FDF7B7FC206828B1102279
:10F190008021BDE81040FDF7AFBC10BDC87200244F
:10F1A000A0F12003F0B503EB83031C4D1C4E85B08A
:10F1B000EC18053530681D4498B10379012B22788D
:10F1C00016D0022B09D00134AC42F7D100224021E5
:10F1D00005B0BDE8F040FDF78FBC4021FDF72EFCE7
:10F1E00030680134AC42E7D10028EFD105B0F0BD62
:10F1F0008168013490F910C001F00107417C8DF85D
:10F200000F20604601970DF10F0740220097F4F799
:10F2100079FBAC423068CFD1E6E700BF28AD0C08DF
:10F22000C8720024F0B59B4D85B02868002800F016
:10F230002E81D4228021FDF75FFC2868002800F091
:10F24000268180221146FDF757FC2868002800F02F
:10F250001E81A8228021FDF74FFC2868002800F0BD
:10F2600016813F228021FDF747FC2868002800F026
:10F270000E81D3228021FDF73FFC2868002800F092
:10F28000068100228021FDF737FC2868002800F065
:10F29000FE8040228021FDF72FFC2868002800F026
:10F2A000F6808D228021FDF727FC2868002800F0D9
:10F2B000EE8014228021FDF71FFC2868002800F052
:10F2C000E680A1228021FDF717FC2868002800F0C5
:10F2D000DE80C8228021FDF70FFC2868002800F09E
:10F2E000D680DA228021FDF707FC2868002800F08C
:10F2F000CE8012228021FDF7FFFB2868002800F055
:10F30000C68081228021FDF7F7FB2868002800F0E5
:10F31000BE80CF228021FDF7EFFB2868002800F097
:10F32000B680D9228021FDF7E7FB2868002800F08D
:10F33000AE80F1228021FDF7DFFB2868002800F075
:10F34000A680DB228021FDF7D7FB2868002800F08B
:10F350009E8040228021FDF7CFFB2868002800F026
:10F360009680A4228021FDF7C7FB2868002800F0C2
:10F370008E80A6228021FDF7BFFB2868002800F0C0
:10F380008680AF228021FDF7B7FB286800287ED059
:10F39000A6228021FDF7B0FB2868002877D0AE2296
:10F3A0008021FDF7A9FB2868002870D02022802149
:10F3B000FDF7A2FB2868002869D000228021FDF714
:10F3C0009BFB2868002862D0B0228021FDF794FBC7
:10F3D000286800285BD040228021FDF78DFB28683B
:10F3E000002854D000228021FDF786FB28680028E1
:10F3F0004DD010228021FDF77FFB28684FF48064F8
:10F4000000270DF10F0628B30379012B2BD0022B17
:10F4100004F1FF3215D094B2002CF6D18122802164
:10F42000FDF76AFB286848B1C8228021FDF764FB1C
:10F43000286818B1AF228021FDF75EFB012005B0DE
:10F44000F0BD8268402112F0010218BF0022FDF7D2
:10F45000F5FA2868013CA4B2002CD4D10028DDD1F3
:10F46000012005B0F0BD8268013C90F910E002F087
:10F47000010CA4B2417C402270468DF80F70CDE99A
:10F48000006CF4F73FFA2868002CBCD1E6E70020B6
:10F49000B4E700BFC8720024FCF7D8BFFCF7D6BFA2
:10F4A000FCF7D4BFFCF7D2BFFCF7D0BFFCF7CEBF50
:10F4B000FCF7CCBF01207047034620B1026812B1AF
:10F4C000D26902B1104793ED017AF6EE007A074B4C
:10F4D000B8EEC77AD3ED016AE7EE267AFDEEE77A59
:10F4E00017EE900A00F30B00704700BFFCB9002430
:10F4F000034620B1026812B1126A02B1104793EDBF
:10F50000027AF6EE007A074BB8EEC77AD3ED026ABC
:10F51000E7EE267AFDEEE77A17EE900A00F30B008D
:10F52000704700BFFCB90024034628B102681AB135
:10F53000516A09B19369184793ED037AF6EE007AA0
:10F54000064BB8EEC77AD3ED036AE7EE267AFDEEF6
:10F55000E77A17EE900A00F30B007047FCB900241D
:10F5600010B5044630B1036823B1DB6813B1BDE8C0
:10F570001040184704F0A4F8D4E9042390429941BC
:10F5800034BF0120002010BDD0B10E4B0E4A70B523
:10F5900006680D4682B0044633449B0A32F81300D5
:10F5A00064F0B0FAC5F381030022A1883046CDE9AA
:10F5B00000326B0905F013026EF038F902B070BD2D
:10F5C000704700BF0000FEA724A30C08D0B10E4B6B
:10F5D000F0B5076816460D4A0D463B4483B0044615
:10F5E0009B0A32F8130064F08DFAC5F38103A188F9
:10F5F000384605F01302CDE900366B096EF016F9B6
:10F6000003B0F0BD704700BF0000FEA724A30C08A4
:10F6100010B50409013C042C19D80F4A00F00F035F
:10F6200032F8140040FA03F212F0010211D0012264
:10F6300002FA03F3013B184078F0A2F8074B084A9E
:10F640001B5D184400EB400002EB800010BD002061
:10F6500010BD104610BD00BF18A30C08B4AB0C08B9
:10F66000D45E00242DE9F04F002104468BB05422D3
:10F67000A74875F02DF8A74B611EE01C1C4611F839
:10F68000012F551E052D88BF0022884244F8042B07
:10F69000F5D103F11002194651F8040B012800F0CE
:10F6A00029818A42F8D1194651F8040B022800F04A
:10F6B00017818A42F8D1194651F8040B032800F04B
:10F6C00005818A42F8D1194651F8040B042800F04C
:10F6D000F3808A42F8D1194651F8040B052800F04E
:10F6E000E1808A42F8D1002053F8041B062908BFA4
:10F6F00043F8040C9A42F7D1874F1A264FF0000ABC
:10F70000DFF80C8207F58065DFF8109298F80C405E
:10F7100054B32046FFF77CFF20B10523C6718371E7
:10F72000002303720321FFF72FFF002302E00133C0
:10F730001C2B37D015F83320A242F8D107EBC303B6
:10F74000D3F804440123D9F8F8200621C8F8104062
:10F75000D0189A4488F81420C9F8F80088F81610D0
:10F7600088F8153089F8F430013608F10C08F6B243
:10F77000202ECBD1BAF1000F11D0DFF8B8A14FF095
:10F78000000BDFF8B4919AF8EC306BB90BF1010B78
:10F790000AF1F40A09F58C79BBF1030FF3D10BB030
:10F7A000BDE8F08F0024CDE7BAF806004FF44037EB
:10F7B00064F0A8F9BAF8040064F0A4F9DAF8F030BB
:10F7C000564CF421012BCAF82830DAF8002001FB4E
:10F7D0000B41D4BF002301234FF0030CCAF81020C3
:10F7E000CAF81C300023CAF838308AF82C30CAF81E
:10F7F0003030CAF820308AF8483004930823CAE928
:10F8000005734FF48063CAF834304FF48073AAF85C
:10F8100024304FF48053CAE90FC3CB6E002B73D052
:10F8200093689E0003D591683D4B0B4093609368AD
:10F83000DD0014D43B4B3C491B689068B3FBF1F3EB
:10F840003A490133014041F0805191600493049B97
:10F850002BB1049B013B0493049B002BF9D19368CB
:10F86000D8001CD4F4234FF0010803FB0B43D96EDE
:10F8700041F01001D966196F41EA08011967F423B4
:10F88000916803FB0B4301F00401D86E00F01000F7
:10F89000014353D0DA6E42F01002DA6676E74FF099
:10F8A0000008ECE72249202491F89C0181F884416A
:10F8B000013081F89C0116E71D49342491F89C0120
:10F8C00081F87841013081F89C0104E7184935241A
:10F8D00091F89C0181F86C41013081F89C01F2E6BD
:10F8E0001349312491F89C0181F86041013081F87D
:10F8F0009C01E0E60E49302491F89C0181F85441C6
:10F90000013081F89C01CEE60B678AF8603087E70A
:10F9100048E9002438E90024CCAB0C08041B00247F
:10F92000C0FFFF5FA0000024400D0300C0FFFF6F79
:10F9300000E800240C1B002400000030D96E21F4E4
:10F94000817141F00201D9669368D90713D4784BCD
:10F950009A4200F0248303F580739A4200F01F83DB
:10F96000744B9B68DF0706D473498B6823F47C13C0
:10F9700043F440338B60714B71491B68D368194065
:10F9800043F208030B43D3609168936801F00401CC
:10F9900003F00803194300F06D82DAF81000DAF87A
:10F9A0001C30012B00F06983036B23F00F0303630A
:10F9B000F42303FB0B43DA6E22F0030242F0010250
:10F9C000DA66B8F1000F7FF4E1AE9AF86020CDF866
:10F9D0001480012A3FF4DAAE8268012196078AF882
:10F9E0006010816802D4CD0700F19482F421554A59
:10F9F000554B01FB0B41CD6E2A4042F00202CA6614
:10FA00008268134043F00043836083684F4A002BB1
:10FA1000C0F2F081F4214E4B4E4D4FF4005701FBE4
:10FA20000B414D484FF0030CCA6E22F0030242F026
:10FA30000102CA66DAF80820DAF80C60AA4218BF98
:10FA40009A424FF48065CAF878600CBF0123002306
:10FA5000CAF89CC0824208BF43F0010318308242BA
:10FA600008BF43F001031830824208BF43F001038E
:10FA70001830824208BF43F001031830824208BFA9
:10FA800043F001031830824208BF43F0010300F540
:10FA90005670824208BF43F001031830824208BF0B
:10FAA00043F001031830824208BF43F001031830CD
:10FAB000824208BF43F001031830824208BF43F07E
:10FAC00001031830824208BF43F00103183082421C
:10FAD00008BF43F0010300208AF86000CAF89800CC
:10FAE000CAE91F00CAE928004FF40060CAE92150A2
:10FAF0004FF480705546CAE923704FF40030174F19
:10FB0000CAF89400386845F8742F1BB9144B9A4210
:10FB100040F0DD84F423022103FB0B4383F8B11092
:10FB2000002113688AF8A81023F0010313601EE077
:10FB30000020024000600258006302580010005C80
:10FB400003C0F0FFFDEEFFFFC0FFFE3F00F8C3253E
:10FB5000100002402800024040000240802D002496
:10FB6000B80402403B681B1A052B00F2C9811368D8
:10FB7000DB07F7D4A94913680868A9496FF30F0098
:10FB80001940A84BB0F1005F43EA01030BD32E2EBE
:10FB900040F236833F3E132E05D8A348F040C007FD
:10FBA00001D5A24B0B4313602846536923F007038A
:10FBB0005361F2F7DDF9DAF8D03003F01F013F238B
:10FBC0008B408360DAF87420994B9A499A4E8A42A6
:10FBD00018BF9A4201F118010CBF012300238A4289
:10FBE00008BF43F0010318318A4208BF43F0010304
:10FBF00018318A4208BF43F0010318318A4208BF16
:10FC000043F0010318318A4208BF43F00103183161
:10FC10008A4208BF43F0010301F556718A4208BFCA
:10FC200043F0010318318A4208BF43F00103183141
:10FC30008A4208BF43F0010318318A4208BF43F0EB
:10FC4000010318318A4208BF43F0010318318A4288
:10FC500008BF43F0010318318A4208BF43F0010393
:10FC60007649A2EB010C7649DCF1000E4EEB0C0E4E
:10FC70008A4208BF43F00103911B4EEA03034E4240
:10FC80004E417049501A3343414241410B43009168
:10FC90006D49A2EB010CDCF1000141EB0C010B43BF
:10FCA00001916A49501A414241416948A2EB000C56
:10FCB0000B430291DCF10000664940EB0C00A2EB23
:10FCC000010CDCF1000143EA000341EB0C01DFF819
:10FCD0009CC1624514BF4FF0000C4FF0010C0B4368
:10FCE00002D1BCF1000F3ED046EA0E06009B334322
:10FCF000019E1E433346029E1E43D3B2304301434E
:10FD00005CEA010100F072831422083B0126DFF84F
:10FD100060C1B3FBF2F3504A9E401A449200DAF8F5
:10FD20007C30CAF8DC60802BCAE9352C00F00A81EF
:10FD3000DAF87830D8B2013B072B1060CCF80460B9
:10FD400000F20681461E002900F07585434B4449A8
:10FD500003449B0001220020B240CAE93831CAF8AE
:10FD6000E82018604A60F42301210020009703FB7B
:10FD70000B430A46C3F8D00083F8B1100AF1100310
:10FD80004FFA8BF1CAF85C50CAF8AC308E46354B4E
:10FD900004E001320C33072A00F00B81597D002961
:10FDA000F7D093F90D107145F3D100219E7D1869AC
:10FDB00006912D49019601EB8801D1F8E0549AF89B
:10FDC000601001293FF4E2AC4FF001018AF86010A5
:10FDD000DAF810108E68760740F11181F42303FBE6
:10FDE0000B43DA6E42F02002DA664FF000038AF825
:10FDF0006030CBE4059B01330593059B9342FFF4F0
:10FE000004AEF422002102FB0B42D36E23F0120356
:10FE100043F01003D3668AF86010B7E40010005C6A
:10FE20003F8010FE002D02000F030F00002D120076
:10FE300010000240280002401C5402580854025886
:10FE4000B8040240305402584454025858540258DE
:10FE50006C54025880540258009600163F960016C3
:10FE60004059025848E90024CCAB0C08945402587D
:10FE700080580258D068AE4B0340DAF8440043F093
:10FE80000303D360136923F001031361136923F0A3
:10FE9000704303431361A74B9A4278D003F58073F4
:10FEA0009A4274D0A44B9B6813F4403F14BF0123C3
:10FEB0000023002B00F0F280F2F7C2F9DAF81430D8
:10FEC0000146B3F5003F00F02A82B3F5403F00F051
:10FED0002A82B3F5803F00F02282984BDAF81000B6
:10FEE0001A6841F20303B3EB124FC0F0CF80944B7A
:10FEF0009942836800F2178123F4807383604EE592
:10FF0000F423202203FB0B43C3F8D020032283F801
:10FF1000B1203BE4826802F00D02012A1ED0DA6EA5
:10FF2000002142F01002DA661A6F42F001021A67ED
:10FF3000F42303FB0B43DA6E42F01002DA668AF810
:10FF4000601023E40023CAF878301360CCF8046012
:10FF50000023CAE93833CAF8E83004E78268794BED
:10FF6000794F134043F002038360032303603A6830
:10FF70008368DB077FF53AAD3B689B1A022BF7D904
:10FF80008368D907F4D5F42303FB0B43C7E76F4B12
:10FF90009B6813F4403F14BF0123002389E7654B9E
:10FFA0006B499B6889680B43DB073FF5E4AC674905
:10FFB000DBE4DAF810105F4B009F9942DAF8F0604A
:10FFC00059D003F58073994255D05B4882688B689D
:10FFD0005B073FF5DBAB9AF86030012B3FF4D6AB03
:10FFE00002F01F0240F221230125D3408AF860501D
:10FFF0002B4040F009818AF86030FFF7C7BB00282A
:020000040805ED
:100000004FEA906C0ADBC0F31306002E40F0F0803C
:10001000012606FA0CF6CF693743CF61AE091F27D8
:1000200005F01F050CF01F0C06F00C060CFA05FC81
:10003000029601F13006039607FA05F6DDE902574C
:100040007D5925EA0605029E45EA0C05BD518E68DC
:100050008D6806F0040605F00805354300F082803F
:100060008D68ED0732D508F1010800215FFA88F8A4
:100070008AF860108DE63548A8E7026BDAF8283078
:1000800022F00F02013B1343036391E4314B994289
:1000900042D8836823F44073836080E42E4B9A6DCA
:1000A00002F44032B2F5803F00F09281B2F5003F99
:1000B00000F07381002A7FF410AF1B681E017FF5EA
:1000C0000CAF07A8F2F7FCF8079906E7D1F8C05083
:1000D000C0F31306002825EA0605C1F8C050C2DAAD
:1000E000144DA94200F0218105F58075A94200F068
:1000F0001C81114D194FAE68BF68FF0740F1228186
:10010000F423002103FB0B43DA6E42F02002DA668F
:100110008AF86010FFF73ABB114B994200F2328126
:10012000836823F4407343F48073836037E400BF33
:10013000FCBFFFFF00200240006302580010005C7B
:10014000002D3101C0FFFF7F802D002400230240DD
:100150000021024021BCBE00004402580060025849
:1001600041787D01C60D4FF0070C01F1140706F030
:100170000405019E0295C0F30455AE400CFA05FC3F
:10018000029D7D5925EA0C053543029EBD51A44DC3
:100190002D6805F07045B5F1805FCD6800D0CD6861
:1001A0000D6E860605F0F845B5EB806F03D10D6E38
:1001B00025F000450D664D6E05F0F845AE4203D1C1
:1001C0004D6E25F000454D668D6E05F0F845AE424A
:1001D00003D18D6E25F000458D66CD6E05F0F84596
:1001E000AE427FF43DAFCD6E25F00045CD6637E7DA
:1001F00090FAA0F60127B6FA86F607FA06F60AE79D
:10020000282E7FF6D0ACCCE48B68DD0733D48D6824
:10021000844B1D421FD18D68834B2B4043F001035B
:100220008B603D688368D80602D0804B994222D00B
:100230007D480B68DB071ED48B68DB0704D48B6812
:10024000034043F001038B603B685B1B022BF0D93A
:100250000B68DB07EDD4F42303FB0B43DA6E42F0AB
:100260001002DA661A6F42F001021A6700238AF858
:100270006030FFF78BBAF4206D4B6C4D00FB0B40E8
:10028000A942C76E03EA070343F48073C36600D133
:1002900032B9F42303FB0B43DA6E22F48012DA66E0
:1002A000F42303FB0B43DA6E12F4805200F0AF80AC
:1002B0001A6F22F006021A67DAF85C0000245D4B20
:1002C000DAF83C20C3635C4B03645C4BC3641C23BF
:1002D0000B604B688AF8604043F010034B60CB68BA
:1002E00023F003031343CB6090F83430012B0CD080
:1002F000012380F8343090F83530012B00F0348140
:100300004FF4006380F834404365DAF81020464B20
:1003100091680B4043F004039360FFF737BA1B0C5E
:10032000B1FBF3F1D9E58108D7E5454D454FDFF83D
:10033000FCC0AE68BF68DCF808C047EA0C07FF07DE
:100340003FF5DEAEDFF81CC106F0E077604500F057
:100350009180DFF814C1604500F0AA80DFF80CC17D
:1003600060457FF480AE70023FF57DAE3648814235
:100370007FF479AEA96821F0E071394341F480013E
:10038000A96070E6314B994283682AD823F4407300
:1003900043F400738360FFF702BBDA6C186802F065
:1003A0004052400701D5002A33D0294B1B68DB059A
:1003B00003D5B2F1805F00F0D580254B1B689F0309
:1003C0007FF58BAD234BB2F1005F08BF194684E582
:1003D0001B689D007FF581AD07A8F2F70BF809991E
:1003E0007BE543F440738360FFF7D9BA1A48103BAA
:1003F00010441822A828B3FBF2F300D80833174A98
:100400000126DFF86CC01A449E40920087E41A6708
:1004100052E71B681249C3F3C103D9405DE500BF31
:100420000010005C3F000080C0FFFF7F0021024001
:10043000FEF0FFFF010004085500040859000408FD
:1004400000230240002002400060025881F0FA02BE
:100450000044025800127A00F0FBFDBF0082001039
:100460000090D003000084CB000052C70000B8CF3A
:100470008008024030023FF5F6AD844881427FF4A7
:10048000F2AD834983480968B1FBF0F1A8680131F6
:1004900020F0E0704900384340F40000A860069165
:1004A00002E006990139069106990029F9D1DAE5A9
:1004B000F6013FF5D8AD754881427FF4D4ADA96807
:1004C00021F0E071394341F08071A960CBE5724BB6
:1004D0007248824218BF9A4200F114000CBF0123F7
:1004E0000023824208BF43F001031430824208BF58
:1004F00043F001031430824208BF43F0010314307B
:10050000824208BF43F001031430824208BF43F027
:1005100001031BB9624B9A4240F09381F4210220FF
:10052000604B01FB0B41134481F8B1001421B3FB74
:10053000F1F38340106842F2A0516FF310100143B1
:1005400000208AF8A80028461160CAF8D030F1F7D8
:100550000FFDDAF8D03003F01F0101238B40436018
:10056000FFF730BB5049B8E4036840314F4A504D63
:10057000876DAB4218BF934205F130050CBF0122D5
:100580000022AB4208BF42F001021835AB4208BF5F
:1005900042F001021835AB4208BF42F001021835A3
:1005A000AB4208BF42F0010205F55675AB4208BFE9
:1005B00042F001021835AB4208BF42F00102183583
:1005C000AB4208BF42F001021835AB4208BF42F00F
:1005D00001021835AB4208BF42F001021835AB42A8
:1005E00008BF42F001021835AB4208BF42F00102D9
:1005F000142505FB06F8022580F8355044652D4C7E
:100600002D4DA34208BF42F00102A4F59564AB4210
:1006100018BFA3420CBF0124002401D0002A4DD0F2
:100620001D6825F001051D60002C78D0D0F86CC045
:10063000D0E919566E60BCF1000F04D0D0E91C5609
:100640006E60002C73D0C56D05F01F0E3F2505FAB6
:100650000EF5BD601D6825F480251D608568C3F812
:100660000480402D00F0F4809960C3F80C9014B918
:10067000002A00F09880196821F01E0141F016014F
:100680001960196841F008011960BEE00060025865
:10069000A0000024400D0300085402581C540258C6
:1006A00094540258F8ABFDA700093D0058000240E1
:1006B00040000240B804024028000240684DDFF8C4
:1006C000A8C1634518BFAB420CF1140C0CBF012547
:1006D0000025634508BF45F001050CF1140C634586
:1006E00008BF45F001050CF1140C634508BF45F047
:1006F00001050CF1140C634508BF45F00105D3F862
:1007000000C02CF0010CC3F800C0DFF864C16345E1
:1007100008BF45F0010515B9524DAB4243D1D0F8A1
:100720006CC0D0E919566E60BCF1000F86D1002A6A
:1007300089D14B4DDFF830C1634518BFAB420CF196
:10074000140C0CBF01250025634508BF45F00105C9
:100750000CF1140C634508BF45F001050CF1140CB5
:10076000634508BF45F001050CF1140C634508BF53
:1007700045F001050CF1140C634508BF45F0010577
:1007800015B9384DAB420ED1C56D05F01F0C0125D2
:1007900005FA0CF57D608568C3F80480402D5BD0B8
:1007A0009960C3F80C902E492F4DAB4218BF8B4275
:1007B00005F114050CBF01210021AB4208BF41F037
:1007C00001011D6825F00E0545F00A051D60274D45
:1007D000AB4208BF41F001011435AB4208BF41F004
:1007E00001011435AB4208BF41F001011D6845F01D
:1007F00004051D601E4DAB4208BF41F0010111B957
:1008000018498B4212D1D0F86CC0016E0868C2033F
:1008100003D5086840F480700860BCF1000F05D073
:10082000DCF8001041F48071CCF800101A6842F036
:1008300001021A6069E50F4B0F4903449B00FFF763
:1008400089BA4023C1F8D03081F8B1C0FEF79EBF0D
:10085000C3F80890D9600AE7C3F80890D960A2E706
:1008600008540258945402581C54025844540258D4
:10087000805402583F82001040090240036810B5BE
:100880001A790446022A03D000232360237110BD85
:10089000987AFEF7BDFE0028F6D040F61A610022D5
:1008A000C18020210272FEF76FFE002323602371B6
:1008B00010BD00BF2DE9F04FBA4E85B0BA4CA6422C
:1008C00056D21D4602E00C36A64251D273798B42B5
:1008D000F9D13379834201D00028F4D1F3799342DE
:1008E000F1D13468002C43D0002326606360A360FC
:1008F000E36023616361A361E36133792371012BB9
:1009000096F806B0C4F808B0317AE16032D0022B14
:100910002ED1F07AFEF77CFE96F90970A061B07ACC
:100920002774FEF775FE06466061F0B1DFF8948229
:1009300007EB47017B0058F8319008EBC1010193A8
:10094000B9F1000F11D0887DE8B10E2200230D21EE
:100950003046F2713372B571FEF716FE3368B28815
:100960009A61204605B0BDE8F08F2046FFF786FF6C
:100970000024F6E7F07AFEF74BFE727AB37AA061B4
:1009800022746374EDE7B1F808A0504663F0BAF83A
:1009900001214FEA5A100AF01F0A023801FA0AF13F
:1009A000092812D8DFE810F0F6001100EE00180157
:1009B0001001E600E000D800D0000A007B4BD3F81D
:1009C0009C0020EA0101C3F89C107B00D91908EBB8
:1009D000C1014879FEF71CFE791CCBB20146019398
:1009E00018B1037240F60A30C8807B000291D81912
:1009F00008EBC000C079FEF70BFE02990346039096
:100A000020B1019A027240F60A50D8807B00029110
:100A1000D81908EBC0008079FEF7FAFD02998246EA
:100A200028B1019B037240F60A40AAF806007B0039
:100A3000D8191BF0040308EBC0000293807A024629
:100A4000084614BF4E212E21FEF7C0FD03987B00FF
:100A50002E2103EB070B08EBCB0B9BF80B20FEF7CB
:100A6000B5FD50469BF80C200E21FEF7AFFD9BF81C
:100A700004A0BAF1000F40F0ED80D9F8002022F078
:100A80000102C9F800204A4A914500F0C180494A54
:100A9000914540F0AC80454AD2F8901041F4804135
:100AA000C2F89010D2F8901021F48041C2F8901052
:100AB000029B002B40F098804FF000714FF0807245
:100AC000D9F80C0040F00040C9F80C00D9F8080033
:100AD00020F4F070C9F80800D9F80000C00727D446
:100AE000D9F80800344B034034481843C9F80800CB
:100AF000D9F80C00C30005D4D9F8000040F48050A8
:100B0000C9F80000D9F80C0011432D4A02400A43ED
:100B100042F08862C9F80C20D9F8002022F4006263
:100B2000C9F80020D9F8502022F00102C9F850205D
:100B3000BAF1000F40F09B807B003B4408EBC308F8
:100B4000012388F8163000E7184BD3F8880020EA14
:100B50000101C3F8881038E7144BD3F88C0020EA61
:100B60000101C3F88C1030E7104BD86F20EA010167
:100B7000D9672AE70D4BD3F8940020EA0101C3F8A6
:100B8000941022E7094BD3F8800020EA0101C3F852
:100B900080101AE7054BD3F8980020EA0101C3F84A
:100BA000981012E7A0020008500400080044025800
:100BB0000030014000380040E0FFBF8F07000020F8
:100BC000FFFF39D8CC0200243E4BD3F8900020EA36
:100BD0000101C3F89010F8E63A4BD3F8840020EAFC
:100BE0000101C3F88410F0E600210A4668E7364A9E
:100BF00091451BD1334AD2F8901041F40041C2F81C
:100C00009010D2F8901021F40041C2F890104FE7F4
:100C10002C4AD2F8981041F48051C2F89810D2F8BA
:100C2000981021F48051C2F8981041E7274A914565
:100C300027D0274A914532D1224AD2F8981041F460
:100C40008011C2F89810D2F8981021F48011C2F8DF
:100C500098102DE75046FEF7DBFC20B1019B40F6D3
:100C60000A620372C2800D21FEF78EFC05E7504632
:100C7000FEF7CEFC00283FF45FAF026883889361E3
:100C80005AE7104AD2F8981041F40051C2F898106F
:100C9000D2F8981021F40051C2F8981008E70D4AD4
:100CA00091457FF405AF02F50C32D2F89C1041F06B
:100CB0002001C2F89C10D2F89C1021F02001C2F84B
:100CC0009C10F5E600440258003C0040003401400E
:100CD0000050014000140058084B53F8203029B14F
:100CE00053B19A88196812048A617047002BFCD0AE
:100CF0001A689B8893617047704700BFC0AB0C08AF
:100D00002DE9F04FDFF84C9283B099F824A1BAF1A5
:100D1000000F02D003B0BDE8F08FD9F82041237C4A
:100D2000002BF7D199F8B9B2D44699F8B87209F501
:100D30002F7099F8BAE201228349CDE900A4DA467E
:100D40008378C578C3F1FF032C469BB293B1B0F80A
:100D50000080C3F1FF037D4E05FB03F3A6FB08B63D
:100D60001B127609052E00F2EA80DFE806F0D5BAFC
:100D7000A1856B4EAE46AB462B46A24601252746C3
:100D800000951E0246EA0446172446EA0B060CEBC1
:100D9000040802FA04F5A8EB0403013C35429BB2B7
:100DA00008BF012503F12A0318BF022541F823508B
:100DB000631CEED10430664B0CF1180C98421FFAFC
:100DC0008CFCBDD14FF44063D346DDF800A0A9F8F8
:100DD000BC348023019CA9F8BE34BAF1000F05D0C1
:100DE00089F8BAE289F8B9B289F8B87299F8C034CA
:100DF000002B8FD0204640F62B41F4F7A1FA204675
:100E000003B0BDE8F04FF4F713BB504EEF1A5FFA92
:100E100083FA1C462B46A6FB08E56D09C5EB0515B4
:100E2000A8EB8505ADB2C5F13C0507FB05F51F46EE
:100E3000A6FB05650AEB55155FFA85FE0125F3460D
:100E400000959EE7414FEE1AAB465FFA83FA1C46C7
:100E5000A7FB0853DE465B09C3EB0313A8EB830330
:100E60009BB203FB06F6A7FB063701230AEB5717D5
:100E70000093FFB23B4684E7344EA5EB030EAB462E
:100E8000DFB2A6FB08546409C4EB0414A8EB840485
:100E9000A4B2C4F13C040EFB04F4DE46A6FB0464D9
:100EA00007EB54145FFA84FA01240094544668E76F
:100EB000DFF898E0EE1AAA46DFB2AEFB08B56D097E
:100EC000C5EB0515A8EB8505ADB205FB06F6AEFB37
:100ED000065E012507EB5E1E00955FFA8EFEF34667
:100EE0004FE71A4EEF1A5FFA83FEAA469B46A6FB0F
:100EF00008535B09C3EB0313A8EB83039BB2C3F155
:100F00003C0303FB07F70123A6FB076700930EEBE7
:100F10005717FFB23B4634E7EC1A0C4E5FFA83FEDC
:100F20009B4608FB04F42B462F46A6FB04640EEBFD
:100F300054145FFA84FA01240094544621E754467D
:100F40003B46F3461DE700BF3C0700308988888890
:100F5000BCEC002400E800240021182070B5F3F751
:100F6000FDFFC36813F080730DD12B4C224602E0C5
:100F700001330C2B2CD0D1681432C901F8D51422BE
:100F800002FB034400E00446244E2046F3F780FFB2
:100F90000546C6F82001D8B12079FEF739FBC6F81E
:100FA000C40420B140F21523C38000230372227AC7
:100FB0004E21FEF70BFB96F8C834022B23D0032BEF
:100FC00007D1FBF729FB2846F4F792F96423036065
:100FD00070BDFBF7E9FA10B986F8C00470BD43F2A2
:100FE000AC0200210E4873F073FB96F8C834012B55
:100FF00003D10C4BFF22C3F8A820012386F8C0348C
:10100000BDE870407CE6FBF707FB2846F4F770F973
:101010000023036070BD00BF2C03002400E80024FF
:101020003C0700303C370030F8B5354DD5F820414D
:1010300074B195F8243106465BB162685379032B8D
:101040005BD8DFE803F04B4E5102136840331E605B
:10105000F8BD63682B4A1B69C3F3032352F82300CE
:10106000E3685F68EFF31183102282F31288DFF8E0
:101070009CC062681CF80000234992F805C031F852
:101080001C10D2F800C001F4F051DCF80C2022EA68
:101090000102E168CCF80C203A5822F001023A50E3
:1010A0000A691F2A23D94868203A202101FA02F24E
:1010B000C260DBB283F3118800222368227458686F
:1010C00090F83D30012B01D16BF08EFCD5F820411A
:1010D0000022E3681A77FBF79FFAAEE71368343310
:1010E000B5E713683833B2E713683C33AFE74868B5
:1010F000202101FA02F28260DBE700231B60FFDEA1
:1011000000E8002418A10C0838A10C084CA20C0817
:1011100010B5224CD4F8203183B194F824216AB15F
:1011200094F8C824032A0AD0022A10D0002384F895
:101130002431FBF739FA08B984F8C00410BD5A68A5
:101140005379032B27D8DFE803F023201D185A68B2
:101150005379032B1FD8DFE803F00D0A0702136849
:10116000403300221A6010BD13683C33F9E713685E
:101170003833F6E713683433F3E7136840336422F7
:101180001A6010BD13683C33F9E713683833F6E78B
:1011900013683433F3E700231B60FFDE00E800240C
:1011A0002DE9F04F0021A7B04FF00A0A7F4D0C4601
:1011B0007F4ECDF800A083E0B9F1000F16D14CF0BE
:1011C000400CBEF18C0F86F808C000F2D980621C7A
:1011D000983498320DEB040974464FF0040E6A44BB
:1011E00009F88CEC04F1020E02F88CCCBEF18C0FE5
:1011F00040F0020C00F2C48004F198024FF005099F
:101200006A4402F88BCC04F1040C02F88C9CBCF10B
:101210008C0F00F2B5800EF1980E4FF0060B9B007C
:10122000EE44DBB20EF88CBC04EB0B0E02F8897CAA
:10123000BEF18C0F00F2A48004F19C0C4FF0070A61
:10124000EC440CF88CAC02F8873C04F108038C2BBE
:1012500000F296800EF1980C0DEB0C0E0EF88C9CA3
:1012600002F8850C04F10A008C2800F2898004F150
:10127000A0036B4403F88CBC02F8837C04F10C02DD
:101280008C2A7DD804F1A20004F1A303144668441B
:101290006B4400F88CAC03F88C8C480901F01F07F4
:1012A000012255F82030BA4023EA020345F82030E5
:1012B000009B013B00936DD00131B1F5F07F69D205
:1012C0003C222846F8F7F4FD011E5CDB394BC1F3E4
:1012D000072096F808C0CFB233F8112004F1020EAF
:1012E0000CF040090196D3B24FEA122852073FF59D
:1012F00063AFB9F1000F03D10CF038029A4217D056
:101300000CF0870CBEF18C0F4CEA030C86F808C079
:1013100036D8631C04F1980298330DEB02040422C2
:101320006B4404F88C2C74460EF1020E03F88CCC3E
:10133000BEF18C0F24D804F198030DEB03020523B2
:1013400002F88C3C231D02F88B0C8C2B18D80EF164
:1013500098000DEB000E06200EF88C0C201802F8F9
:10136000897C8C280CD8621D04F19C03044607205C
:1013700098326B446A4403F88C0C02F88C8C8CE72E
:101380006FF0004489E71CB9204627B0BDE8F08F14
:10139000074B01930198234603AA002100686AF0D5
:1013A000CDF9012027B0BDE8F08F00BFCCEC0024C0
:1013B0002C96002438960024F0B5244C83B0206885
:1013C00008B1A3790BB103B0F0BD012384210DF165
:1013D0000702A371FBF730FA227A042120680A433E
:1013E000FBF78AFB0DF1070284212068FBF724FA42
:1013F0009DF8073013F00405F4D13C222946144827
:10140000237273F065F913482A46134F4FF0010E0B
:1014100000F570760E4D30F8023F02F01F014FEAE2
:10142000521C01323B400EFA01F19BB223B155F838
:101430002C300B4345F82C30B042ECD1FFF7B0FE16
:101440000028FBD1A07103B0F0BD00BF2C96002492
:10145000CCEC00243696002404DFFFFF70B53D4D30
:1014600082B02C686CB32B79012B3DD0022B2AD192
:10147000082294F910300021EA718DF8052040F21D
:10148000044203EB43038DF80410ADF80620324A02
:1014900052F83300A3689A073FD5042300210DEBCF
:1014A0000302F2F73DFFA3689B071FD53C22FF21F3
:1014B0002A4873F00DF96B791BB9FFF77DFF012303
:1014C0006B7102B070BD0DF10302A0212046FBF745
:1014D000B3F99DF8033003F00503012B37D0002B3F
:1014E0002FD12C680822C4E74822C2E71C4A4FF4D7
:1014F000FA701C4B12681C4900FB02F24868A3FBFF
:10150000023292094B681B1A9A42FBD26369002B84
:10151000CCD01A689B889361C8E763691BB11A68CD
:101520009B881B0493610E4B0F491A680D4BD20028
:101530004E68A3FB023292094B689B1B9A42FBD276
:10154000ABE70A4A40F2DC5312689A42B9D92C68D8
:1015500048228EE72C960024CC020024CCEC0024F8
:10156000CC300024D34D6210001000E0D0300024B5
:101570002DE9F0412D4D82B0AB7903B1FEE7012298
:1015800004460E462868AA711946EA7902F0F70265
:10159000EA71FBF7B1FAE2B2074609212868FBF7C6
:1015A000ABFAB4F5807F3BD0502208212868DFF8E1
:1015B0008080FBF7A1FA0BE0D8F80C23B8F81033C1
:1015C000516901EA030023EA010343EA00439361FE
:1015D0000DF10702A0212868FBF72EF90028EBD0B7
:1015E0009DF8074014F02004E6D1E2B20A212868F1
:1015F000FBF782FA32190134C0212868FBF71CF985
:10160000362CF2D13FB9EA793946286802F0F70260
:10161000EA71FBF771FA0023AB7102B0BDE8F0810B
:1016200040220A212868FBF767FABDE72C960024C0
:10163000D45E00242DE9F04F5E4DC3B0AF7907B101
:10164000FEE7EA79044601230E4602F0F702394626
:101650002868EA71AB71FBF74FFA0923FF2C01AA46
:101660005470137073D9A40804F0C0084FF0020C32
:101670004FF0000E4FF00A0B0DF1050A4FF00B0969
:1016800011E0B1F5827F02F80CB00AF80C0016F8F0
:101690000E0017D80EF1010E02F804908C46D055BA
:1016A000BEF1360F17D00CF10204634648EA0E0073
:1016B0000CF10401B4F5827F03F10307C0B203F11A
:1016C0000603DED90EF1010E6FF000413A4BBEF178
:1016D000360F8C46E7D1B3F5827F67D80823A02068
:1016E00053540DF105010CF1020301F80C002C68B4
:1016F000324894F9101001EB410150F83100A16813
:10170000890726D50021F2F70BFEA3689B0736D583
:101710002B4C0BE0D4F80C23B4F81033516901EAD8
:10172000030023EA010343EA004393610DF103023E
:10173000A0212868FBF780F80028EBD09DF8033043
:1017400013F02003E6D1AB7143B0BDE8F08FB8468B
:101750008CE7616919B18E880F683604BE6119493A
:10176000194F0E681949F600D7F804C0A1FB0616F8
:10177000B6097968A1EB0C018E42FAD2C2E7114A90
:101780004FF4FA70114B12680F4900FB02F24868DF
:10179000A3FB023292094B681B1A9A42FBD263697F
:1017A000002BB5D01A689B889361B1E76FF00043B6
